:020000022000DC
:107000000000042045020A0085020A000D150A004E
:1070100089020A008B020A008D020A0000000000AB
:10702000000000000000000000000000D5000A0081
:1070300091020A0000000000F5000A0095020A0013
:1070400045040A0097020A00BDDB0900D5DB0700F2
:1070500097020A0097020A0055DE090097020A000B
:1070600097020A0097020A0097020A0097020A0094
:1070700097020A0097020A0097020A0097020A0084
:1070800097020A004DFE090097020A0097020A00C3
:1070900097020A0097020A00EDBD090097020A0054
:1070A00097020A0097020A0097020A0097020A0054
:1070B00097020A0097020A0000000000000000008A
:1070C00097020A0097020A0097020A00C50A0A00FE
:1070D00097020A0097020A0097020A00BD7C02008C
:1070E000CDDB090097020A0097020A0000000000A9
:1070F0000000000097020A0000000000D90A0A0000
:10710000000000000000000000000000000000007F
:10711000000000000000000000000000000000006F
:10712000000000000000000000000000000000005F
:10713000000000000000000000000000000000004F
:10714000000000000000000000000000000000003F
:10715000000000000000000000000000000000002F
:10716000000000000000000000000000000000001F
:10717000000000000000000000000000000000000F
:1071800000000000000000000000000000000000FF
:1071900000000000000000000000000000000000EF
:1071A00000000000000000000000000000000000DF
:1071B00000000000000000000000000000000000CF
:1071C00000000000000000000000000000000000BF
:1071D00000000000000000000000000000000000AF
:1071E000000000000000000000000000000000009F
:1071F000000000000000000000000000000000008F
:1072000010B5054C237833B9044B13B10448AFF3E0
:1072100000800123237010BDFC6C002000000000E2
:107220003CB00D0008B5034B1BB103490348AFF355
:10723000008008BD00000000006D00203CB00D0083
:10724000A3F5803A704700BF174B002B08BF134BC4
:107250009D46FFF7F5FF00218B460F461348144A61
:10726000121A8EF0A3FE0E4B002B00D098470D4B48
:10727000002B00D098470020002104000D000D488D
:10728000002802D00C48AFF300808EF0B7FD20003C
:10729000290079F019F88EF081FC00BF0000080089
:1072A000000000000000000000000420FC6C002032
:1072B0003C8B0120000000000000000008B50146E2
:1072C000014800F0F3FA08BD346D002038B5064BD4
:1072D0001D780024AC4205D2204600F0EDFD0134BB
:1072E000E4B2F7E738BD00BF306D00202DE9F04F64
:1072F00095B0074601939146002A00F0AA805A4BA8
:1073000093F81C41A21C83F81C2193F81D61751C85
:10731000EDB246F080066A1C83F81D2145F0800519
:1073200093F81E8108F1010283F81E213E220021FC
:1073300004A88EF03BFE4FF0080A8DF80CA00B233A
:107340008DF80D3002238DF80F308DF810308DF848
:1073500011304FF0090E8DF814E004208DF815005F
:107360004FF0010C8DF818C08DF819308DF81A30D7
:1073700005228DF81D2024218DF81E104FF0200BC2
:107380008DF820B08DF821C08DF822208DF82310C3
:107390008DF824C08DF827008DF828108DF829303D
:1073A0008DF82A308DF82B208DF82C1006218DF8C1
:1073B0002D1007218DF830108DF831204FF0030C7F
:1073C0008DF833C08DF834A04FF0100C8DF836C016
:1073D0008DF837E08DF838008DF83B300A208DF8B5
:1073E0003C008DF840108DF841208DF8433040204E
:1073F0008DF844008DF847108DF848208DF84A30FC
:107400008DF84B008DF80E408DF816403B7D8DF8C1
:107410001C30631CDBB28DF826308DF82E408DF8C1
:107420002F308DF832608DF839308DF842808DF82C
:107430004950B9F1000F12D0019B412B11D94224C0
:10744000224603A948468EF089FD204615B0BDE8C6
:10745000F08F4FF0000845464646444666E7422016
:10746000F4E70020F2E700BF346D0020A0F1100027
:10747000FFF73CBF00B583B08DF8071003685B6869
:1074800001220DF10701984703B05DF804FB407D30
:10749000FF2809D010B500F0D7FC044608B12046FB
:1074A00010BD79F0E5FCFAE700207047407DFF2829
:1074B0000BD000B583B00DF1070100F0EFFC38B13F
:1074C0009DF8070003B05DF804FB4FF0FF307047F4
:1074D0004FF0FF30F6E7407DFF280FD000B583B0B6
:1074E00001220DF1070100F0BDFC20B19DF807005D
:1074F00003B05DF804FB4FF0FF30F9E74FF0FF30C9
:107500007047407DFF2803D008B500F0D5FC08BDCA
:107510007047F8B5437DFF2B18D006460D46174639
:10752000144603E0381BF8BD79F0A2FC002CF9D01A
:10753000707D00F05BFC0028F4D022462946707D67
:1075400000F018FD0544241AF0D0EDE70020EAE72A
:10755000407DFF2803D008B500F030FD08BD0020B5
:1075600070470000002242604FF47A71816002751A
:10757000044A02F10801016030320261FF224275C3
:10758000704700BF48BC0B00012800D0704708B509
:107590004FF6FF73994200D008BD0248FFF7E2FFA3
:1075A000FAE700BF186D0020437DFF2B02D10A4B84
:1075B0001B7803B1704710B5591C074A1170437509
:1075C00000F110040549204600F000FA2146044865
:1075D00000F04AF910BD00BF306D002038BC0B0030
:1075E000346D002008B5FFF7DFFF08BD10B5044675
:1075F000044800F0EDF8044B00221A70FF23637575
:1076000010BD00BF346D0020306D002010B5407DEE
:10761000FF2808D000F0EAFB044608B1204610BD60
:1076200079F026FCFAE70024F8E701B900B17047C9
:1076300000B583B0694600F0F9FB009BB3F5966F87
:1076400002D003B05DF804FB00F050FBF9E708B589
:107650004FF6FF710120FFF797FF08BD70B44FF69A
:10766000FD730B60047804F14003DBB2012B58D9A1
:10767000F42C5AD814F0800F0ED101250122954226
:1076800022DD835C03F0C006802E54D103F03F035B
:1076900043EA84140132F2E704F0E003C02B0BD07C
:1076A00004F0F003E02B0BD004F0F803F02B3FD1F3
:1076B00004F007040425E1E704F01F040225DDE7D8
:1076C00004F00F040325D9E7012D0DD0022D10D0B1
:1076D000032D16D0042D1CD0A4F55843B3F5006F2C
:1076E0002CD30C6068B21EE07F2CEFD94FF0FF3036
:1076F00019E0A4F18003B3F5F06FE9D34FF0FF3048
:1077000011E0A4F50063B3F5784FE3D34FF0FF30F9
:1077100009E0A4F58033B3F5801FDDD34FF0FF30CF
:1077200001E04FF0FF3070BC70474FF0FF30FAE7D8
:107730004FF0FF30F7E74FF0FF30F4E74FF0FF3046
:10774000F1E72DE9F04182B006460F46904600254C
:107750002C4613E0013411E0691C414521DAA3F500
:10776000803301939A0AA2F5205227F81520C3F31B
:1077700009030235A3F5105327F811303019335D92
:107780007BB101A9FFF76AFF0028E3DB0444019BFA
:10779000B3F5803FE0D2454503D027F815300135D9
:1077A000ECE7284602B0BDE8F081034690F85001AE
:1077B0000B2808D849B1421C83F8502100F1480237
:1077C00043F82210704700207047002070470000E7
:1077D000F0B589B00446214F03AD3E460FCE0FC52C
:1077E00033682B80254603AE0FCE0FC533682B8040
:1077F0006D4607F1140393E8070003C504F118056B
:107800006B4603CBA061E16184F8202065614FF4F1
:107810008073A4F81A310923A4F81831002584F8DC
:107820001C51012384F81E3184F81D312022294681
:1078300004F598708EF0BAFB40F20943C4F8203189
:10784000074BC4F82431074BC4F82831C4F82C5135
:10785000042384F8503109B0F0BD00BFACBC0B006C
:107860007CBC0B008CBC0B0038B504460846616933
:10787000B4F8182103681D68B4F81A319B1A9BB23A
:107880000A4494F81C11A84768B10346B4F81821BB
:1078900013449BB2A4F818316269538094F81C31E8
:1078A0001371012038BD0020FCE7000070B50446CC
:1078B0000D46FFF78DFFEF2323710223637101262D
:1078C000A6714FF4E1310448FFF76EFE284600F040
:1078D000FBF9304670BD00BF186D0020F0B589B0CF
:1078E0000D46D0F82C0130B120220231FFF729FFDC
:1078F000C0B209B0F0BD684600F0FCF907460026AA
:107900001DE0124B0FCB0DF1200C0CE90F0063466C
:10791000334413F8203CA200134103F00F0372001C
:107920000132C4F101010A44634413F8103C25F804
:1079300012300134E4B2012CE3D90136F6B2BE4272
:1079400001D20024F7E77800C0B2D2E798BC0B0060
:1079500010B5044681B10B4603291BD090F8502185
:107960008A421DD94833202200F5AA7150F823001D
:10797000FFF7E7FEC3B204E0D0F82031A0F854319D
:10798000012301335B0043F44073A4F8523104F542
:10799000A97010BD00F5A971FFF7A0FF0346F0E73D
:1079A0000020F6E700487047346D0020014B58690D
:1079B000704700BF346D002008B50A4601460248F2
:1079C000FFF7C6FF08BD00BF346D002010B50446A8
:1079D0000248FFF7EAFE207110BD00BF346D0020A1
:1079E000024B53F8200000B1C0687047C86E0020F9
:1079F00038B50C4611461A46074B53F8203033B1C0
:107A00001D6935B1BDF810302046A84738BD0020AB
:107A1000FCE70020FAE700BFC86E002038B50C462E
:107A200011461A46054B53F820302BB15D691DB144
:107A3000BDF810302046A84738BD00BFC86E0020F2
:107A40000020704790F860007047000008B5044BB4
:107A5000186810B1FFF7F6FF08BD0020FCE700BF73
:107A6000D06E00202DE9F84304461D46204B1868CF
:107A7000A0B3884616462C2303FB0403D3F82090BA
:107A8000B9F1000F2CD02C2303FB04035F6A57B31A
:107A90002C2303FB0404A46A3CB348468FF05AFD30
:107AA0000246072800D90822494640468EF056FA79
:107AB00038468FF04FFD02460F2800D91022394674
:107AC00030468EF04BFA20468FF044FD02460328E4
:107AD00000D90422214628468EF040FABDE8F883FA
:107AE000DFF81890CFE7034FD2E7034CD5E700BF8C
:107AF000D06E0020D8BC0B00E8BC0B00CCBC0B0047
:107B000038B5114B1D68E5B104462C2303FB005327
:107B10005B692BB198472C2303FB045585F8320091
:107B2000094B1A682C2303FB042393F832500DB140
:107B3000284638BD00233A220221204601F06CF885
:107B4000F6E70025F4E700BFD06E0020074B1B6866
:107B500053B110B42C2404FB0030C36A0B60038EB5
:107B600013805DF8044B7047704700BFD06E002053
:107B700008B500232022052101F04EF84FF0FF3018
:107B800008BD000038B50446084611461A46074BA2
:107B90001B6833B12C2505FB0434E3691BB19847FE
:107BA00038BD0120FCE70120FAE700BFD06E0020BD
:107BB000024608461946094B1B6843B110B52C24F0
:107BC00004FB023293682BB1029A984710BD4FF024
:107BD000FF3070474FF0FF30F8E700BFD06E002055
:107BE000024608461946094B1B6843B110B52C24C0
:107BF00004FB0232D3682BB1029A984710BD4FF0B4
:107C0000FF3070474FF0FF30F8E700BFD06E002024
:107C100008B5054B1B682BB12C2202FB0030036911
:107C200003B1984708BD00BFD06E002008B5074BD0
:107C30001B6833B12C2202FB003083691BB19847CB
:107C400008BD0120FCE70120FAE700BFD06E00204C
:107C500010B582B04FF08043D3F8384400238DF83C
:107C6000043001A878F070FB074B0093684678F069
:107C7000DDFB78F0ABFB14F0010F01D102B010BDB9
:107C8000002005F097F9F9E78D7C020008B505F0B2
:107C900091F908BD08B5084B402283F8272300203E
:107CA00003F022FCFFF7D4FF00214FF0FF3004F077
:107CB000B9F8FFF70BFBF7E700E100E008B500209B
:107CC00004F054FF08BD000000B583B00023019309
:107CD00003220092C8220349034877F027FA03B031
:107CE0005DF804FBECBC0B00957C020008B579F054
:107CF000EDFC08BD4FF08052536E1BBA0360136E4B
:107D00001BBA43600820704700487047F4BC0B0062
:107D100038B5224B1B68002B37D01546012936D1C8
:107D20001478C4F34114012C1AD0022C31D15278AA
:107D3000012A03D0022A08D0012029E09A6952B30F
:107D40001378294604F0F4F922E0AB88072B01D020
:107D500000201DE0124A1389294604F0E9F917E0D2
:107D60005278222A01D0012012E06A88003A18BF16
:107D700001225A75294604F0C1F9084B1A68D369E3
:107D80000BB1507D9847012002E0002000E0012067
:107D900038BD0020FCE70020FAE700BFD46E0020C9
:107DA0000460002038B5044600F11005284603F0B1
:107DB0006EF93F2801D8002038BDE178002003F09B
:107DC00073FD0028F8D0284603F061F93F2807D951
:107DD000402304F53672E178002003F08DFDEBE7D7
:107DE000E178002003F074FD0020E5E710B50446BB
:107DF00003F062FB60B900238BB10B484FF456735C
:107E000003FB0400037913F0010F0AD0012007E0FF
:107E100003F05AFB08B90123EEE70023ECE700204A
:107E200010BD0020FCE700BFD86E0020054B4FF4CA
:107E3000567202FB0033986808609A899B7B8A809F
:107E40008B717047D86E002008B54FF4567303FB52
:107E500000F310330248184403F0FCF808BD00BFDB
:107E6000D86E002038B50C4C4FF4567303FB00F06D
:107E70002518103020444FF6FE739A4208D892B26B
:107E800003F01BF904462846FFF78CFF204638BD57
:107E90004FF6FF72F4E700BFD86E002008B54FF42C
:107EA000567303FB00F310330248184403F00AF939
:107EB00008BD00BFD86E002070B5054603F0FCFA7F
:107EC00018B9002242B9002070BD03F0FDFA08B9CC
:107ED0000122F7E70022F5E74FF4567303FB05F3A1
:107EE0002033224C1C440434204603F0B3F808B974
:107EF0000020E9E71D4A4FF4567303FB05239978E8
:107F0000002003F0D1FC08B90020DDE74FF45673E0
:107F100003FB05F303F54673144E1E44402231461D
:107F2000204603F0CAF80446A8B1104B4FF456702F
:107F300000FB0530234632468178002003F0DCFC4C
:107F400038B90B4B1B6813F0010F00D000BE0020A6
:107F5000BAE72046B8E7054B4FF4567202FB0533EB
:107F60009978002003F0B4FC0020ADE7D86E002023
:107F7000F0ED00E070B505464FF4567404FB00F4D4
:107F800004F120030C4C1C4404344FF6FE739A4257
:107F90000BD892B2204603F0B0F80646204603F014
:107FA00059F83F2804D8304670BD4FF6FF72F1E70C
:107FB0002846FFF781FFF6E7D86E002008B54FF49A
:107FC000567303FB00F02030024B1844043003F0DA
:107FD0005EF808BDD86E00202DE9F04383B04FF461
:107FE0005672002126488DF0E1FF002616B103B03D
:107FF000BDE8F083224F4FF4567404FB06F43D199C
:10800000FF236B714FF4E133AB604FF0000885F84C
:108010000C8085F80D800823AB7304F1380104F15E
:108020001000CDF8008001234FF4807239443844A9
:1080300002F0D9FF04F59C7104F1200038444FF0A0
:108040000109CDF800904B464FF48072394404305A
:1080500002F0C9FF04F50E713944484676F0A4FCDD
:10806000C5F81C80286204F522713944484676F030
:108070009BFC2863C5F834804E44F6B2B6E700BFD7
:10808000D86E002070B5002606B170BD0D4C4FF4BF
:10809000567505FB06F5621900236351137105F14E
:1080A0001000204403F02EF820352C4404342046E0
:1080B00003F028F80121204603F044F80136F6B217
:1080C000E2E700BFD86E0020F0B583B04B79022BF9
:1080D00067D106468B79022B67D1002383B1002735
:1080E000F7B18B783B700D780D4409246B78242B05
:1080F0001ED194421CD82B781C44A4B21D44F5E731
:108100001F462B4C4FF4567000FB0340807810B193
:108110000133DBB2E2E74FF4567000FB0747DFE7BD
:10812000244B1B6813F0010F00D000BE002439E07F
:10813000052B09D06B78042B02D16B790A2B17D051
:108140003846FFF72FFE2DE02946304603F044FB6A
:1081500030B1AB787B702B781C44A4B21D44E9E7A6
:10816000144B1B6813F0010F00D000BE002419E06F
:1081700029780C44A4B2BB1C0193FB1C009302237E
:108180001A462944304603F051FB10B10E34A4B214
:10819000D6E7084B1B6813F0010F00D000BE002487
:1081A00000E00024204603B0F0BD0024FAE700BF41
:1081B000D86E0020F0ED00E0137803F06003202B70
:1081C0006CD170B514463B4A0025002D68D1167855
:1081D000A3889E4204D00135EDB202F55672F4E751
:1081E0006378203B032B5DD8DFE803F002192445B8
:1081F000012903D0032908D0012052E007230832C7
:10820000214603F095FF01204BE02B4B002B4BD078
:1082100002F108012846AFF30080012041E0012966
:1082200001D001203DE007230832214603F080FF02
:10823000012036E0012903D0032906D0012030E0D7
:10824000214603F05BFF01202BE0638813F001045B
:10825000C3F3400613710CBF0121002102F1240079
:1082600002F070FF154B0BB3324621462846FFF74C
:10827000DCF9012015E0012903D0032906D00120F3
:108280000FE0214603F03AFF01200AE00C4B7BB1DE
:1082900061882846AFF30080012002E0002070478B
:1082A000002070BD0020FCE70120FAE70120F8E77C
:1082B0000120F6E7D86E0020000000002B760200B7
:1082C000000000002DE9F04780460E469946002444
:1082D00054B1BCB9EB78B3421CD0AB78B3424AD0AE
:1082E00001242046BDE8F087384B4FF4567505FB56
:1082F0000435EB78B342ECD0AB78B342E9D001342B
:10830000E4B2E5E7324B1B6813F0010F00D000BE6A
:108310000024E6E705F1100A1FFA89F205F5367127
:10832000504602F0EAFE2B4BBBB16B79FF2B14D009
:10833000002700E001374F450FD26A79EB1993F817
:10834000D8329A42F6D1504602F098FE0028F1D178
:1083500069792046AFF30080ECE71F4B1BB1504614
:1083600002F08CFE18B12846FFF71CFDB5E7204649
:10837000AFF30080F7E7194B13B12046AFF300804D
:108380002046FFF799FD08B10124AAE705F1240072
:1083900002F060FEB0B9B9F1000F15D019F03F0F2F
:1083A00001D001249DE7A978404603F07DFA0446F8
:1083B00008B9012495E700231A46A978404603F03E
:1083C0009BFA8EE701248CE701248AE7D86E00200F
:1083D000F0ED00E0000000000000000000000000E0
:1083E00008B54FF48C72002101488DF0DFFD08BD07
:1083F0003072002008B50020FFF7F2FF08BD000032
:10840000F0B583B04B79032B6ED106460D460C793F
:10841000C4EBC404A4B21234A4B294420CD8002316
:10842000012B15D81F4632498C2202FB03125278C9
:1084300052B10133DBB2F3E72E4B1B6813F0010F8F
:1084400000D000BE002450E08C2202FB071700E0A1
:10845000002767B12B78E9184A78212A0FD0254BDD
:108460001B6813F0010F00D000BE00243DE0214B3B
:108470001B6813F0010F00D000BE002435E0C7F8E0
:108480008810E85C7B1C0193BB1C009303232A79B2
:108490000144304603F0CAF9D8B1AB79012B20D0A2
:1084A00001233B71AB783B70D7F88830B3F80730C5
:1084B000FB80B978C9B1402307F14802304603F088
:1084C0001BFA90B90B4B1B6813F0010F0DD000BEC7
:1084D0000BE0084B1B6813F0010F00D000BE002416
:1084E00003E0EB79FB70DBE70024204603B0F0BD2E
:1084F00030720020F0ED00E02DE9F04182B0154629
:10850000127802F01F03012B40F01F810646AF884E
:10851000FFB20024012C09D88C2303FB04F39348F9
:10852000C35C9F4203D00134E4B2F3E7FF24012C83
:1085300000F20F81274612F060022FD1012901D0ED
:10854000012003E16B881B0A6A78062A06D0062AF6
:1085500040F00381222B12D00020F7E0212BF6D12E
:10856000824A8C2303FB0427D7F88820002A00F0D6
:10857000F28013782946304603F0DAFDE6E0204623
:10858000FFF72EFA024679498C2303FB0717FB8875
:108590002946304603F0CCFD0120D7E0202A40F0E8
:1085A000DE806B78013B0A2B00F2DB80DFE803F012
:1085B0000693A3D9D9D9D9D9457BB300012901D0D4
:1085C0000120C3E06B881A0ADFF8A0E18C2000FBD1
:1085D00004F008300EEB0008EF88BC46402F28BF9F
:1085E0004FF0400C13F0FF010BD0012F1BD908F105
:1085F00001030EF800100CF1FF3C1FFA8CFC012760
:1086000001E043460027CDF800C02046FFF7F0F90F
:108610003B189BB253B9564B1B6813F0010F00D0A7
:1086200000BE002092E043460027ECE74246294680
:10863000304603F07DFD012088E0012903D00329A5
:1086400012D0012082E0EB88402B01D900207DE090
:108650008C2202FB04F2483244490A44294630463F
:1086600003F066FD012071E069880A0A3F4E8C2004
:1086700000FB04F048303318EF883D46402F28BFF8
:10868000402511F0FF0104D0012F02D9305C88424F
:1086900005D000952046FFF7C1F9012056E00133CF
:1086A000013DADB2F5E7012901D001204EE0698816
:1086B000090A2E4A8C2303FB042779712D4B23B121
:1086C0002046AFF30080002840D02946304603F012
:1086D00015FD01203AE0012901D0012036E0234BAD
:1086E0008C2202FB0432012305322946304603F076
:1086F0001FFD01202AE0012901D0012026E01B4BAB
:108700008C2202FB0432012304322946304603F056
:108710000FFD01201AE0012903D0032907D0012011
:1087200014E02946304603F0E9FC01200EE0698898
:10873000C9B20E4B8C2202FB043739710E4B93B138
:108740002046AFF30080012000E0002002B0BDE829
:10875000F0810020FAE70020F8E70020F6E700208B
:10876000F4E70020F2E70120F0E700BF30720020BC
:10877000F0ED00E00000000000000000F0B583B064
:108780000646234C002001E00130C0B2012809D880
:108790001F4C8C2505FB0044A5788D4202D06578DE
:1087A0008D42F1D1012807D862788A420DD0A27893
:1087B0008A4213D0012006E0164B1B6813F0010F0C
:1087C00000D000BE002003B0F0BD134AF2B19AB24F
:1087D00004F10801AFF300800120F4E704F148053B
:1087E0009BB200932B4600221146FFF717F9402356
:1087F0002A46A178304603F07FF80028E3D1054BE4
:108800001B6813F0010FDED000BEDCE70120DAE7C1
:1088100030720020F0ED00E00000000038B50446A2
:1088200000F11005284602F032FC3F2800D838BD80
:10883000A178002003F038F80028F8D0284602F08C
:1088400026FC3F2807D9402304F5EC72A1780020CC
:1088500003F052F8EBE7A178002003F039F8E6E7DF
:1088600070B5044600F12405284602F0F3FB08B970
:10887000002070BD6178002003F016F808B90020D0
:10888000F7E704F5067640223146284602F015FC4B
:10889000054680B1034632466178002003F02CF88B
:1088A00038B9084B1B6813F0010F00D000BE002040
:1088B000DFE72846DDE76178002003F009F80020B3
:1088C000D7E700BFF0ED00E02DE9F04182B04FF4B2
:1088D000167200211E488DF069FB002515B102B00B
:1088E000BDE8F0814FF4167404FB05F404F138017F
:1088F000174E04F110004FF00008CDF8008001235E
:1089000080223144304402F06EFB04F1B80104F1DE
:1089100020003044CDF8008001238022314404300F
:1089200002F061FB04F59C713144012076F03CF8C3
:108930003719C7F81C80386204F5C471314401202E
:1089400076F032F83863C7F834800135EDB2C5E708
:10895000F087012070B5002505B170BD4FF4167485
:1089600004FB05F40A4EA2190023A351536093603F
:10897000D36004F11000304402F0C4FB04F1200085
:108980003044043002F0BEFB0135EDB2E4E700BF35
:10899000F08701202DE9F0474B79012B40F08380CF
:1089A000064615468B79012B40F08180CB79002B50
:1089B0007FD10C78A3B20C446278242A06D1AB4252
:1089C00004D8227813449BB21444F5E7042A72D1E8
:1089D0006279012A71D1A279032A70D194F80780B3
:1089E000B8F1000F6DD142466AB14FF00009B9F1FC
:1089F000000F1ED0A27889F8002094F800A05344FC
:108A00009FB2A24435E091462F484FF4167101FB06
:108A10000201497829B94FF4167101FB02018978E6
:108A200011B10132D2B2DFE74FF4167101FB09092F
:108A3000DDE7264B1B6813F0010F00D000BE0027B6
:108A400032E0224B1B6813F0010F00D000BE00275C
:108A50002AE089F801309AF80020D3199FB2924495
:108A600008F101085FFA88F89AF80020D3199FB23C
:108A700092442379434512D9AF4210D89AF8013075
:108A8000052BF1D15146304602F0A6FE0028D8D081
:108A90009AF80230DA09DCD189F80230DBE748467F
:108AA000FFF7BCFE00E000273846BDE8F08700274E
:108AB000FAE70027F8E70027F6E70027F4E70027A2
:108AC000F2E70027F0E700BFF0870120F0ED00E0BB
:108AD00000207047F8B506461F4600244CB1B4B9D3
:108AE000AB788B421BD06B788B4229D00124204677
:108AF000F8BD4FF41675244B05FB0435AB788B425B
:108B0000EDD06B788B42EAD00134E4B2E6E71F4B3C
:108B10001B6813F0010F00D000BE0024E7E7BAB2D3
:108B200005F5EC7105F1100002F0E7FA184B13B1EE
:108B30002046AFF300802846FFF770FE0124D6E7F9
:108B40002846FFF78DFE08B10124D0E705F1240087
:108B500002F080FAA0B9AFB117F03F0F01D00124A5
:108B6000C5E76978304602F09FFE044608B9012443
:108B7000BDE700231A466978304602F0BDFEB6E72D
:108B80000124B4E70124B2E7F0870120F0ED00E012
:108B900000000000002380F830304363836380F8D6
:108BA0003C3080F83D3080F83E307047C38A5BBA75
:108BB0009BB2826812B9DBB900207047C17B2829BB
:108BC00006D02A291ED013B39A4222D30020704720
:108BD00010B4047BE4090DD02A2904D063B19A4271
:108BE0000ED3002009E0017BC909F7D0022004E080
:108BF00002207047022000E001205DF8044B70471E
:108C00000220FAE7017BC909DDD00220704701206C
:108C10007047022070470000044880F83C1080F83C
:108C20003D2080F83E300120704700BF487500208D
:108C3000F0B58DB0064615461F460C78252C00F27F
:108C40004681DFE814F02600440144010901440193
:108C500044014401440144014401440144014401EC
:108C600044014401440144014401B300440144016E
:108C700044014401440144014401E3003A00440139
:108C80004401440144014401440144018000440181
:108C90005800FEF735FF002840F01E81914B93F8F5
:108CA0003C3013B14FF0FF3413E13A220221304639
:108CB000FFF7B2FF4FF0FF340BE18B4B002B00F0BE
:108CC0000D810979C1F3400301F001020909FEF7A2
:108CD00059FF002840F00481824B93F83C3013B1D7
:108CE0004FF0FF34F5E03A2202213046FFF794FFBF
:108CF0004FF0FF34EDE00DF1060202A9FEF726FF6A
:108D0000BDF80620029B03B172B9764B93F83C3054
:108D100013B14FF0FF34DCE03A2202213046FFF776
:108D20007BFF4FF0FF34D4E0013B1BBA039312BA30
:108D30000492072F05D903AB03CB28606960082490
:108D4000C7E00024C5E000230393049305930823A0
:108D50008DF80F3002238DF814300DF1060202A9B0
:108D6000FEF7F4FE029B13B1BDF8062072B95D4B0D
:108D700093F83C3013B14FF0FF34AAE03A220221BD
:108D80003046FFF749FF4FF0FF34A2E01BBA0493CF
:108D900052BAADF816200B2F06D903AB07CB2860CB
:108DA0006960AA600C2494E0002492E000230393FD
:108DB000049380238DF80D3002238DF80E308DF84A
:108DC0000F301F238DF810304FF02033059306939A
:108DD0000793089309930A930B930BAB07AA05A972
:108DE000FEF740FE232F0FD903AE0BAF34460FCC56
:108DF00028606960AA60EB6026461035BC42F5D158
:108E000020682860242464E0002462E003238DF8B5
:108E10000C3000238DF80D309DF80E2063F3060210
:108E20008DF80E208DF80F30304B8BB1FEF7FEFE23
:108E3000034683F00103DBB29DF80E2063F3C712F3
:108E40008DF80E20032F05D9039B2B60042440E0EE
:108E50000123EEE700243CE00023039304930593F1
:108E60000693ADF81C30F0238DF80C300A238DF8F2
:108E700013301C4B93F83C104FF0000261F30302D7
:108E80008DF80E2093F83D208DF8182093F83E3091
:108E90008DF81930112F18D903AC0FCC28606960F8
:108EA000AA60EB6023882B82114B63B1BAB22946CA
:108EB0003046AFF30080044600231A461946304678
:108EC000FFF7AAFE05E01224F6E7002401E04FF0C8
:108ED000FF3420460DB0F0BD0024FAE70024F8E787
:108EE0000024F6E748750020857B02002D7C0200F7
:108EF0000000000038B505460C4681F82C208B6830
:108F00008A6B9B1A8B62022381F8303091F83C30D7
:108F100063B1A3684BB1A36A3BB1237BDB090BD0E0
:108F200094F82E10284602F031FD38BD202205218C
:108F3000607BFFF771FEECE794F82F10284602F0F3
:108F400025FDF2E770B586B006460D46CC8A64BAB8
:108F5000A4B21CB18A68B2FBF4F4A4B2D5F8111023
:108F600009BAAA6BB2FBF4F0AB689B1AB3F5007FA9
:108F700028BF4FF4007300931C4B04FB10220144E4
:108F8000687BFEF715FE002814DBF8B995F82E3043
:108F90000021039104918DF80C6007228DF80D20BB
:108FA0008DF8103005918DF8111003A802F01CFB0C
:108FB00006B070BD00233A220221687BFFF72CFE29
:108FC000012229463046FFF795FFF1E783B2074AB1
:108FD00095F82E10304602F08FFC0028E8D1044BA3
:108FE0001B6813F0010FE3D000BEE1E748730020D7
:108FF000F0ED00E038B505460C46154B1BB1487B3B
:10900000FEF714FE80B1A368A26B9B1AB3F5007F34
:1090100028BF4FF400739BB20E4A94F82F102846D5
:1090200002F06AFC60B138BD002327220721607B73
:10903000FFF7F2FD012221462846FFF75BFFF2E72A
:10904000054B1B6813F0010FEDD000BEEBE700BF2E
:109050002D7C020048730020F0ED00E0F0B587B0F1
:1090600007460C461646CD8A6DBAADB21DB18A6868
:10907000B2FBF5F5ADB2D4F8111009BAA26BB2FB90
:10908000F5F00096244B05FB10220144607BFEF7AF
:10909000A7FD011E18DBB1422FD2761A002922DC6F
:1090A00094F82F300021039104918DF80C70072261
:1090B0008DF80D208DF8103005968DF8111003A84D
:1090C00002F092FA07B0F0BDA26B3244A263002313
:1090D0003A220221607BFFF79FFD0122214638469C
:1090E000FFF708FFEEE7A36B13FA81F3A3630A48C7
:1090F000324601448CF040FFD2E7A26B1644A663CF
:10910000636B9E4203D3022384F83030DAE72146B2
:109110003846FFF76FFFD5E74873002008B54022B7
:10912000002102488CF042FF08BD00BF48750020B6
:1091300008B54022002102488CF038FF08BD00BF6E
:10914000487500204B79082B40D110B582B00446F9
:109150008B79062B3CD1CB79502B3CD1162A07D8E2
:109160001E4B1B6813F0010F00D000BE002030E042
:109170008A781B4B83F82D20087803F12E02019288
:109180002F33009302231A460144204602F04EFB7F
:1091900038B9124B1B6813F0010F00D000BE00203D
:1091A00017E00F4A002382F830301F2392F82F1067
:1091B000204602F0A1FB08B117200AE0074B1B680C
:1091C00013F0010F00D000BE172002E0002070470E
:1091D000002002B010BD0020FBE700BFF0ED00E072
:1091E00048750020012940F09C8030B583B00546C9
:1091F0001446137803F07F02022A13D003F06003B1
:10920000202B40F090806378FE2B6CD0FF2B40F039
:109210008D806388002B40F08B80E388002B59D031
:10922000002081E06278012AE8D16288002AE5D135
:10923000A188C9B23F4B93F83030042B24D03D4A6B
:1092400092F82E00884222D03A4A92F82F408C425F
:109250001FD1F3B92146284602F08AFB002830D0FE
:109260000023B3B1334A002382F830301F2392F831
:109270002F10284602F040FB58B92F4B1B6813F003
:10928000010F51D000BE4FE002F080FB01E0022B45
:1092900001D0012048E09368916B5B1A936203232D
:1092A00082F830300D2320320146284602F024FB9C
:1092B0000028EED1204B1B6813F0010F34D000BE04
:1092C00032E02146284602F0B1FB08B90123C8E785
:1092D0000023C6E71748FFF75DFC2146284602F049
:1092E0000DFF012020E063886BB9E388012B0AD1D0
:1092F0008DF80730114B1BB1FEF7A8FB8DF8070066
:109300009DF807300BB900200EE0013B8DF80730C7
:1093100001230DF107022146284602F009FF012032
:1093200002E001207047002003B030BD0020FBE7C1
:109330000020F9E748750020F0ED00E04D7A0200CA
:1093400070B50546A44C94F83040012C00F0C7805D
:10935000032C00F006813CB19F4B93F83030022B78
:1093600000F04A81012070BD9B4A92F82F0088428C
:1093700040F075811F2B03D11268984B9A420FD091
:10938000954C042384F8303094F82E10284602F0CF
:10939000FDFA94F82F10284602F0F8FA0020E2E7D0
:1093A0008D4B8F4A1A625A685A6200229A6283F879
:1093B0002C20012183F830109C685C639A63DE7B6B
:1093C000282E10D02A2E0ED0002C37D0824B1B7B9B
:1093D000DB0933D1B4F5007F21D901227E4928462B
:1093E000FFF788FDB8E77C48FFF7E0FB024638B995
:1093F00084B1282E09D078492846FFF7FBFDABE75A
:1094000075492846FFF776FDA6E773492846FFF71A
:1094100099FDA1E7704B022283F830209CE7A3B2AC
:10942000704A0146284602F067FA002894D16E4B34
:109430001B6813F0010F96D000BE94E766484FF406
:109440000073684A00F10F01407BFFF7F1FB031E38
:109450000ADB002B17DB13BB5F4B9B68CBB95E4B62
:10946000022283F8302077E75B4A92F83C20002AFA
:10947000EFD15948838E5B4A00F10F01407BFEF724
:1094800077FB0346E5E7012253492846FFF732FD03
:1094900062E7012250492846FFF72CFD5CE74E4A5F
:1094A00092682AB901224C492846FFF723FD53E769
:1094B000934228BF134648494B639BB2494A91F8EF
:1094C0002E10284602F018FA00287FF445AF464BCC
:1094D0001B6813F0010F3FF446AF00BE43E73E4A5E
:1094E000D27B282A12D02A2A1FD03B498A6B1344E8
:1094F0008B630B7BDB091DD0374B9A6B5B6B9A42FE
:1095000027D3354B022283F8302025E732498A6B76
:1095100013448B634A6B934203D3022281F83020B9
:109520001AE72D49FFF70EFD16E71A462A49FFF7FD
:1095300095FD11E708468B8E2A4A0F31407BFEF7D6
:1095400017FB0028D8DA012223492846FFF7D2FC6E
:10955000D2E7254B1B6813F0010F3FF4FDAE00BEB0
:10956000FAE61D4A92F82E208A427FF4F5AE0D2BC2
:109570007FF4F2AE184BDB7B282B0AD02A2B23D0AA
:109580001A4B63B1144B03F10F01587BAFF300800A
:1095900005E0174B1BB1104B587BAFF300800E4A10
:1095A000002382F830301F2392F82F10284602F053
:1095B000A3F900287FF4D0AE0B4B1B6813F0010F0A
:1095C0003FF4D1AE00BECEE60A4B002BE7D0024BF3
:1095D000587BFEF71DFBE2E74875002055534243D8
:1095E0005553425348730020F0ED00E000000000A6
:1095F00000000000117C02001A4B93F82E10284640
:1096000002F014FA00287FF4AEAE164A9368926B0B
:10961000934203D91349097BC90918D19B1A1149EF
:109620008B62032381F830300D2301F1200291F881
:109630002E10284602F060F900287FF494AE0A4B01
:109640001B6813F0010F3FF48EAE00BE8BE6054B96
:1096500093F82E10284602F099F9012083E60120A4
:1096600081E600BF48750020F0ED00E010B504462B
:109670008178002002F018F900B910BD201D01F01A
:1096800006FD3F2807D9402304F5A672A1780020E3
:1096900002F032F9F1E7A178002002F019F9ECE7C5
:1096A00070B5054601F008FF18B9002242B9002044
:1096B00070BD01F009FF08B90122F7E70022F5E7C4
:1096C0004FF4E67303FB05F31833224C1C44204689
:1096D00001F0C0FC08B90020EAE71E4A4FF4E67327
:1096E00003FB05235978002002F0DEF808B90020BA
:1096F000DEE74FF4E67606FB05F606F5C473154E75
:109700001E44043640223146204601F0D6FC044671
:10971000A8B1104B4FF4E67000FB053023463246EB
:109720004178002002F0E8F838B90B4B1B6813F0C1
:10973000010F00D000BE0020BAE72046B8E7054B75
:109740004FF4E67202FB05335978002002F0C0F8AE
:109750000020ADE788750020F0ED00E02DE9F04134
:1097600082B04FF4E67200211F488CF01FFC0026E7
:1097700016B102B0BDE8F0811B4D4FF4E67404FB56
:1097800006F404F1280129442F194FF00008CDF800
:109790000080012340220431381D01F024FC04F133
:1097A0006801294404F11800CDF80080012340220B
:1097B0000431284401F017FC04F1A80129440431C4
:1097C000012075F0F1F8C7F81080786104F1F80114
:1097D00029440431012075F0E7F87862C7F8288041
:1097E0000136F6B2C4E700BF8875002070B50024CA
:1097F00004B170BD094E4FF4E67505FB04F5701910
:1098000000237351043001F07DFC05F11800304451
:1098100001F078FC0134E4B2EAE700BF887500206B
:109820004B79FF2B5AD1F0B583B006460D460C7824
:109830000C44A318002252B10027002F50D0AA7860
:109840003A702A79CAB9601B80B203B0F0BD1746DE
:1098500024484FF4E67101FB0201497829B94FF41D
:10986000E67101FB0201897811B10132D2B2E2E75F
:109870004FF4E67101FB0707DFE76178052904D0A3
:109880009C4202D221780C44F7E77B1C0193BB1C5D
:10989000009302232146304601F0C8FF90B12B7996
:1098A000C3EBC3031C44BB78A3B97B78002BCAD09D
:1098B0000C48381A80100C4B03FB00F0C0B2FFF7C5
:1098C000EFFEC0E7094B1B6813F0010F00D000BE8C
:1098D0000020BAE73846FFF7C9FEE6E700207047E8
:1098E0000020B2E788750020BBA4F261F0ED00E033
:1098F00038B5194D002464BBAA788A4207D068782D
:10990000884204D00134E4B205F5E675F3E78A42F3
:1099100004D06A788A4211D001201BE09AB205F582
:10992000A671281D01F0E9FB0C4B13B12046AFF3E3
:1099300000802846FFF79AFE01200BE0084A1AB182
:1099400099B22046AFF300802046FFF7A9FE012020
:1099500000E0002038BD00BF887500200000000036
:10996000000000000268C08810447047C28842B1FD
:10997000037803EB830103EB41030349C858104408
:1099800070470020704700BF54770020884205D2FE
:109990004378934202D003781844F7E7704788422F
:1099A0000CD210B44478944205D09C4203D0047881
:1099B00020448842F6D35DF8044B704770472DE988
:1099C000F0410C4617461E46DDF8188005E0057884
:1099D0003A4621462844FFF7D9FFA04206D28178B3
:1099E000B142F4D1C3784345F1D104462046BDE8E5
:1099F000F08170B50C468678A0420AD283789E42E8
:109A000007D105780B23042221462844FFF7C7FF1E
:109A1000F2E770BD0346084601E01A78134483421A
:109A200005D25A78052A03D0042AF6D101E07047FE
:109A30001846704738B50D460478C3891C44044461
:109A400005E00378242221461844FFF79FFFA04237
:109A500008D28378023BDBB2052BF2D8C378AB4245
:109A6000EFD10446204638BD2DE9F0410446076990
:109A700041697F1A90F850608369BD199D4200D3F7
:109A80001D46B54209D2104B1B6813F0010F00D0E0
:109A900000BE00252846BDE8F081A5EB060806F1CA
:109AA0005000E3684246194420448CF057FA62693A
:109AB00042446261761BFE42ECD194F8513043F08F
:109AC000020384F85130E5E7F0ED00E02DE9F041C4
:109AD00082B080460D460F688E883E44BB78009267
:109AE000042231463846FFF76AFF864230D90446E1
:109AF000037D012B0CD80078E18901446618637A54
:109B0000184420442379C3B1012B09D0002020E060
:109B1000114B1B6813F0010F00D000BE002018E0AD
:109B200005223146FFF732FFB04201D3002010E09A
:109B30000146404601F050FE18B1E41BEC800120C4
:109B400007E0054B1B6813F0010F02D000BE00E0D8
:109B5000002002B0BDE8F081F0ED00E070B50646EF
:109B60000D460846FFF7FEFE03460278417A11448F
:109B70000844D9890A449C181B7923B90023AB7186
:109B8000EB71012070BD05222146FFF7FFFEA042C8
:109B900007D3064B1B6813F0010F00D000BE002056
:109BA000F0E78178304602F049FAE7E7F0ED00E0AF
:109BB00038B515465488240A012C0AD0022C61D0ED
:109BC000484B1B6813F0010F00F08A8000BE07208D
:109BD00038BD5278812A2DD0862A43D0012AEFD170
:109BE000012903D0022916D00020F1E7EA88012AD2
:109BF00001D0FF20ECE703EB830203EB42030833C1
:109C0000394A1A4401230232294602F091FA002807
:109C10005CD00020DCE7354A0AB90020D8E703EB26
:109C2000830203EB4201304A0A44917A1846AFF3AB
:109C30000080CDE7012901D00020C9E7EA88012A88
:109C400001D0FF20C4E703EB830203EB4203083398
:109C5000254A1A4401230232294602F069FAB8B3B0
:109C60000020B5E7012901D00020B1E7EB88012BE6
:109C700001D0FF20ACE71E4A294602F059FA48B34A
:109C80000020A5E75278812A05D0862A98D101299B
:109C900014D000209CE7012901D0002098E703EBB5
:109CA000830203EB420308330F4A1A4401231A4488
:109CB000294602F03DFA78B1002089E701230D4AD8
:109CC000294602F035FA48B1002081E7FF207FE7FE
:109CD000FF207DE7FF207BE7FF2079E7FF2077E784
:109CE000072075E7F0ED00E0547700200000000049
:109CF0002EBD0B002DBD0B0070B582B0054614467D
:109D000052780A2A09D00B2A27D0264B1B6813F059
:109D1000010F45D000BE072002E0012902D000203B
:109D200002B070BDE288012A15D103EB830003EB7A
:109D300040031D481844FFF715FE60B1C3788DF845
:109D4000073001230DF107022146284602F0F0F901
:109D500008B10020E4E7FF20E2E7012901D000205C
:109D6000DEE7E288B2B903EB830003EB40030E4E5B
:109D70001E4431462846FFF7F1FE68B1628831463D
:109D80002846FFF7A3FE48B12146284602F0B6F95F
:109D90000020C5E7FF20C3E7FF20C1E7FF20BFE7A2
:109DA0000720BDE7F0ED00E05477002038B51478C7
:109DB000C4F3411514F0600F03D0012D04D0072027
:109DC00038BDFFF799FFFBE79488240A0DD003EB19
:109DD000830003EB400307481844FFF7C3FD214607
:109DE000FFF728FE20B10020EAE7FFF7E1FEE7E7F2
:109DF0000720E5E754770020F8B50D46FFF7B6FDDC
:109E0000AB7890B31E460446027B93422DD823B90B
:109E1000012A00F2DB800126AE70002301222A72A3
:109E20006B72AB72EB72AA73EB732B746B746FF083
:109E30003F01A9766FF00301E9766FF0640129779D
:109E40006A770322AA770122EA7785F8202085F82D
:109E5000212085F82230082385F823302078B4F8B3
:109E60000D7007442744044411E05C4B1B6813F059
:109E7000010F00D000BE0020F8BDE3789E4213D051
:109E80002078242239462044FFF780FD0446A7426B
:109E900009D9A378042BF0D0062BEED00C2BECD0F4
:109EA000112BEDD1E9E73C46A74206D0A378042B5D
:109EB0000BD0062B0DD00020DEE7484B1B6813F0BB
:109EC000010F00D000BE0020D6E701232B73002332
:109ED0006B73EE7823799E4207D81EB9012B77D891
:109EE0000126EE702078204410E03C4B1B6813F0F4
:109EF000010F00D000BE0020BEE7C3789E4210D004
:109F00000378242239461844FFF740FD874207D9D9
:109F10008378052BF1D0072BEFD0112BF0D1ECE794
:109F2000384687422ED0D5F8123033B9A278042AA9
:109F300030D0062A39D0C5F81230696861B9427E3E
:109F4000012A47D82AB9D0F81E10D0F81A20914219
:109F500042D1D0F81A106960214AA2FB0102520BCB
:109F600042F20F70814229D91344013BB3FBF2F353
:109F70000233B3F5807F01D94FF48073C5F81630F2
:109F8000012079E7154B1B6813F0010F00D000BECC
:109F9000002071E7B0F80520B0F8073003FB02F2AB
:109FA000637D03FB02F3DB08C5E7B0F80520B0F8DA
:109FB000073003FB02F31B01DB08BCE7074B1B6800
:109FC00013F0010F00D000BE002055E7012053E739
:109FD000012051E701204FE701204DE7F0ED00E0BF
:109FE0005917B7D138B5044600214177816100F196
:109FF0001E05302228468BF0D9FF29462046FFF760
:10A00000FBFE38BD2DE9F04F83B081460D469246E8
:10A010000B7803EB830203EB4203494A52F80380B7
:10A020000024012C0ED805EB44031B8953B1434493
:10A030009978484602F002F805EB440300221A81A1
:10A040000134EEE70023EB602B616B6168884044CC
:10A05000AF8847448378CDF800A004223946FFF743
:10A06000AEFC0446874261D990F804B0BBF1020F00
:10A070000CD8A0EB0803EB80BAF1000F02D16B7F84
:10A08000012B0BD120782044002629E02D4B1B68A2
:10A0900013F0010F00D000BE002348E02846FFF770
:10A0A000A1FF03460028EDD141E0264B1B6813F0C9
:10A0B000010F00D000BE002339E0C37803F0030392
:10A0C000022B38D12146484601F086FB0346F8B101
:10A0D000A4EB080205EB46031A81013620782044E0
:10A0E0005E451CD23946FFF795FC04468742DCD911
:10A0F000AA69BAF1000FE0D0C37803F00303012B83
:10A10000E0D18388C3F30A039342DBD200230EE03D
:10A110000C4A126812F0010F09D000BE07E0BAF134
:10A12000000F0AD002236B77012300E000231846BA
:10A1300003B0BDE8F08F0023F9E70123F7E700BF84
:10A1400054770020F0ED00E030B583B005461446AA
:10A150001F484FF4A87202FB030063780A2B09D052
:10A160000B2B20D01B4B1B6813F0010F2ED000BE11
:10A1700007201BE0012901D0002017E0E388012B14
:10A180000FD1FFF7F3FB60B1C3788DF807300123DF
:10A190000DF107022146284601F0CAFF08B1002050
:10A1A00004E0FF2002E0012902D0002003B030BD0E
:10A1B000628801462846FFF725FF28B12146284638
:10A1C00001F09CFF0020F1E7FF20EFE70720EDE71B
:10A1D00060770020F0ED00E02DE9F8430D461446CD
:10A1E00092F80290B9F1000F34D1832906D0872963
:10A1F0000AD0822908D00020BDE8F883FFF7B6FB1B
:10A2000020B1037BA37001E00123A370002301228E
:10A2100022726372A372E37222736373A273E37395
:10A22000237463746FF03F01A1766FF00301E17650
:10A230006FF06401217762770322A2770120E07733
:10A2400084F8200084F8210084F82230082384F860
:10A250002330D1E7D778002F75D1FFF787FB06466B
:10A2600030B10078B6F80D7007443744064411E069
:10A27000864B1B6813F0010F00D000BE0020BBE727
:10A28000F378994513D03078242239463044FFF7CB
:10A290007DFB0646B74209D9B378042BF0D0062BD4
:10A2A000EED00C2BECD0112BEDD1E9E73E46832DFF
:10A2B00005D0872D05D0822D0ED000209CE7357962
:10A2C0000BE0B378042B03D0062B03D0002093E7D8
:10A2D000B57D02E0B57900E00125E57030783044C5
:10A2E00008E0C3789D420FD00378242239461844F1
:10A2F000FFF74CFB874208D98378052BF1D0072B59
:10A30000EFD0112BF0D1ECE70746B378042B03D044
:10A31000062B0FD000206FE7B7F80520B7F80730FD
:10A3200003FB02F2737D03FB02F3DB08C4F8123077
:10A33000012061E7B7F80520B7F8073003FB02F307
:10A340001B01DB08F2E7D2F80480B8F1000F40F0FF
:10A350009980FFF70BFB034630B10078B3F80D602E
:10A3600006441E44184410E0484B1B6813F0010FCC
:10A3700000D000BE00203FE7C378994512D0037893
:10A38000242231461844FFF701FB864209D983781D
:10A39000042BF1D0062BEFD00C2BEDD0112BEED1EE
:10A3A000EAE730460378184408E0C3789F420FD0AC
:10A3B0000378242231461844FFF7E8FA864208D988
:10A3C0008378052BF1D0072BEFD0112BF0D1ECE7E0
:10A3D0000646823D052D57D8DFE805F01F033756A6
:10A3E0005630737EB3B1053306EB8303D3F8028096
:10A3F000D6F81A30264AA2FB03235B0BC4F804806C
:10A40000B8F1000F2CD10023A375E3752376637692
:10A410000120F1E6D6F81E80EAE7737E5BB10533D2
:10A4200006EB8303D3F80230D6F81A80184AA2FB51
:10A4300003235B0BE2E7D6F81E30F5E7D6F815806C
:10A44000134BA3FB08235B0BD8E7737E33B9D6F815
:10A4500022800F4BA3FB08235B0BCFE74346CDE7DE
:10A46000D4F8122043B9931CB3F5807F01D94FF47F
:10A470008073C4F81630CBE71A44013AB2FBF3F309
:10A480000233F1E70120B7E60020B5E6F0ED00E089
:10A490005917B7D12DE9F0418CB0074615461E4635
:10A4A000B84B4FF4A87000FB063C5488240A022CD9
:10A4B00000F0F180062C0AD0012C32D0B24B1B6880
:10A4C00013F0010F00F0A58100BE0720A2E1537830
:10A4D000812B05D0862BF1D1012917D0002099E1DD
:10A4E000012901D0002095E14FF4A87202FB06F289
:10A4F0001832A44B1A44012304322946384601F08D
:10A5000017FE002800F06B81002083E101239F4AA1
:10A510002946384601F00CFE002800F06281002038
:10A5200078E1984A4FF4A87303FB06235B7F2BB1B5
:10A530004FF4A87303FB062300225A776C78012C92
:10A540000FD063B2002BB9D0872CB7D8812CB5D3EC
:10A55000813C062CB2D8DFE804F02C464646758BC9
:10A560004600012903D0022913D0002052E14FF404
:10A57000A87303FB06F31833824A1A4430230632C9
:10A580002946384601F0D4FD002800F02C81002037
:10A5900040E14FF4A87303FB06F31833794A1344E0
:10A5A000991D6046FFF728FC002800F01E8100205E
:10A5B00030E1012901D000202CE1EB88002B00F0D4
:10A5C00016814FF4A87303FB06F318336D4A1A443F
:10A5D000302306322946384601F0AAFD002800F053
:10A5E0000881002016E1012901D0002012E1EB884A
:10A5F0000BB9FF200EE1634B4FF4A87808FB063639
:10A6000006F11E04EE4606F14E08764620686168A3
:10A61000A268E3680FC61034B6464445F5D16A46D1
:10A6200069786046FFF7D8FD08B90820F2E03023CA
:10A630006A462946384601F07BFD08B10020E9E072
:10A64000FF20E7E0012901D00020E3E0EB88022BA6
:10A6500001D0FF20DEE03023ADF8003002236A464F
:10A660002946384601F064FD0028F2D00020D1E0F0
:10A67000012901D00020CDE0EB88012B01D0FF2083
:10A68000C8E0434A2946384601F052FD002800F050
:10A69000B2800020BEE05378852B7DD008D8012BF6
:10A6A0000ED0812B7FF40AAF012957D00020B1E0F2
:10A6B000862B7FF403AF012900F084800020A9E0FD
:10A6C000012903D0022913D00020A3E04FF4A8737E
:10A6D00003FB06F318332B4A1A443023063229466B
:10A6E000384601F025FD002800F08780002091E029
:10A6F0004FF4A87303FB06F31833224C23449C1D2C
:10A7000021466046FFF778FB002878D01D4A4FF4B9
:10A71000A87303FB06235A6B9A611E4B63B1194859
:10A720004FF4A87303FB06F3C11822464978C05CB6
:10A73000AFF30080002864D112494FF4A87303FBE3
:10A7400006F3CA18012050770020D06010615061D4
:10A750005033CA180224CC5450705BE0D388002BCD
:10A7600051D04FF4A87303FB06F31833054A1A447B
:10A77000302306322946384601F0DAFC002844D05E
:10A78000002047E060770020F0ED00E02DBD0B00D9
:10A790002EBD0B0000000000012901D0002039E08F
:10A7A000D388022B01D0FF2034E03023ADF80030F5
:10A7B00002236A462946384601F0BAFC0028F2D046
:10A7C000002027E0D388012B01D0FF2022E0134A8C
:10A7D0002946384601F0ACFCC8B100201AE0FF2041
:10A7E00018E0FF2016E0FF2014E0082012E0FF2010
:10A7F00010E0FF200EE0FF200CE0FF200AE0082020
:10A8000008E0002006E0FF2004E0FF2002E0FF2037
:10A8100000E007200CB0BDE8F08100BF2EBD0B00AA
:10A8200038B51478C4F3411514F0600F03D0012D2E
:10A8300004D0072038BDFFF787FCFBE79488240A83
:10A8400002D1FFF727FEF5E70720F3E710B5002355
:10A850000BB1002416E00D4C03EB830203EB420224
:10A86000A0180021A1504160C0F807100133EFE7A4
:10A8700050220021064B4FF4A87000FB04308BF0EF
:10A8800095FB0134002CF3D010BD00BF547700209D
:10A890006077002010B500230BB1002416E00D4CAA
:10A8A00003EB830203EB4202A0180021A150416098
:10A8B000C0F807100133EFE750220021064B4FF498
:10A8C000A87000FB04308BF071FB0134002CF3D036
:10A8D00010BD00BF54770020607700202DE9F04FB5
:10A8E00085B002904B790E2B40F0A3800C468B79FB
:10A8F000012B40F0A280CB79012B40F0A0804FF0DB
:10A900000008404668B180464FF0000AB8F1000FD9
:10A910001BD04C4B1B6813F0010F00D000BE002071
:10A9200088E000EB800300EB43034749CB5823B199
:10A9300000F101085FFA88F0E4E7804600EB80034D
:10A9400000EB430A404B9A44E0E7A518CAF80040E0
:10A95000AAF80420002251460298FFF7B7F808B978
:10A96000002067E05046FEF7FDFF90F814B029463E
:10A970002046FFF73EF807464646CDF80CA0AA460B
:10A9800025E032494FF4A87202FB031252882ABB19
:10A990002E4A4FF4A87101FB0325039A3244137227
:10A9A000FDB185F800806E70A7EB04091FFA89F9E4
:10A9B000A5F8029051463846FFF71BF80746031BDF
:10A9C0009BB2AB8000226A779EB10136F6B2B345E6
:10A9D00028D94346002BD4D00025E1E70133DBB270
:10A9E000F8E7184B1B6813F0010F00D000BE0020E1
:10A9F00020E0BBF1010FE8D104EB090004EB0309EF
:10AA000001230093837804224946FEF7D8FF81454D
:10AA1000DBD1002229460298FFF7F4FA0028D4D1AE
:10AA2000002007E0DDF80CA03C1BA0B2AAF804400F
:10AA300000E0002005B0BDE8F08F0020FAE700201C
:10AA4000F8E700BFF0ED00E05477002060770020C9
:10AA5000F8B5137803F01F03012B47D19388DBB2BD
:10AA600000242CB184B10024DCB19CB300203EE072
:10AA700004EB840504EB45051F4E755915B1AD78FF
:10AA80009D42EFD00134ECE72346FFF78FF904EB4A
:10AA9000840304EB4304184B1C44607240B3002051
:10AAA00025E0164E4FF4A87505FB04656F887FB14D
:10AAB0004FF4A87606FB04F6104DAD5D05EB850658
:10AAC00005EB46050C4E75593D44AD789D42CCD002
:10AAD0000134C9E72346FFF7A3FE084B4FF4A872E1
:10AAE00002FB0434207728B1002000E00020F8BDEC
:10AAF0000120FCE70120FAE754770020607700206E
:10AB000070B506460D4600238BB143BB62692369CD
:10AB10009A422CD30023E36023616361214B002B15
:10AB20003ED061782078AFF3008001201EE01E4AFD
:10AB30004FF4A87404FB0324208970B14FF4A8716A
:10AB400001FB03F1525C02EB820102EB4102174967
:10AB50008A5802449278AA42D7D00133D4E7144BE2
:10AB60001B6813F0010F00D000BE002070BD294605
:10AB7000304600F099FE0028F8D02046FEF774FF1A
:10AB800083B204F150022946304600F0B5FE002899
:10AB9000ECD1074B1B6813F0010FE7D000BEE5E7CF
:10ABA0000120E3E7000000006077002054770020D8
:10ABB000F0ED00E003460A4490B2814202D8B0EBC7
:10ABC000430F03DB5B009BB2C01A80B2704770B5C5
:10ABD00006460846B4889A420ED3D51AADB2F5B1EE
:10ABE000AC4204D294420DD8131B9BB273819C4299
:10ABF0000BD81B1B9BB2FAE7D51A610011FA85F539
:10AC0000ADB2ECE7A3189BB2F0E73168F288C2F36B
:10AC10000E0202FB03118BF0A1F9012070BD002090
:10AC2000FCE730B583B005469408631E9BB224B19F
:10AC300051F8044B2C601C46F7E712F0030201D1D7
:10AC400003B030BD0023019301A88BF087F9019B6D
:10AC50002B60F5E72DE9F04383B006460F469DF8DB
:10AC600028108588EC1A1FFA84FC5D1B1544B0F887
:10AC700006E0CEF30E0914FB09F4A4B215FB09F5A6
:10AC8000ADB2006809FB030821B1012916D003B059
:10AC9000BDE8F083944506D309FB02F241463846ED
:10ACA0008BF05CF9F3E72246414638468BF056F9C3
:10ACB0002A46316838198BF051F9E8E7944507D3F3
:10ACC00019FB02F292B241463846FFF7AAFFDEE7CF
:10ACD00024F003091FFA89F94A4641463846FFF72E
:10ACE000A0FFC84414F0030428D0C4F1040080B2CB
:10ACF000A84228BF2846C0B22D1AADB20023019346
:10AD000001AB04E018F8012B03F8012B0C46611E7F
:10AD1000C9B2002CF6D13168421ED2B228B111F866
:10AD2000010B03F8010B1046F6E7019B3B60002D79
:10AD3000ADD02A463846FFF774FFA8E73168F6E73A
:10AD4000F0B583B01E46BDF8203084889E4212D3F1
:10AD5000F51AADB2F5B1AC4205D2B44211D8331BED
:10AD60009BB243812546954200D315469C420BD8A1
:10AD70001B1B9BB2FAE7F51A670017FA85F5ADB20F
:10AD8000E8E7A3199BB2ECE79DF8242000922A463D
:10AD9000FFF760FF284603B0F0BDF0B583B004466E
:10ADA0000D4616461F46006918B14FF0FF3173F08B
:10ADB000F3FE2389628992B2019700929BB23246D8
:10ADC00029462046FFF7BCFF05466189024689B245
:10ADD000A088FFF7EFFE6081206920B100231A46AA
:10ADE000194673F047FD284603B0F0BD10B582B098
:10ADF0009408631E9BB224B10C6840F8044B1C46B7
:10AE0000F7E712F0030201D102B010BD0B68019305
:10AE100001A98BF0A3F8F7E72DE9F04383B00646CC
:10AE20000F469DF828108588EC1A1FFA84FC5D1BDC
:10AE30001544B0F806E0CEF30E0914FB09F4A4B2F1
:10AE400015FB09F5ADB2006809FB030821B1012922
:10AE500016D003B0BDE8F083944506D309FB02F297
:10AE6000394640468BF07AF8F3E7224639464046A9
:10AE70008BF074F82A46391930688BF06FF8E8E7E0
:10AE8000944507D319FB02F292B239464046FFF7C8
:10AE9000ADFFDEE724F003091FFA89F94A46394677
:10AEA0004046FFF7A3FFC84414F003021FD0C2F1CD
:10AEB0000404A4B2AC4228BF2C46E4B22D1BADB2B0
:10AEC0003B68019301AB04E013F8012B08F8012B58
:10AED0000A46511EC9B2002AF6D13068621ED2B2AB
:10AEE00034B113F8011B00F8011B1446F6E7306873
:10AEF000002DAED02A463946FFF778FFA9E72DE9A5
:10AF0000F04383B09146002A6BD0044688461F4622
:10AF1000C06818B14FF0FF3173F03EFE2689B6B21B
:10AF2000618989B2E379DB0918D1A3888E420DD3F8
:10AF3000751AADB2AB420FD95D1BADB24D4528BFFE
:10AF40004D46002D42D0A288334631E0751A590093
:10AF500011FA85F5ADB2EDE70025EFE7A5884D457F
:10AF600009D8FFB9A9EB0509E388C3F30E0303FB76
:10AF700009880E46E5E78E420ED3731A9BB24B4406
:10AF8000B3EB450F10DBA5EB090292B22846FFF7A1
:10AF900011FE06464D46D4E7731A6A0012FA83F38F
:10AFA0009BB2ECE70E46CCE74D46CAE79B1A9BB234
:10AFB0009A42FBD900972A4641462046FFF72CFFCC
:10AFC0002A463146A088FFF7F5FD2081E06820B1D0
:10AFD00000231A46194673F04DFC284603B0BDE81D
:10AFE000F0831546F9E7B2F5004F2FD8F8B50446BF
:10AFF0000F4615461E46C06818B14FF0FF3173F07A
:10B00000CBFD206918B14FF0FF3173F0C5FD27600B
:10B01000A580E28866F30E02E280C2F307229DF863
:10B02000183063F3C712E271002363812381E06863
:10B0300018B11A46194673F01DFC206940B100236F
:10B040001A46194673F016FC0120F8BD002070471F
:10B050000120FAE70246808813899BB2528992B296
:10B06000934205D39B1A9BB2984228BF184670475B
:10B070009B1A420012FA83F39BB2F5E7028992B25F
:10B0800043899BB29A4214BF0020012070478288F6
:10B0900003899BB2408980B2834206D31B1A9BB2BC
:10B0A0009A4208D9D31A98B270471B1A500010FA66
:10B0B00083F39BB2F4E70020704708B50023FFF745
:10B0C0006CFE08BD38B504460D46006918B14FF056
:10B0D000FF3173F061FD228963899BB292B22946E8
:10B0E0002046FFF774FD0546206920B100231A466B
:10B0F000194673F0BFFB284638BD08B50023FFF79B
:10B10000FEFE08BD10B50446C06818B14FF0FF310F
:10B1100073F042FD206918B14FF0FF3173F03CFD30
:10B12000002363812381E06818B11A46194673F041
:10B13000A1FB206920B100231A46194673F09AFB3F
:10B14000012010BD38B504460D46C06818B14FF057
:10B15000FF3173F021FD206918B14FF0FF3173F01A
:10B160001BFDE37965F3C713E371E06820B10023A9
:10B170001A46194673F07EFB206920B100231A4657
:10B18000194673F077FB012038BD000038B505463D
:10B1900000240BE09B1A03EB4302184B03EBC203A2
:10B1A0009BB15B68284698470134E4B2144B1A7887
:10B1B000511D2346A1420FDBA242EBD9114B1B6864
:10B1C00004EB440203EBC203EAE70F4B1B6813F0E6
:10B1D000010F12D000BE10E00C4C38220021204696
:10B1E0008AF0E4FE4FF0FF336360A360E360236105
:10B1F0006361A361E3612362A38438BD3CBD0B009E
:10B20000B4780020B0780020F0ED00E0087900204C
:10B2100008B5FFF7BBFF00F0CBFF08BD70B50546D2
:10B220000C461646C86800F0CDFFE368324601219F
:10B230002846984770BD00002DE9F04F83B0824644
:10B24000481EC0B2FCF7B2FB20B10346427801921F
:10B25000022A09D0544B1B6813F0010F00D000BE26
:10B26000002003B0BDE8F08FC179C1F340144F480E
:10B27000027864F30412C1F3801161F34512027085
:10B2800003F109085A8813440093009B984580F005
:10B29000888098F801300B2B0BD04FF0010B98F8F9
:10B2A0000130042B0BD1009BA3EB0807BFB2002495
:10B2B00048E098F803B098F800309844EFE73A4B2C
:10B2C0001B6813F0010F00D000BE0020C9E7A9EBF6
:10B2D000030303EB4303364D05EBC30540E0324B5C
:10B2E0001B6813F0010F00D000BE0020B9E7AB6867
:10B2F000304A934205D0304A934240D1DDF804B041
:10B300003DE0DDF804B0F6E7274B1B6813F0010FB2
:10B3100000D000BE0020A4E723463246414627481D
:10B3200001F0E2FFB044264B1B7805339945ACDDB4
:10B330001D4B1B6813F0010F00D000BE002090E7EA
:10B340000134E4B21E4B1B785A1DA146A242EADB2F
:10B35000A342BCD91B4B1B6804EB440503EBC5059A
:10B36000002DBCD0AB683A46414650469847082865
:10B37000E6D98742E4D30646BBF1010FB7D00022DD
:10B380009345C9D998F802301344DBB207491944F0
:10B390000979FF29B8D105490B441C710132D2B299
:10B3A000EEE701205DE700BFF0ED00E00879002046
:10B3B0003CBD0B00C9800200958902001C79002069
:10B3C000B4780020B078002038B505460C464B888C
:10B3D0001A0AD8B2531E0E2B57D8DFE803F00826FE
:10B3E0003F56564A26565656565656561100FCF7A4
:10B3F000D9FA024612232146284600F099FE45E07C
:10B40000284B002B43D0FCF77FFC024628B1438831
:10B410002146284600F08CFE38E0234B1B6813F0D1
:10B42000010F00D000BE002030E0022A0CD01F4BDC
:10B430007BB3AFF3008050B91B4B1B6813F0010FB7
:10B4400000D000BE002021E0FCF7B0FAF3E743880B
:10B4500002462146284600F06BFE17E0A188FCF763
:10B46000ABFA0246B8B103782146284600F060FEE8
:10B470000CE00F4B8BB1AFF30080024678B103783C
:10B480002146284600F054FE00E0002038BD002090
:10B49000FCE70020FAE70020F8E70020F6E70020AC
:10B4A000F4E700BF097D0200F0ED00E000000000BD
:10B4B0000000000070470000024B5878003818BFA9
:10B4C0000120704708790020024B1878C0F38000F3
:10B4D000704700BF08790020024B1878FF3818BF6A
:10B4E0000120704714610020F0B583B00546FFF7D6
:10B4F000F3FF064610B1304603B0F0BD38220021FC
:10B500002E488AF053FD2E49012073F04DFA2D4B41
:10B510001860C8B12C4C0023009304F10C0362683E
:10B520006188208873F071F90746A16873F0ECFB1D
:10B53000264B1F607FB1264B23B12648AFF3008016
:10B54000254B1860002418E0244B1B6813F0010FF2
:10B55000D1D000BECFE7214B1B6813F0010FCAD03A
:10B5600000BEC8E79B1A03EB43021D4B03EBC2036B
:10B5700093B11B6898470134E4B2164B1A78511DF9
:10B580002346A1420FDBA242ECD9134B1B6804EB0C
:10B59000440203EBC203EBE7104B1B6813F0010FEF
:10B5A000A9D000BEA7E70F4B1D70284601F058F840
:10B5B000284601F057F801269DE700BF08790020D2
:10B5C000B878002040790020B8600020447900203D
:10B5D00000000000B4780020B0780020F0ED00E01A
:10B5E0003CBD0B001461002030B585B005460C460B
:10B5F0004378023B042B13D8DFE803F0033A242FEF
:10B600009300554B1A786FF300021A701A786FF393
:10B6100041021A70002159701A7861F382021A707F
:10B620004E4B1868002C40F0828000234FF0FF3210
:10B63000294673F01FF9224669782878FFF73AFF08
:10B6400005B030BD444B1B7813F0010FF8D0424ACF
:10B65000137843F004031370E2E73F4B1B7813F0B9
:10B66000010FEDD03C4A13786FF382031370D7E7D4
:10B67000394B1B7813F0040F1ED0374A13786FF341
:10B6800082031370002301930293039303788DF8D0
:10B69000043005238DF80530304B186871B900234C
:10B6A0004FF0FF3201A973F0E5F822469DF805102E
:10B6B0009DF80400FFF7FEFE00241BE0002300932A
:10B6C0006A4601A973F07FF9009B002BEDD0244B53
:10B6D0004FF080525A6040BFBFF34F8FBFF36F8F60
:10B6E000E3E79B1A03EB43021E4B03EBC2030FE09D
:10B6F0000134E4B21C4B1A78511D2346A1429FDB52
:10B70000A242EED9194B1B6804EB440203EBC203BF
:10B71000002BEDD05B69002BEAD069682878984748
:10B72000E6E70D4AD3780133DBB2D37078E7002324
:10B73000019301AA294673F046F9019B002B3FF4BF
:10B740007AAF074B4FF080525A6040BFBFF34F8F24
:10B75000BFF36F8F6FE700BF0879002044790020A6
:10B7600000ED00E03CBD0B00B4780020B078002074
:10B7700010B584B00023019308238DF805300290A2
:10B780000391134B1868144672B900234FF0FF322F
:10B7900001A973F06FF822469DF805109DF804008A
:10B7A000FFF788FE04B010BD002300936A4601A98C
:10B7B00073F009F9009B002BEDD0064B4FF080523F
:10B7C0005A6040BFBFF34F8FBFF36F8FE3E700BFF7
:10B7D0004479002000ED00E038B5114B1D788B78DE
:10B7E00003F07F03082B07D90E4B1B6813F0010FE2
:10B7F00000D000BE002038BD0C460B4B9978204687
:10B8000001F022FD30B9074B1B6813F0010FF2D095
:10B8100000BEF0E72146284600F048FFEBE700BFF6
:10B8200014610020F0ED00E0087900202DE9F047D8
:10B8300080460C4616461F46DDF82090DDF824A011
:10B84000002515E0174B1B6813F0010F00D000BE58
:10B8500000231846BDE8F087124A126812F0010F63
:10B86000F7D000BEF5E789F8003023781C44013595
:10B87000AE4214DD6378052BE4D1E17801F00301D9
:10B88000B942DFD121464046FFF7A6FF0346002814
:10B89000E2D0A378DA09E6D08AF80030E5E70123A0
:10B8A000D7E700BFF0ED00E008B501F07F004000F1
:10B8B00000EBD1102030044B1844044B19680630BB
:10B8C00001F072FC08BD00BF08790020407900201B
:10B8D00008B501F07F00400000EBD1102030044B90
:10B8E0001844044B1968063001F08BFC08BD00BFFA
:10B8F0000879002040790020F8B51A48007801F056
:10B900007F05194C04EB450404EBD1142034A479D1
:10B9100014F0010F07D0154B1B6813F0010F00D076
:10B9200000BE0020F8BDCE090F4C04EB45043444A2
:10B9300094F8267047F0010784F82670203400F050
:10B94000FBFF0028EED1A3796FF30003A371A37965
:10B950006FF38203A371054B1B6813F0010FE1D055
:10B9600000BEDFE71461002008790020F0ED00E060
:10B9700001F07F02044B03EB420303EBD11191F87A
:10B98000260000F0010070470879002038B5114BFF
:10B99000187801F07F05104B03EB450303EBD1133F
:10B9A00020339B7913F0020F00D038BDCC0901F091
:10B9B00057F8094B03EB4503234493F8262042F044
:10B9C000020283F8262093F8262042F0010283F831
:10B9D0002620EAE7146100200879002038B5114BD1
:10B9E000187801F07F05104B03EB450303EBD113EF
:10B9F00020339B7913F0020F00D138BDCC0901F040
:10BA00005BF8094B03EB4503234493F826206FF3BF
:10BA1000410283F8262093F826206FF3000283F872
:10BA20002620EAE7146100200879002001F07F0257
:10BA3000044B03EB420303EBD11191F82600C0F352
:10BA400040007047087900202DE9F04182B005469A
:10BA50000C46002000F0B6FB237803F06003602B57
:10BA600014D0402B1CD0227802F01F02012A00F0D3
:10BA7000F280022A00F03881FAB1AB4B1B6813F058
:10BA8000010F00F0C68100BE002006E0A64B1B6837
:10BA900013F0010F00D000BE002002B0BDE8F0811D
:10BAA000A24B002B00F0A181184600F08BFB224630
:10BAB00001212846FCF72CF9EFE7202B0BD07BBBAC
:10BAC0006378092B00F2BE80DFE803F0A999BC89F6
:10BAD000BC3284BC414EA388DBB20F2B00F28781BD
:10BAE000934A13441B79934A127893420DD2924A97
:10BAF000116803EB430301EBC301002900F07B81D4
:10BB000022462846FFF78AFBC7E7511D9942C0F23B
:10BB100070819B1A03EB4303884901EBC301ECE7F7
:10BB2000814B1B6813F0010F00D000BE0020B4E76A
:10BB3000204600F04DFB6188C9B2284600F0A4FD04
:10BB40007B4A137843F0020313700120A5E7784B7A
:10BB50005B788DF8063001230DF106022146284658
:10BB600000F0E6FA012098E76688F6B2704B5B7841
:10BB7000DBB2B34207D06E4B5B7863B9BEB9704B92
:10BB80000BB1AFF300806A4B5E702146284600F08F
:10BB9000B5FA012081E7284600F022FE644F97F8AD
:10BBA00002802846FFF7F2FA87F80280E6E731467E
:10BBB0002846FFF741FB28B1624B002BE3D0AFF3DF
:10BBC0000080E0E7584B1B6813F0010F3FF465AFAE
:10BBD00000BE62E721462846FFF7F6FB5DE7638873
:10BBE000012B01D0002058E7514A137843F0080395
:10BBF00013702146284600F081FA01204DE7638842
:10BC0000012B01D0002048E7494B1A786FF3C3029B
:10BC10001A702146284600F071FA01203DE7444B96
:10BC20001A78930803F00203C2F340121343ADF8ED
:10BC3000063002230DF106022146284600F078FA6C
:10BC400001202AE7384B1B6813F0010F00F0D58064
:10BC500000BE002021E7A388DBB20F2B00F2CF80CB
:10BC6000334A13441B79334A1278934225D2324A1D
:10BC7000116803EB430301EBC301002900F0C3800B
:10BC800022462846FFF7CAFA00287FF406AF237839
:10BC900013F0600F7FF401AF63780A3B012B3FF68E
:10BCA000FCAE002000F08EFA63780A2B10D02146FB
:10BCB000284600F023FA0120EFE6511D9942C0F218
:10BCC000A0809B1A03EB43031C4901EBC301D4E79B
:10BCD00000238DF8063001230DF106022146284687
:10BCE00000F026FA0120D8E6A288D1B202F07F0641
:10BCF000C2F3C012082E27D80D4800EB46000244BC
:10BD0000127D0C480078824226D20B48066802EB6E
:10BD1000420206EBC2065BB3002E76D022463146C5
:10BD20002846FFF77BFAB8E6F0ED00E0117D02004F
:10BD300008790020B4780020B07800203CBD0B00CA
:10BD40000000000000000000334B1B6813F0010FDF
:10BD500000D000BE0020A0E6461D964206DB121A67
:10BD600002EB42022D4E06EBC206D4E70026D2E7D4
:10BD70006378012B18D0032B16D03BB1264B1B68E0
:10BD800013F0010F00D000BE002086E62846FFF722
:10BD90004DFEADF8060002230DF1060221462846AD
:10BDA00000F0C6F9012078E6628822B9012B18D08C
:10BDB0002846FFF7EBFD56B3224631462846FFF7EB
:10BDC0002DFA002000F0FEF9154B93F8273013F000
:10BDD00001007FF462AE2146284600F08FF9012071
:10BDE0005BE62846FFF7FAFDE5E7002055E6002070
:10BDF00053E6002051E600204FE600204DE60020EB
:10BE00004BE6002049E6002047E6002045E60120F9
:10BE100043E6002041E600BFF0ED00E03CBD0B0032
:10BE20000879002030B585B00446FFF755FB40BBCC
:10BE300005B030BD224600E0224601A9284672F036
:10BE400023FE0028F4D09DF80530013B072B00F2BB
:10BE5000DA80DFE813F008002900D800B300C4003E
:10BE600033006A00D1009DF80400FFF7D1F99DF876
:10BE70000820694B9A70694B186872F031FF0028EE
:10BE8000D6D0664B1D68B4F1FF3FD3D0002CD3D081
:10BE90004FF47A720023A002A10D89F089FC0246BA
:10BEA0000028CAD10122C8E79DF80400FFF7B0F9C5
:10BEB0005B4B002BDFD0AFF30080DCE7564AD37832
:10BEC000013BDBB2D370D378002BD4D11346127868
:10BED00042F001021A7093F826206FF3000283F8F3
:10BEE000262093F826206FF3820283F8262093F809
:10BEF00027206FF3000283F8272093F827206FF3A1
:10BF0000820283F8272002A99DF80400FFF79CFD18
:10BF10000028B0D100219DF8040000F0A1FD80218F
:10BF20009DF8040000F09CFDA5E79DF8081001F0C5
:10BF30007F00CD09384B03EB400303EBD11393F89B
:10BF400026206FF3000283F8262093F826206FF353
:10BF5000820283F82620B8B12F4B03EB40032B4419
:10BF60001B7D304A1278934216D22F4A126803EB97
:10BF7000430302EBC303CBB11D69039B9DF809206A
:10BF80009DF80400A84776E7039B9DF809209DF8DB
:10BF9000040000F02BF96EE7501D984206DB9B1A57
:10BFA00003EB4303214A02EBC303E4E7204B1B6886
:10BFB00013F0010F3FF43CAF00BE39E7164B1B787E
:10BFC00013F0010F3FF457AF1A4B002B3FF453AF60
:10BFD000114B1878C0F3C000AFF300804BE70E4B55
:10BFE0001B7813F0010F3FF446AF134B002B3FF4C7
:10BFF00042AFAFF300803EE7029B002B3FF43BAF24
:10C000000398984737E70A4B1B6813F0010F3FF47A
:10C0100032AF00BE2FE700BF08790020447900202E
:10C0200000000000B4780020B07800203CBD0B0078
:10C03000F0ED00E0000000000000000038B5134BF8
:10C040001878134BDBB101F07F05CC0900F00AFC36
:10C05000104B03EB4503234493F826206FF3410272
:10C0600083F8262093F826206FF3000283F8262019
:10C0700093F826206FF3820283F8262038BD064B02
:10C080001B6813F0010FF9D000BEF7E71461002020
:10C0900065C8020008790020F0ED00E0F8B5074619
:10C0A000134B9E89DD89741BA4B2402C28BF402409
:10C0B00093F90030002B08DB0021AE4213D00D4A6B
:10C0C00023463846FFF718FCF8BDAE4209D0084BAE
:10C0D0009968402C09D82246064889F03FFF802104
:10C0E000EBE78021E9E70022EAE70020ECE700BF68
:10C0F000087A00201C7A00207047000038B50546F9
:10C100000B460A4A14460868496803C40021916036
:10C11000D181918193F900308B4200DB8021002393
:10C120001A462846FFF7E8FB38BD00BF087A002012
:10C13000F8B507460C461C4D2E460868496803C6EC
:10C14000AA600021E981E1888B4228BF0B46AB81C0
:10C15000E188A1B103B152B13846FFF79FFFC8B9DA
:10C16000124B1B6813F0010F14D000BE12E00F4BEE
:10C170001B6813F0010F00D000BE00200AE094F904
:10C180000030002B07DB802100231A463846FFF7DA
:10C19000B3FB10B1F8BD0021F6E7044B1B6813F0A8
:10C1A000010FF7D000BEF5E7087A0020F0ED00E0BF
:10C1B000034B00221A605A609A60DA601A61704775
:10C1C000087A0020014B1861704700BF087A0020F0
:10C1D0000146054B1A460068496803C200229A606E
:10C1E000DA819A81704700BF087A002038B5054689
:10C1F0001C46364B1B78DB09B3EBD11F14D03CB186
:10C20000334B1B6813F0010F00D000BE002038BD77
:10C210002E4C2146FFF770FF23691BB122460321F4
:10C22000284698470120F2E7284B93F90030002B6D
:10C2300007DB264B9868002845D02246254989F01F
:10C240008DFE224AD38913FA84F39BB2D38191687D
:10C2500021449160D288934201D03F2C27D81B4BB8
:10C260001B6923B1194A022128469847A8B1174BE8
:10C2700093F90030002B0EDB802100231A4628465C
:10C28000FFF73AFB0028C2D1114B1B6813F0010FD6
:10C29000BDD000BEBBE70021EFE70021284600F03B
:10C2A000DFFB8021284600F0DBFB0120AFE72846BA
:10C2B000FFF7F4FE0028AAD1054B1B6813F0010F0D
:10C2C000A5D000BEA3E70020A1E700BF087A0020A8
:10C2D000F0ED00E01C7A0020084B1A6804331B685C
:10C2E000082A01D000207047032B03D8DFE803F0B1
:10C2F000040404040020704701207047300100103E
:10C30000084B1A6804331B68082A01D000207047C4
:10C31000032B03D8DFE803F0040404040020704773
:10C3200001207047300100100A4B1A6804331B6863
:10C33000082A01D000207047022B07D0032B07D01A
:10C34000012B01D000207047012070470120704769
:10C35000012070473001001042DF704743DF704713
:10C3600044DF704712DF704700B583B043F2040327
:10C370001A68154B9A420ED04FF08042D2F80C3416
:10C3800003F00103D2F80C2412F4803F17D10020EF
:10C3900003B05DF804FB00238DF8043001A8FFF71B
:10C3A000E1FF9DF80430002BE6D00023019301A8A3
:10C3B000FFF7D6FF0198003818BF0120E8E70BB956
:10C3C0000020E5E70120E3E7DBE5B15100B583B0EC
:10C3D000FFF7CAFF78B943F204031A680E4B9A427A
:10C3E0000CD00E4B00221A601B680193019B4FF08A
:10C3F000804301221A6003B05DF804FB00238DF82E
:10C40000043001A8FFF7AEFF9DF80430002BE8D000
:10C41000FFF7A2FFEFE700BFDBE5B15100010040ED
:10C4200043F204031A680E4B9A4203D00D4B0122CB
:10C430001A60704700B583B000238DF807300DF106
:10C440000700FFF78FFF9DF807302BB9054B01223E
:10C450001A6003B05DF804FBFFF780FFF9E700BF47
:10C46000DBE5B1510400004001230360BFF36F8F8F
:10C47000BFF34F8F074B984203D0043B984200D044
:10C480007047BFF35B8F044B002283F82021BFF37A
:10C490005B8FF5E7507002405C7A002008B50C4ACB
:10C4A0004FF00101BFF35B8FD2E84F3FC2E84C1F52
:10C4B000BCF1000FF8D1BFF35B8FDBB22BB10122CF
:10C4C00001460448FFF754F908BDFFF7CDFFFBE72D
:10C4D0007C7B00209DC4020010B5104A02EB401284
:10C4E000938AD18A89B25B1A9BB2118B8B4228BF87
:10C4F0000B4614690A4A00EB800102EB8101C1F886
:10C50000004600EB800102EB8102C2F80436054BC5
:10C5100003EB8000FFF7C2FF10BD00BF5C7A002074
:10C52000007002400470024070B5354A4FF00101BE
:10C53000BFF35B8FD2E84F3FC2E8441F002CF9D114
:10C54000BFF35B8FDBB2C3B9082834D12D4BD3F8CE
:10C55000C02412F4803F1CD12B4B03EB4013DB7A39
:10C5600003B34001284B1958264BC3F8A017C3F852
:10C57000A4272648FFF778FF41E0254B5A68C2F30D
:10C580000802003A18BF012201462248FFF7F0F8DE
:10C5900035E0BFF35B8F1C4B002283F82021BFF3F3
:10C5A0005B8F2CE0BFF35B8F174B002283F82021B9
:10C5B000BFF35B8F23E0134B00F5947253F82220F6
:10C5C00092B2114D460105EB4014A188E488A4B253
:10C5D000091B89B28A4228BF0A46AC5900EB800188
:10C5E00003EB8101C1F8004700EB800103EB8103FD
:10C5F000C3F80427084B03EB8000FFF735FF70BD3D
:10C600007C7B0020007002405C7A00204870024071
:10C6100000ED00E01DC602002870024008B5C0B25F
:10C62000FFF782FF08BD0000BFF35B8F0A4B93F852
:10C630002031BFF35B8F33B9084B1B6813F0010F38
:10C6400009D000BE7047BFF35B8F034B002283F815
:10C650002021BFF35B8F70475C7A0020F0ED00E093
:10C6600070470000014B80225A60704700E100E0F3
:10C67000044B8022C3F88420BFF34F8FBFF36F8F2A
:10C68000704700BF00E100E0074BD3F80014D3F877
:10C6900000240A43C3F800240022C3F858214FF4B1
:10C6A0008002C3F8042370470070024070B48B7896
:10C6B00003F07F02DE098C88C4F30A04500000EB0B
:10C6C000D315434800EB05100481C97801F003013C
:10C6D000012930D006BB02F10C04012000FA04F459
:10C6E0003C49C1F80443D1F8144590402043C1F8B7
:10C6F000140502F59472002041F82200354AC2F870
:10C70000183543F48073C2F80C35BFF36F8FBFF355
:10C710004F8F012070BC7047941C012101FA04F472
:10C720002C48C0F80443D0F8104501FA02F2224325
:10C73000C0F81025E2E7082A07D0274B1B6813F042
:10C74000010F00D000BE0020E4E7FEB9204BB3F893
:10C7500018311BB11F4B8022C3F81C251D4B002232
:10C76000C3F85021D3F8003313F4001F02D1194B42
:10C77000C3F85421174B4FF44012C3F80423D3F8E5
:10C78000142542F48072C3F81425BEE7114B002231
:10C79000C3F82C210E4BB3F808311BB10D4B80228E
:10C7A000C3F81C250B4BD3F8003313F4001F03D13F
:10C7B000084B0022C3F85421064B084AC3F804234F
:10C7C000D3F8102542F48072C3F810259DE700BF0E
:10C7D0005C7A002000700240F0ED00E000082000CC
:10C7E00038B50546FFF744FF01241AE004F10C03B5
:10C7F000012202FA03F3A11C8A401343154AC2F82E
:10C80000083302EB84030021596004F10A0342F863
:10C8100023102022104800EB441089F0C7FB01349C
:10C82000E4B2072CE2D90B4C0C4BC4F808330021BE
:10C83000C4F81C156162A1642022094889F0B6FB86
:10C840000123C4F81435C4F810352846FFF70AFF51
:10C8500038BD00BF007002405C7A00200008300044
:10C860005C7B002010B401F07F03C909082B2CD099
:10C87000E1B903F10C04012202FA04F42C48C0F8D7
:10C880000843D0F814459A4024EA0202C0F814255F
:10C8900001EB4301274B03EB01110023CB72BFF3E4
:10C8A0006F8FBFF34F8F5DF8044B70479C1C0122C4
:10C8B00002FA04F41E48C0F80843D0F810459A4024
:10C8C00024EA0202C0F81025E2E71A4A02EB01123C
:10C8D0000020A2F80801F1B9154A4FF48010C2F8FF
:10C8E0000803D2F8140520F48070C2F81405002063
:10C8F000C2F850010E4A0020C2F81C050D4AB2F8D9
:10C900001801B2F80821D042C2D1094A4FF40010F0
:10C91000C2F80803BCE7064A4FF40060C2F80803F7
:10C92000D2F8100520F48070C2F81005E2E700BFCD
:10C93000007002405C7A0020F0B585B00C4601F032
:10C940007F00CE09410001EBD4153F4901EB0511F1
:10C95000C97AA9B93C4D06EB40010F0105EB011165
:10C96000EA518B800022CA80A0B9002B41D1374BFD
:10C97000D3F88034C3F3C013B3423CD001230AE0A0
:10C98000334B1B6813F0010F00D000BE0025284672
:10C9900005B0F0BD00231D467BBB002E4DD106EB3C
:10C9A0004003294A02EB03130122DA7200283FD028
:10C9B000BFF36F8FBFF34F8F06EB4003224A02EBAA
:10C9C00003139B7A03F0FF05002B3AD006EB4003DC
:10C9D00002EB0313DB7A03F0FF04002BD7D006EB46
:10C9E000400302EB031300229A72FFF79DFD2546D8
:10C9F000CDE70023CFE70023CDE71648FFF74EFD34
:10CA0000154B5968C1F308010023019302938DF877
:10CA1000043007228DF805208DF8084003938DF827
:10CA20000930C91A18BF012101A8FEF7DDFDAEE7E4
:10CA30000A48FFF733FD0125A9E7FFF74DFD012562
:10CA4000A5E70125A3E700BF5C7A00200070024043
:10CA5000F0ED00E05070024000ED00E04C7002404C
:10CA600008B511F07F0007D1114B01225A65BFF3C1
:10CA70006F8FBFF34F8F08BDCB090828F7D041F463
:10CA800080710B4AC2F81815002BF0D103EB40025D
:10CA9000084901EB0212927A002AE8D003EB400326
:10CAA00001EB031300229A72FFF73EFDDFE700BFA0
:10CAB000007002405C7A002011F07F0319D0CA098F
:10CAC000082B16D010B40B48C0F80C1541F4807434
:10CAD000C0F80C45C0F8181522B903F5947300216D
:10CAE00040F82310BFF36F8FBFF34F8F5DF8044BF7
:10CAF000704770470070024010B5194B0122C3F80F
:10CB00001425C3F81025002309E0154A02EB830021
:10CB10000021416003F10A0042F820100133072B85
:10CB2000F3DD0F4B002159629964C3F85811D3F813
:10CB30000004D3F800240243C3F80024D3F80023F0
:10CB4000C3F80823074AC3F80423074C4FF4927232
:10CB5000204689F02BFA40232383238110BD00BF98
:10CB6000007002400514C0015C7A0020F0B587B067
:10CB7000BD4BD3F8000300231D4601E00133DBB2B7
:10CB8000182B15D820FA03F212F0010FF6D0B74A8D
:10CB900052F82340002CF1D0012404FA03F10D4394
:10CBA000002142F82310BFF36F8FBFF34F8FE5E7EB
:10CBB00015F0010F24D115F4006F09D0AA4BD3F85A
:10CBC000A8369BB2AA4AA2F81631012382F81C317A
:10CBD00015F4001F3FD0A44BD3F8143513F4807F15
:10CBE0001FD015F4800F06D09F4BD3F8003413F0FC
:10CBF000010F40F099800820FFF796FC012211E018
:10CC0000FFF77AFF00230393049305938DF80C300C
:10CC100001218DF80D108DF8103003A8FEF7E4FC0B
:10CC2000C9E70022904BD3F8103513F4807F00F051
:10CC300096808F4B93F81C31002B77D10023039300
:10CC4000049305938DF80C3003238DF80D300121EA
:10CC500003A8FEF7C9FC15F4800F23D0824BD3F84C
:10CC6000004440F201722240C3F8002414F4807F93
:10CC70007ED114F4806F12D07B4B0122C3F80825BB
:10CC80009A65D3F8003313F4001F03D1764B0022CA
:10CC9000C3F85421744B4FF40012C3F8042314F466
:10CCA000007F75D115F4000F38D06F4BD3F8802476
:10CCB000D2B28DF80420D3F88414C9B28DF80510CF
:10CCC000D3F888048DF80600D3F88C048DF807009B
:10CCD000D3F890048DF80800D3F894048DF8090077
:10CCE000D3F898048DF80A00D3F89C348DF80B30F3
:10CCF00012F07F0F01D1052910D00023ADF80E30BE
:10CD00008DF80C3006238DF80D300299019806AB92
:10CD100003E90300012103A8FEF766FC554B2B40F5
:10CD2000002B43D1002465E001227BE7504A002319
:10CD300082F81C31B2F8162192B2039304938DF855
:10CD40000C3007218DF80D1088218DF810100592F8
:10CD50008DF81130012103A8FEF746FC6EE7002A8A
:10CD60007FF46CAF404B4FF40012C3F8082365E723
:10CD70000121C3F82C1500230393049305938DF828
:10CD80000C3004238DF80D3003A8FEF72DFC70E75E
:10CD900000230393049305938DF80C3005238DF83D
:10CDA0000D30012103A8FEF71FFC7BE7FFF73CFCD9
:10CDB000B8E72F4A02EB4612D37A002B4BD02C4B0C
:10CDC00003EB4613DA889A800022DA72DB889BB282
:10CDD000039204928DF80C2007218DF80D108DF828
:10CDE000104005938DF81120012103A8FEF7FCFBEC
:10CDF0000134E4B2082C43D804F10C03DBB225FA69
:10CE000003F313F0010FF3D0264604EB84029300E2
:10CE100003F1804303F51C33D3F8082792B2144979
:10CE2000630101EB4417C8581044C850FB8812FA3C
:10CE300083F39BB2FB80082CBBD03B899342B8D1D3
:10CE4000FA8892B2BB889A42B3D2002CD0D10A4859
:10CE5000FFF724FBCCE7094B1B6813F0010F00D050
:10CE600000BE07B0F0BD00BF00700240007102407C
:10CE70005C7A0020FCFB1F004C700240F0ED00E0EB
:10CE8000494B2B40002BECD0484BD3F86C64C3F8D3
:10CE90006C64BFF36F8FBFF34F8F15F4806506D0BE
:10CEA000D3F8803413F0800F0BD1002700E0002767
:10CEB0004DB13E4BD3F8803413F0800F06D00025DF
:10CEC00002E00127F4E70025002420E00125FBE72C
:10CED00001EB8102930003F1804303F51C33D3F887
:10CEE0000806C0B2324B03EB41131A6902441A61BF
:10CEF000DA8A10FA82F292B2DA82DA8A92B29B8AE3
:10CF00009A4211D22046FFF7E7FA0134E4B2072C27
:10CF100023D8214626FA04F313F0010FD8D1002CB0
:10CF2000F3D1002FF1D0D3E744F08000204B03EB86
:10CF30004111CA8A92B20023039304938DF80C30F6
:10CF400007218DF80D108DF8100005928DF8113025
:10CF5000012103A8FEF748FBD7E7002411E0204693
:10CF6000134B03EB4413DA7A22B1D98889B29B8838
:10CF7000994216D30E4B03EB401301229A720134EF
:10CF8000E4B2072C3FF66DAF04F11003DBB226FAD2
:10CF900003F313F0010FE2D1002CF0D1002DEED0FD
:10CFA000DDE7FFF7C1FAEAE7000400010070024084
:10CFB0005C7A002010B584B0012800F0B18002280E
:10CFC00043D008B104B010BD704BD3F80035002B2E
:10CFD000F8D16E4B4FF48002C3F808234FF400627F
:10CFE000C3F80024BFF36F8FBFF34F8FFFF79CF997
:10CFF00050B1674B1B6803BB654B49F275321A6031
:10D000006449032008601A60FFF77AF950B1604B59
:10D010001B68B3B95E4B49F275321A605E49C02095
:10D0200008601A60594B0122C3F80025BFF36F8FC7
:10D03000BFF34F8FFFF7CAF9C4E7564B03221A60BC
:10D04000E2E7554BC0221A60ECE7504BD3F80435A9
:10D05000002B57D14D4BD3F8003413F4006FF9D0A7
:10D060004A4B4FF40062C3F80024BFF36F8FBFF345
:10D070004F8FFFF745F958B1454B1B68002B47D13F
:10D08000434B49F275321A604349002008601A6028
:10D09000FFF74AF958B13E4B1B68002B3CD13C4B83
:10D0A00049F275321A603B49002008601A60FFF7A8
:10D0B00013F950B1394B40F2E3721A600433402245
:10D0C0001A60BFF36F8FBFF34F8F304A8023C2F8CF
:10D0D0001C350121C2F80413314AC2F88431FEF72D
:10D0E000FBF910B12E4B80225A60FFF73DF9002862
:10D0F000FBD0264B0122C3F80425BFF36F8FBFF38B
:10D100004F8F5FE7FFF730F900287FF45BAFA1E7AF
:10D11000214B00221A60BBE71E4B00221A60C6E7B3
:10D120001A4BD3F80035002B3FF44CAF174B0024BB
:10D13000C3F80445BFF36F8FBFF34F8F184A8021A8
:10D14000C2F88410BFF34F8FBFF36F8FD3F8002363
:10D15000C3F80823C3F80045BFF36F8FBFF34F8FA9
:10D16000FFF75EF90F4B5968C1F30801019402946F
:10D1700003948DF8044002238DF80530091B18BF75
:10D18000012101A8FEF730FA1CE700BF0070024041
:10D1900000EC064014ED064014EC06400078024016
:10D1A00000E100E000ED00E070B5037813F0010449
:10D1B00024D105460E46037813F0040F1FD14FF01B
:10D1C000FF31304671F0E8FC2B7813F0010F05D1E8
:10D1D0002B7813F0040F0FD0002300E000231C462F
:10D1E0001BB12B7843F004032B7000231A46194619
:10D1F000304671F03FFB02E00123F0E700242046B7
:10D2000070BD70B504460D464FF0FF31284671F0F1
:10D21000C3FC237813F0040F0ED100231E461BB16C
:10D2200023786FF38203237000231A461946284699
:10D2300071F020FB304670BD237813F0010F01D050
:10D240000023EBE70123E9E78388C3F30A02C378ED
:10D2500003F00303022B18D0032B2FD0012B01D096
:10D2600000207047022905D040F2FF33934204D3D7
:10D27000012070474FF48063F8E71A4B1B6813F0E6
:10D28000010F00D000BE00207047022903D0402AC1
:10D290000CD801207047B2F5007F21D0114B1B68DC
:10D2A00013F0010F00D000BE002070470D4B1B682B
:10D2B00013F0010F00D000BE00207047022904D0F7
:10D2C0004023934204D3012070474FF48063F8E772
:10D2D000044B1B6813F0010F00D000BE0020704704
:10D2E00001207047F0ED00E00A44914212D230B4C0
:10D2F00003E00C78214491420AD24C78052CF8D1F5
:10D300008C7804F07F0500EB4505E4092B55F0E728
:10D3100030BC7047704710B5044600F0AEF90023EA
:10D3200084F8E830204610BD012800D0704708B5C9
:10D330004FF6FF73994200D008BD0248FFF7EBFF9C
:10D34000FAE700BF807B002038B590F8E8500DB1B7
:10D35000284638BD0446012380F8E83076F0E0FA2C
:10D360000028F5D1204600F08CF90546F0E790F84A
:10D37000E83003B9704710B50446002380F8E83060
:10D3800076F002FB204600F099F910BD08B54FF683
:10D39000FF710120FFF7C8FF08BD000002680B689D
:10D3A0009A4201D00020704770B584B004460D4603
:10D3B0004FF4537071F0EBF80646A8B10C4800F03A
:10D3C00088F9234653F8042B002102910196043575
:10D3D0000095084976F03EF90446304671F0F1F8C0
:10D3E00024B9012004B070BD0020FBE70020F9E75C
:10D3F000807B002019240A00F0B585B005460C4654
:10D40000164603934FF4537071F0C1F878B1074694
:10D41000009003AB3246291D201D76F099F9044691
:10D42000384671F0CEF824B9039805B0F0BD00205D
:10D43000FBE70020F9E700220260704710B50446C0
:10D44000084676F0F7F92060003818BF012010BDBB
:10D4500000220260704710B50446084676F0EAF9EB
:10D460002060003818BF012010BD00230360704702
:10D4700000B583B0019201AB0A460421084476F05E
:10D4800063F818B9019803B05DF804FB0020FAE7CF
:10D49000F0B583B004460D4616464FF4637071F044
:10D4A00076F888B1074654F8040B019700940123DD
:10D4B0003246294675F084FF0446384671F081F8FB
:10D4C00024B9012003B0F0BD0020FBE70020F9E7FC
:10D4D00000220260012141608260C160032101617C
:10D4E0008261C2610275704710B50446007D00B1CB
:10D4F00010BD0023237576F013FA034608B9012204
:10D500002275B3FA83F04009F2E708B500230375EA
:10D5100076F03AFA08BD0F2908D911F00F0F03D0A1
:10D52000090901310901C9B2084670471020704746
:10D530002DE9F04F9BB002AF79609B4697F88C8045
:10D54000D7F89060D7F898A0037D002B7DD00546D2
:10D55000914676F0E5F900287AD118F007047AD1DF
:10D56000B8F10F0F7AD9B8F1200F7AD8AB695246CB
:10D57000D7F8941007F1140075F0F4FDD7F888304F
:10D58000FB60C7F81080082307F10C02E96907F176
:10D59000140075F027FE002866D1AB6853451FD1F3
:10D5A00049462846FFF7B7FF054610F00F0202D0A4
:10D5B000C2F11002D2B2AB46EB1D23F00703ADEB74
:10D5C000030D0DF1080AD0468DF808200DF109026F
:10D5D000AB1E002B0EDB002102F8011B013BF8E71C
:10D5E000594607F1140075F021FE0028D8D06FF0DD
:10D5F000060B25E04A467968504688F0AFFC2A467B
:10D600000021304688F0D2FCAC420BD233191022F4
:10D6100008EB040107F1140075F020FE38BB10344C
:10D62000E4B2F1E7264407F10803019300960023D2
:10D630000AEB0402194607F1140075F04DFEC8B953
:10D6400058466437BD46BDE8F08F4FF0FF3BF7E723
:10D650006FF0010BF4E76FF0020BF1E76FF0020BD4
:10D66000EEE76FF0020BEBE76FF0030BE8E76FF00C
:10D67000040BE5E76FF0050BE2E7002280F8E420F9
:10D68000704770B590F8E4500DB1284670BD04465F
:10D69000012380F8E4304FF4BF5070F078FF064665
:10D6A0000028F2D00146204675F0A2F80446304624
:10D6B00070F087FF002CE8D10125E6E708B590F867
:10D6C000E43003B908BD002380F8E43075F0F4F8C5
:10D6D000F8E7704708B513460A46194674F09CFEF1
:10D6E00008B9012008BD0020FCE708B5012116207B
:10D6F00074F0F8F80021162074F078F901210D205B
:10D7000074F0F0F80D2074F0C2F901210C2074F0CF
:10D71000E9F80C2074F0BBF901210B2074F0E2F859
:10D720000B2074F0B4F908BD0EB400B582B0014608
:10D7300003AB53F8042B0193064B186820B1019BEF
:10D7400000F52A6002F01AFD02B05DF804EB03B0A8
:10D75000704700BFBC7F00201AB308281ED8DFE83E
:10D7600000F017141D0E11080B1A0500D9B1174847
:10D770007047D1B116487047C9B116487047C1B15A
:10D7800015487047B9B115487047B1B11448704792
:10D79000A9B114487047A1B11348704799B1134813
:10D7A0007047124870471248704712487047124835
:10D7B0007047124870471248704712487047124825
:10D7C0007047124870471248704700BF44BF0B00B3
:10D7D0003CBF0B0034BF0B002CBF0B0024BF0B0061
:10D7E0001CBF0B0014BF0B000CBF0B00A0BE0B0036
:10D7F000A8BE0B00B4BE0B00C0BE0B00CCBE0B001D
:10D80000D8BE0B00E4BE0B00F0BE0B00FCBE0B004C
:10D8100004BF0B000C281CD8DFE800F0071D171B05
:10D820001B0F1113090D15190B000C4870470C48FC
:10D8300070470C4870470C4870470C4870470C48BC
:10D8400070470C4870470C4870470C4870470C48AC
:10D8500070470C4870470C48704700BFB0BF0B00C2
:10D8600060BF0B0070BF0B007CBF0B0094BF0B00B0
:10D870000C670D008CBF0B0090BF0B009CBF0B0012
:10D88000A4BF0B004CBF0B0054BF0B00F0B5D5B0CC
:10D890000E461746002302464E4935A869F05EF849
:10D8A00035A869F03CFB08B955B0F0BD35A869F062
:10D8B0003CFB0028F8D0002235A91CA869F038FBF1
:10D8C0001CA869F02CFB002834D01CA869F02BFBA5
:10D8D0000378002B2ED01CA869F027FB04460028F3
:10D8E0002CD10546002C3DD1002C3FD1002D5AD023
:10D8F000002E3FD1002235A903A869F019FB049B33
:10D900001D93059B1E93069B1F93079B20939DF8D9
:10D9100020308DF88430099B22930A9B23930BAC13
:10D92000402324A8002BCBDB14F8015B00F8015B3B
:10D93000013BF7E735A869F075FAB5E71CA869F06F
:10D94000F2FA01464EA870F039FB234951A870F055
:10D9500035FB51A94EA870F0EBFC08B92546C1E78C
:10D960000025BFE751A870F0E1FABDE74EA870F0BE
:10D97000DDFABBE7194B1C6804F52A641CA869F0A2
:10D98000D2FA0346164A1749204602F0EFFD1CA8BA
:10D9900069F0C9FA711E3A46C9B2FFF777FF1CA8B1
:10D9A00069F040FAA6E70D4B1C6804F52A641CA830
:10D9B00069F0B9FA05461CA869F0F0F900902B4609
:10D9C000094A0849204602F0D1FD1CA869F02AFA4C
:10D9D00090E700BF184C0120D8D60B00BC7F002078
:10D9E000B8BF0B00C8BF0B00D0BF0B0008B5014685
:10D9F000014869F049F808BD184C012000B583B012
:10DA0000134B196801A803F07EFD4FF0FFF8114891
:10DA10006BF040FD90B1104B1868104A104900F5AA
:10DA20002A6002F0A3FD00220A210E48FFF72EFF14
:10DA300001A803F070FD03B05DF804FB064B186805
:10DA4000094A0A4900F52A6002F090FDE3E700BFA9
:10DA5000B87F0020184C0120BC7F002004C00B00C0
:10DA6000C8BF0B0040030D00E4BF0B00FCBF0B0060
:10DA70002DE9F04F83B017460123009343680468F3
:10DA80001C1BE410C4EBC41204EBC202C2EB8232D2
:10DA900004EB021404EB8404354A121B002A4CD018
:10DAA00005460E460194002C4AD001AA1068044491
:10DAB0002A689B1ADB10C3EBC31203EBC202C2EB52
:10DAC000823203EB021303EB83039C423AD3284BCD
:10DAD0009C4239D8D5F800B0D5F804A0A6EB0B08C5
:10DAE000B4B3234B9C4231D8E82000FB04F04EF045
:10DAF00063FF8146E822394609EB080088F02EFAD8
:10DB0000B8F1000F27DC08F1E808C844AAEB060AC0
:10DB1000BAF1000F25DC08EB0A06BBF1000F02D0BA
:10DB200058464EF06DFFC5F800906E60E82000FB8F
:10DB30000494AC6003B0BDE8F08F0E4880F02DFF78
:10DB40006A46B3E70A4CC5E7094CC3E780F01FFFFC
:10DB50004FF00009CEE742465946484688F00CFA95
:10DB6000D1E752463146404688F006FAD3E700BF77
:10DB7000CB3D8D0018C00B0070477047934200F0FA
:10DB800028812DE9F04F85B00546884616461F4688
:10DB9000A3EB020A4FEAEA04C4EBC41304EBC30389
:10DBA000C3EB833304EB031404EB84048368D0F8E1
:10DBB0000490A3EB0903DB10C3EBC31203EBC20217
:10DBC000C2EB823203EB021303EB8303A34279D34C
:10DBD000A9EB010B4FEAEB03C3EBC31203EBC20249
:10DBE000C2EB823203EB021303EB830300939C42EC
:10DBF0003AD306EB0B0A5046FFF7BEFF01903846BA
:10DC0000FFF7BAFF0199421A814202D0484688F0D4
:10DC1000B3F9009BE41A6B68E82202FB04346C60E1
:10DC20004046FFF7AAFF07464846FFF7A6FFC21B7C
:10DC3000874203D03946204688F09EF96B685B44E2
:10DC40006B603046FFF798FF04465046FFF794FF9D
:10DC500005464046FFF790FF2A1BAC4200F0A88023
:10DC6000214688F089F9A3E0A9EB0A0B5846FFF793
:10DC700084FF04464846FFF780FF021B844203D01E
:10DC80002146484688F078F96B6853446B60ABEBEB
:10DC90000802C34504D04146A9EB020088F06CF9A4
:10DCA0003046FFF769FF04463846FFF765FF054633
:10DCB0004046FFF761FF2A1BAC4279D0214688F02D
:10DCC0005BF975E0029442680368D31ADB10C3EB7A
:10DCD000C31103EBC101C1EB813103EB011303EB72
:10DCE00083033C49C91AA14265D30393A34265D378
:10DCF00003A90C681C442B68D31ADB10C3EBC312B6
:10DD000003EBC202C2EB823203EB021303EB830389
:10DD10009C4255D32F4B9C4254D8002C56D02D4BAF
:10DD20009C4251D8E82000FB04F04EF045FE8146AD
:10DD30002868FFF722FF82464046FFF71EFFA0EB50
:10DD40000A0B824504D05A465146484688F014F9D9
:10DD5000CB443046FFF710FF82463846FFF70CFFF2
:10DD6000A0EB0A06824504D032465146584688F058
:10DD700003F95E44D5F804A04046FFF7FEFE0746CF
:10DD80005046FFF7FAFEA0EB0708874204D0424650
:10DD90003946304688F0F0F84644286808B14EF01D
:10DDA0002FFEC5F800906E60E82000FB0494AC6084
:10DDB00005B0BDE8F08F084880F0EFFD02A998E7B4
:10DDC000044CAAE7034CA8E780F0E1FD4FF00009FE
:10DDD000AEE77047CB3D8D0034C00B00F0B5FBB013
:10DDE0000646174600230360436083600A46604985
:10DDF00055A868F0B3FD55A869F091F810B9304600
:10DE00007BB0F0BD55A869F090F80028F7D000224B
:10DE100055A93CA869F08CF83CA869F080F8002866
:10DE200000F0A1803CA869F080F80446002828D1C1
:10DE30000546002C39D1002C3BD1002D59D0002FA4
:10DE40003BD1002255A902A869F072F8039B3D93CB
:10DE5000049B3E93059B3F93069B40939DF81C308B
:10DE60008DF80431089B4293099B43930AAC4023ED
:10DE700044A9002BD0DB14F8015B01F8015B013BE6
:10DE8000F7E73CA869F04FF801466EA870F096F8E5
:10DE9000384971A870F092F871A96EA870F048FA2C
:10DEA00008B92546C5E70025C3E771A870F03EF81C
:10DEB000C1E76EA870F03AF8BFE73CA869F033F804
:10DEC00001467A1ED2B202A8FFF788FF4FF0000386
:10DED0008DF80030039B029A71683046FFF74EFEC2
:10DEE0003CA868F09FFF02980028AAD04EF088FD59
:10DEF000A7E7E822002102A888F058F83CA868F0BB
:10DF00004DFF3B903CA869F00EF8014602A889F04D
:10DF1000D5FA02A974A870F051F8164977A870F0E4
:10DF20004DF877A974A870F003FA044677A86FF04B
:10DF3000FDFF74A86FF0FAFF1CB13CA868F072FFF7
:10DF40007FE77068B368984207D0E82202A988F09A
:10DF500005F87368E8337360EFE702AA01463046BC
:10DF6000FFF786FDE9E755A868F05CFF47E700BFCB
:10DF7000184C0120D8D60B002DE9F041DEB08DED14
:10DF8000030ACDED040A8DED051ACDED001A8DEDD5
:10DF9000012ACDED022A012800F02481022800F098
:10DFA000398220B19FED8A0A5EB0BDE8F0810DADE7
:10DFB0000DF10C0E9EE8070085E8070010AC6B46DB
:10DFC00093E8070084E80700D5ED016A94ED026A42
:10DFD00066EE865A95ED027AD4ED017A27EE275A3D
:10DFE00075EEC55A13ABC3ED005AD4ED005A27EEB7
:10DFF000257A95ED005A26EE056A37EE467A83EDCE
:10E00000017A67EE857A66EEA56A77EEE67AC3ED69
:10E01000027A2BAE93E8070086E8070016AF87E880
:10E0200007000AAE86E8070085E8070084E80700D5
:10E0300093ED007AD4ED007A27EE277AD3ED016ACA
:10E04000D4ED017A66EEA76AD3ED027A94ED026A06
:10E0500067EE867A37EE267A77EE877A5D4F17EE8F
:10E06000902AA7EB620206EE902A9FED5B4A67EECC
:10E07000847A66EEA77A66EEA77ADFED585A75EED7
:10E08000E77A66EEA77A94ED007A27EE877A83ED39
:10E09000007AD4ED016A67EEA66AC3ED016A94EDD9
:10E0A000027A67EE877AC3ED027A0DF5807C93E8F9
:10E0B00007008CE807000DF5867888E807000DF169
:10E0C0001C0C8CE8070085E807009EE8070084E840
:10E0D0000700D5ED017A94ED025A67EE854A95ED79
:10E0E000026AD4ED016A26EE267A74EEC74AC3EDC1
:10E0F000004A94ED007A26EE076AD5ED004A25EE37
:10E10000245A36EE456A83ED016A66EEA46A67EE2C
:10E11000877A76EEE76AC3ED026A0DF1A00893E80C
:10E12000070088E807000DF1640E8EE8070086E816
:10E13000070085E8070084E8070093ED006A94ED86
:10E14000007A26EE076A93ED017AD4ED017A27EE84
:10E15000277AD3ED026AD4ED027A66EEA76A36EE2C
:10E16000076A36EE867A17EE102AA7EB620207EEF0
:10E17000902A27EE047A27EE877A27EE877A35EE03
:10E18000C77A67EE877A94ED007A27EE877A83ED77
:10E19000007A94ED017A27EE877A83ED017A94ED87
:10E1A000027A67EE877AC3ED027A3AAD93E8070008
:10E1B00085E807003DAC84E80700D3ED000A9CED3C
:10E1C000000A81F0FBFCDFED067A20EE270AEBE681
:10E1D0000000000012141F5F12D3363FFF51D83FDA
:10E1E000E02E65420DAD0DF10C0E9EE8070085E8AE
:10E1F000070010AB6A4607CA83E80700D5ED016A3D
:10E2000093ED026A66EE865A95ED027AD3ED017AB5
:10E2100027EE275A75EEC55A13ACC4ED005AD3ED5C
:10E22000005A27EE257A95ED005A26EE056A37EE5C
:10E23000467A84ED017A67EE857A66EEA56A77EE16
:10E24000E67AC4ED027A31AE94E8070086E807006A
:10E250001CAF87E807000AAE86E8070085E80700DC
:10E2600083E8070094ED007AD3ED007A27EE277A51
:10E27000D4ED016AD3ED017A66EEA76AD4ED027A95
:10E2800093ED026A67EE867A37EE267A77EE877A22
:10E29000E24F17EE902AA7EB620206EE902A9FED5E
:10E2A000E04A67EE847A66EEA77A66EEA77ADFED3B
:10E2B000DD5A75EEE77A66EEA77A93ED007A27EEDF
:10E2C000877A84ED007AD3ED016A67EEA66AC4ED21
:10E2D000016A93ED027A67EE877AC4ED027A0DF552
:10E2E000987C94E807008CE807000DF59E7888E894
:10E2F00007000DF11C0C8CE8070085E807009EE87C
:10E30000070083E80700D5ED017A93ED025A67EE26
:10E31000854A95ED026AD3ED016A26EE267A74EEFF
:10E32000C74AC4ED004A93ED007A26EE076AD5EDA0
:10E33000004A25EE245A36EE456A84ED016A66EEFF
:10E34000A46A67EE877A76EEE76AC4ED026A0DF199
:10E35000B80894E8070088E807000DF17C0E8EE805
:10E36000070086E8070085E8070083E8070094EDCA
:10E37000006A93ED007A26EE076A94ED017AD3EDF8
:10E38000017A27EE277AD4ED026AD3ED027A66EE9F
:10E39000A76A36EE076A36EE867A17EE102AA7EBE2
:10E3A000620207EE902A27EE047A27EE877A27EE9C
:10E3B000877A35EEC77A67EE877A93ED007A27EE93
:10E3C000877A84ED007A93ED017A27EE877A84EDDF
:10E3D000017A93ED027A67EE877AC4ED027A46AE4F
:10E3E00094E8070086E8070049AD85E8070083E860
:10E3F00007009CE8070084E80700D4ED000AF1EE6E
:10E40000600A93ED000A81F0D9FBDFED877A20EEF8
:10E41000270AC9E513AB03AA07CA83E80700D3EDAF
:10E42000005A93ED016A93ED025A10AC6A4607CA8E
:10E4300084E80700D4ED026A26EE667AD4ED017A0C
:10E4400065EE674A37EE647A83ED007A94ED007AE0
:10E4500065EE474A65EEE66A74EEE66AC3ED016A68
:10E4600065EEE77A26EE477A77EEC77AC3ED027A51
:10E4700037AD93E8070085E8070022AE86E807007D
:10E480000AAD85E807000DAE86E8070084E80700BE
:10E4900093ED007AD4ED007A27EE277AD3ED016A66
:10E4A000D4ED017A66EEA76AD3ED027AD4ED024A82
:10E4B00067EEA47A37EE267A77EE877A574F17EE13
:10E4C000902AA7EB620206EE902A9FED554A67EE6E
:10E4D000847A66EEA77A66EEA77ADFED524A74EE8A
:10E4E000E77A66EEA77A94ED007A27EE877A83EDD5
:10E4F000007AD4ED016A67EEA66AC3ED016A94ED75
:10E50000027A67EE877AC3ED027A0DF5B07C93E864
:10E5100007008CE807000DF5B67E8EE807000DF1C8
:10E520001C0C8CE8070084E8070094ED017A65EE86
:10E53000477AD4ED026A66EE663A77EEE37AC3ED87
:10E54000007A65EEE66AD4ED007A25EE675A76EE3B
:10E55000C56AC3ED016A26EE676A65EEC75A36EEF4
:10E56000656A83ED026A0DF1D00893E8070088E838
:10E5700007000DF1940E8EE8070085E8070086E895
:10E58000070084E8070093ED006A94ED007A26EE18
:10E59000076A93ED017AD4ED017A27EE277AD3ED5D
:10E5A000026AD4ED027A66EEA76A36EE076A36EEA4
:10E5B000867A17EE102AA7EB620207EE902A27EE62
:10E5C000047A27EE877A27EE877A34EEC77A67EEE9
:10E5D000877A94ED007A27EE877A83ED007A94EDBE
:10E5E000017A27EE877A83ED017A94ED027A67EE5D
:10E5F000877AC3ED027A52AD93E8070085E80700F9
:10E6000055AC84E80700D3ED000A9CED000A81F0C8
:10E61000D5FADFED057A20EE270AC5E412141F5F54
:10E6200012D3363FFF51D83FE02E654208B503793B
:10E63000994207D039B101230371806810B1036892
:10E640001B68984708BD0023F6E738B504460D4619
:10E650000121406873F046F92946606873F0C6F9F5
:10E6600038BD0000014A026041607047A4C10B0040
:10E6700008B5406803681B68984708BD08B58368FB
:10E680001979022904D0003918BF0121FFF7F0FFE2
:10E6900008BD08B583681979022904D0B1FA81F15F
:10E6A0004909FFF7E5FF08BD10B583681B79C2680B
:10E6B0001479022B0FD0022C0BD0027C012A1BD024
:10E6C000022A21D082B1124B124A602112484EF028
:10E6D000C9F9194600E021460229EED0003918BFD9
:10E6E0000121FFF7C5FF10BD13B11CB90021F5E7EB
:10E6F0000021F3E70121F1E713B91CB10121EDE796
:10E700000121EBE70021E9E7191B18BF0121E5E72B
:10E710004CC00B0054C00B0084C00B0038B504463D
:10E720000D461146FFF79EFF064B2360A560AB68C0
:10E7300013B9AC60204638BD034B044A1C21044881
:10E740004EF090F9C8C10B0098C00B00B0C00B0090
:10E7500084C00B0070B504460D4616461946FFF7F7
:10E7600081FF0D4B2360A560E6609DF81030237497
:10E77000AB682BB9AC60B36843B9B460204670BDD8
:10E78000064B074A3F2107484EF06CF9064B044AF6
:10E79000412104484EF066F9D4C10B00F4C00B00CF
:10E7A0000CC10B0084C00B0084C10B0010B50C46DB
:10E7B000094B186820B149B1084A802101F070FC6A
:10E7C000074803681B682146984710BD034A80210B
:10E7D00001F080FCF4E700BF147F0020FC230C0054
:10E7E00018610020012800D070474FF6FF7399424E
:10E7F000FAD110B582B00B4A0B4B13600D23536056
:10E800000A4C0B492046FFF789FF0A4B236001237E
:10E810000093094B094A0A490A48FFF79BFF02B0D7
:10E8200010BD00BF787C0020E0C10B006C7C002094
:10E8300018610020BCC10B003C6100202461002055
:10E8400030610020807C002008B54FF6FF71012068
:10E85000FFF7C8FF08BD0020704700002DE9F04118
:10E860002DED028B84B0804603685B68984707EE05
:10E87000900AB8EE678AD8ED087AF4EEC87AF1EE1D
:10E8800010FA58DC00240A2C37DC08EB44039D887E
:10E89000A84201D20134F6E7002C40D0204686F091
:10E8A00077FA02460B460020244986F023F90646F3
:10E8B0000F4607EE905AF8EEE77A38EE678A013C89
:10E8C00008EB4404A3885D1B07EE905AF8EEE77A44
:10E8D000C8EE277A17EE900A86F06CFA02460B46CD
:10E8E0003046394686F008F90022144B86F0BAFA11
:10E8F00086F0B0FD07EE900A01E0DFED117AFDEE43
:10E90000E77A17EE903ACDED017A00220292642266
:10E910000392002B06DB93420BDD03AB03E0DFED3C
:10E92000097AECE702AB186804B0BDEC028BBDE8D5
:10E93000F08101ABF7E74FF0FF30F5E7000024402E
:10E94000000000000000C84208B503681B68984733
:10E95000013018BF012008BD10B5044603685B688C
:10E96000984707EE900AF8EEE77A94ED077AF4EE0E
:10E97000C77AF1EE10FACCBF0120002010BD91F84B
:10E980005030012B14BF0023012390F850209342F4
:10E990001BD00122012380F8203091F8503080F8FC
:10E9A00050304B6D436591F85030012B21D000233E
:10E9B00080F8583091F8593080F8593091F85A3031
:10E9C00080F85A30CAB90020704791F85930012BAD
:10E9D00014BF0023012390F85920934201D0012253
:10E9E000D8E74A6D436D9A4201D00122D2E7002256
:10E9F000D0E791F95830DBB2DAE770B500F12806BC
:10EA00000546836A1C469E4207D0986803689B6847
:10EA10002946984708B92368F4E7002070BD70477D
:10EA200070477047704738B503460469826904EB44
:10EA3000620012F0010F02D15B69984738BD551092
:10EA400062595B69D358F8E738B5034604698269AF
:10EA500004EB620012F0010F02D15B69984738BDE8
:10EA6000551062595B69D358F8E708B5172072F062
:10EA7000DBFFB0FA80F0400908BD08B501210E2087
:10EA800072F0B4FF08BD08B501210E2072F02AFF14
:10EA900000210E2072F0AAFF0A206FF04EFD08BD83
:10EAA0002DE970432DED028B06467E4B93F8B43072
:10EAB000002B59D07C4A92F82820934210D07A4AF1
:10EAC00092F8102193421CD0774A92F8202093426A
:10EAD00028D0754A92F87020934234D0002344E045
:10EAE000724B1B7C2BB1714BDB68003B18BF0123C1
:10EAF0003BE06E4844F04AFC0028D4BF00230123C9
:10EB000033E06B4B1B7C2BB1694BDB68003B18BFC0
:10EB100001232AE0664844F063FD0028D4BF0023A7
:10EB2000012322E0634B1B7C2BB1624BDB68003B73
:10EB300018BF012319E05F4844F0E8FD0028D4BF66
:10EB40000023012311E05C4B1B7C2BB15A4BDB688B
:10EB5000003B18BF012308E0574844F067FE002837
:10EB6000D4BF0023012300E00023CBB94D4B93ED2C
:10EB7000288AB5EEC08AF1EE10FA3ADD96F8243014
:10EB800033B141F28831F06A2FF0ADFD002864D135
:10EB90006FF0BCFCF062FFF776FF0024254630E002
:10EBA000414B93F828203F4B93F8B4309A4210D051
:10EBB0003D4A92F8102193420FD03B4A92F8202010
:10EBC00093420ED0384A92F8702093420DD0002024
:10EBD0004AE0364844F05CFC46E0354844F094FC9A
:10EBE00042E0344844F0FCFD3EE0334844F07AFE15
:10EBF0003AE0B0EE088AC1E7202072F041FE0544F9
:10EC000001340E2CF8D92D4BA3FB0535ED0818EE79
:10EC1000100A86F0CFF80022294B86F023F98046AF
:10EC20008946284686F0A4F842464B4686F01AF9F3
:10EC300086F010FC08EE100AFFF71FFF96F824304C
:10EC4000B3B9D6ED0A7AF4EEC87AF1EE10FA01D52E
:10EC500086ED0A8A012386F82430D6ED0A7AFCEE86
:10EC6000E77A17EE903A98B2BDEC028BBDE870835C
:10EC7000D6ED0A8A78EE687A17EE900A86F09AF84E
:10EC80000022104B86F0EEF804460D4618EE900A6E
:10EC900086F090F822462B4685F02EFF86F0DAFBB0
:10ECA000B062DAE7B0B2002004870020987C002030
:10ECB000C87C0020087D0020307D0020898888885D
:10ECC00000200C400000E03F08B5406845F0FEFB26
:10ECD00008BD08B5406845F0D7F908BD08B54068DB
:10ECE00045F0B4F908BD08B5406845F017F908BD0E
:10ECF00008B5406845F05EF908BD0000012800D065
:10ED0000704738B54FF6FF73994200D038BD174DA4
:10ED1000284644F0DBFB164C2246164928467FF075
:10ED200073FD154D284644F013FC2246134928462E
:10ED30007FF06AFD124D284644F05EFD22461149DF
:10ED400028467FF061FD104D284644F0EDFD224637
:10ED50000E4928467FF058FD0D4D284645F0DEF956
:10ED600022460C4928467FF04FFDCFE7987C0020D3
:10ED70000060002099ED0200C87C00201FEA02001C
:10ED8000087D002021EA0200307D002023EA0200F5
:10ED9000607D002025EA020010B50446054B0360A3
:10EDA00003F134024261403383611C305CF041FD69
:10EDB000204610BD50E90C00F8B504460E4B002269
:10EDC0000E4902F0FBFC23460D4A43F8302B6363E7
:10EDD00023630027A76304F13C050A4E0FCE0FC53D
:10EDE00096E8030045F8040B2980E765676584F819
:10EDF00058702046F8BD00BF0C80002054940C00D1
:10EE0000D0C30B00B0C30B0008B50021172072F06F
:10EE100069FD0C4B186820230B4A0C4900F52A6049
:10EE200001F0A4FB0021202072F05CFD012072F0B3
:10EE3000F1FC0A2072F0E8FC054B064A1A6001203A
:10EE400008BD00BFBC7F0020F0C10B00C8BF0B0095
:10EE5000947C00204061002008B50D4B1B681C46C7
:10EE60000B4A934207D0986803689B680021984733
:10EE700008B92368F3E7BFF34F8F0649CA6802F465
:10EE8000E062054B1343CB60BFF34F8F00BFFDE73C
:10EE9000D030012000ED00E00400FA0508B50F4B6A
:10EEA000186818B100220E490BF096FB02F054FAD4
:10EEB0001F210C4B186827F037FE0D2072F0E7FD7C
:10EEC0000C2072F0E4FD0B2072F0E1FD01221146EE
:10EED0004FF0FF304EF0BAF808BD00BF9888002010
:10EEE00018C20B000CBE002010B50446124B1B6864
:10EEF0001BB9124B1B688BB910BD6FF007FB0E4B93
:10EF00001B689842F5D90E4B18680E4A0E4900F559
:10EF10002A6001F02BFB2046FFF79EFF6FF0F6FA08
:10EF2000064B1B689842E7D9044B00221A60204622
:10EF3000FFF7B4FFE0E700BF88880020A488002026
:10EF4000BC7F00202CC20B0038C20B000020704791
:10EF500010B5144B5B68E3B1134B93F8E030EBB1A1
:10EF6000104B586803681B680F4AD2F8E4109847A2
:10EF700004460E4B186800F52A608CB10C4B0D4A04
:10EF80000D4901F0F3FA14B10C4B064A1A60204601
:10EF900010BD45F06FF9034B5860DDE70024E8E74A
:10EFA000074BECE77061002004870020BC7F002045
:10EFB00050C20B0058C20B00C8BF0B00947C00204D
:10EFC00040C20B00002070470020704710B5044677
:10EFD000FFF7BCFF034628B12375002284F85820B0
:10EFE000184610BD2046FFF7B3FF03460028F3D1B3
:10EFF0002046FFF7E7FF03460028EDD12046FFF744
:10F00000E3FF03460028E7D12046FFF7FDFE034655
:10F01000E2E738B505460068854204D004684DF043
:10F02000EFFC2046F8E738BD38B505460068854254
:10F0300004D004684DF0E4FC2046F8E738BD38B54C
:10F0400005460068854204D004684DF0D9FC20468E
:10F05000F8E738BD38B505460068854204D0046835
:10F060004DF0CEFC2046F8E738BD000010B5044650
:10F07000044B40F8303BFFF7EDFF204602F06AFBFF
:10F08000204610BDD0C30B0010B50446064B40F817
:10F09000303BFFF7DFFF204602F05CFB20464DF0DF
:10F0A000AFFC204610BD00BFD0C30B002DE9F843D4
:10F0B00007460E4603688046814609E0BB68013B6F
:10F0C000BB6028467FF0ACFB28464DF099FC2346F8
:10F0D0001D4698450AD01C68996832689142F6D15D
:10F0E00003F108029642E9D19946F0E74F4508D06E
:10F0F000BB68013BBB6048467FF092FB48464DF041
:10F100007FFCBDE8F883000030B583B005460D4BA9
:10F11000036044682B1D9C4206D0019501A9A0689C
:10F12000FFF7C4FF2468F5E72C1D2046FFF771FFA9
:10F13000AC606C600023EB602046FFF76AFF284656
:10F1400003B030BD10C30B0010B50446FFF7DCFF61
:10F1500020464DF055FC204610BD000010B5044679
:10F16000024B0360FFF7D0FF204610BD24C30B0005
:10F1700010B50446064B40F8283BFFF755FF2046E4
:10F18000044B40F8043FFFF7BFFF204610BD00BF0F
:10F1900038C30B0024C30B0010B50446074B40F8DE
:10F1A000283BFFF741FF2046054B40F8043FFFF79F
:10F1B000ABFF20464DF024FC204610BD38C30B00A9
:10F1C00024C30B0010B50446044B0360FFF79CFFFB
:10F1D00020464DF015FC204610BD00BF24C30B0097
:10F1E0002DE9F84307460E4603688046814609E04C
:10F1F000BB68013BBB6028467FF012FB28464DF000
:10F20000FFFB23461D4698450AD01C689968326862
:10F210009142F6D103F108029642E9D19946F0E70E
:10F220004F4508D0BB68013BBB6048467FF0F8FA09
:10F2300048464DF0E5FBBDE8F883000030B583B0EB
:10F2400005460D4B036044682B1D9C4206D001957A
:10F2500001A9A068FFF7C4FF2468F5E72C1D20462C
:10F26000FFF7EDFEAC606C600023EB602046FFF71B
:10F27000E6FE284603B030BD48C30B0010B5044677
:10F28000FFF7DCFF20464DF0BBFB204610BD000021
:10F2900010B50446024B0360FFF7D0FF204610BDB7
:10F2A0005CC30B0010B504460A4B03600A4B40F8E0
:10F2B000343FFFF7C3FF2046084B40F8283BFFF7D9
:10F2C000B3FE2046064B40F8043FFFF71DFF2046E3
:10F2D00010BD00BF70C30B005CC30B0038C30B0034
:10F2E00024C30B0010B50446044B0360FFF7A6FFD0
:10F2F00020464DF085FB204610BD00BF5CC30B00CF
:10F3000010B504460B4B03600B4B40F8343FFFF73E
:10F3100095FF2046094B40F8283BFFF785FE204625
:10F32000074B40F8043FFFF7EFFE20464DF068FB27
:10F33000204610BD70C30B005CC30B0038C30B002C
:10F3400024C30B002DE9F04FA7B00446934B186877
:10F3500000285AD003689B68984728B301258F4B33
:10F3600018680368DB68984700B34FF0010A8B4BBD
:10F37000186803681B699847D8B10126002D4CD046
:10F38000864F386803685B68984780460590386800
:10F3900003681B68984700280DDB386803681B6802
:10F3A00098474FFA80FE3CE00025D8E74FF0000A6E
:10F3B000DDE70026E2E7B4F850B0A8EB0B0085F0DB
:10F3C000E7FC0022764B85F04DFD80468946A08FF4
:10F3D000A0EB0B0085F0DCFC02460B46404649469C
:10F3E00085F06AFE85F0EEFF1F90002320936423D2
:10F3F0002193002803DB984205DD21AB00E020AB20
:10F4000093F900E00DE01FABFAE702263546B2465D
:10F410004FF0FF3ECDF814E003E04FF0FF3ECDF893
:10F4200014E0604B22930027239706AB39465D48D2
:10F4300083E8030008AA0AA90B910A910C975A497C
:10F4400009910D920DF1380893E8030088E8030054
:10F450008DF84070119712A9139112911497534986
:10F46000089153492491259726A911E9030083E8BF
:10F47000030016A91791169118974E4915911992E4
:10F480001AAA93E8030082E803008DF870508DF803
:10F4900079A08DF87A60059B1D938DF878E06FF068
:10F4A00035F8E36D03F54343503398421FD9424B7F
:10F4B000186800F52A609DF87930012B14BF0023ED
:10F4C00001239DF87A20012A14BF002201221D9DEC
:10F4D0009DF87010012918D0002102910195009229
:10F4E000364A374901F042F86FF010F8E06504F150
:10F4F0003005236B1E469D420BD0986803689B68BD
:10F5000008A9984728B93368F4E79DF97810C9B27B
:10F51000E3E7224B186818B19DF87030012B13D027
:10F52000224B0893234B159315A8FFF787FE254B15
:10F53000089312A8FFF778FD1B4B099309A8FFF762
:10F54000E3FD27B0BDE8F08F9DF87930012BE7D0BF
:10F5500003685B689847B4F85030984203D300239F
:10F5600084F85830DCE794F858300133DBB284F883
:10F570005830114A1068144A114900F52A6000F009
:10F58000F5FF94F858300A2BCAD90B4B18680F4A6C
:10F590000B4900F52A6000F0E9FFC1E7947C0020E8
:10F5A0000000594057E8020024C30B0070C30B0051
:10F5B0007FE902005CC30B00BC7F00207CC20B0013
:10F5C000C8BF0B0038C30B00B8C20B00D4C20B007D
:10F5D00010B50446FFF7B6FE636D2BB193F82030EB
:10F5E0002BB144F6206010BD4FF0FF30FBE74FF029
:10F5F000FF30F8E710B50446074B036003F134020F
:10F600004261403383611C305CF013F920464DF0B9
:10F61000F7F9204610BD00BF50E90C0010B50446B4
:10F620004DF0EEF9204610BD10B504464DF0E8F956
:10F63000204610BD10B504464DF0E2F9204610BD3D
:10F6400010B504464DF0DCF9204610BD08B54FF664
:10F65000FF710120FFF752FB08BD00000C4B1A7927
:10F6600093F8980078B9022A0CD00A4B1B684BB16A
:10F6700093F85020012A01D00120704793F85930A7
:10F68000012B02D07047002070470120FAE700BF2D
:10F69000B0B200207C8800207047000008B5044B01
:10F6A0001868044A044900F52A6000F05FFF08BDAD
:10F6B000BC7F0020F4C30B00C8BF0B0008B5044B8F
:10F6C0001868044A044900F52A6000F04FFF08BD9D
:10F6D000BC7F002000C40B0038C20B00012800D002
:10F6E00070474FF6FF739942FAD130B583B02E4B75
:10F6F000009300231A462D492D4850F09BFB2D4CBA
:10F70000009400231A462C492C4850F093FB009497
:10F7100000231A462A492B4850F08CFB2A4B0093B1
:10F720002A4B2B4A2B492C4850F084FB2B4B00933F
:10F7300000231A462A492B4850F07CFB2A4B0093A1
:10F7400000231A4629492A4850F074FB294B00939C
:10F75000294B002229492A4850F06CFB294D2A4B9D
:10F76000009300231A462949284650F063FB284B92
:10F7700000930023274A2849284850F05BFB284B78
:10F780000093284B284A2949294850F053FB294C1B
:10F790002946204650F057FB274A284920467FF04B
:10F7A00033F803B030BD00BF10C40B0009FB0200EA
:10F7B000047F00201CC40B00D1FA0200E47E00206C
:10F7C00099FA0200A47E00200CC40B00BDF60200D2
:10F7D00099F6020089F80200947E002020C40B00F4
:10F7E00041F80200B47E002024C40B00B9F90200E5
:10F7F000847E00202CC40B00D9F8020069F90200B5
:10F80000F47E0020747E002034C40B009DF60200BC
:10F810003CC40B001DFA020019F90200C47E00204E
:10F8200040C40B00E5F80200E9F9020035FA0200D5
:10F83000D47E0020807D00200060002059FE07005B
:10F8400000B585B00C4B18680C4A0D4900F52A60CC
:10F8500000F08CFE0B4B186850B1002102916A46F3
:10F860000BF086F8029B1BB1032269466846984755
:10F8700005B05DF804FB00BFBC7F002048C40B004E
:10F88000C8BF0B009888002000B585B00D4B1868E4
:10F890000D4BD3F8AC300D4A0D4900F52A6000F04D
:10F8A00065FE0C4B186850B1002102916A460BF0BE
:10F8B0005FF8029B1BB1032269466846984705B072
:10F8C0005DF804FBBC7F0020B0B2002054C40B00E4
:10F8D00038C20B009888002008B501204DF016F9B9
:10F8E00008BD000000B585B00A4B186858B1002368
:10F8F00002936A4601210BF03BF8029B1BB10322E5
:10F9000069466846984701204DF000F905B05DF85A
:10F9100004FB00BF9888002000B585B00E4B186826
:10F920000E4A0F4900F52A6000F020FE0D4B1868C2
:10F9300058B1002302936A4601210BF019F8029B8B
:10F940001BB1032269466846984701204DF0DEF856
:10F9500005B05DF804FB00BFBC7F002070C40B0045
:10F96000C8BF0B009888002000B585B00E4B186802
:10F970000E4A0F4900F52A6000F0F8FD00204DF016
:10F98000C5F80C4B186858B1002302936A46012150
:10F990000AF0EEFF029B1BB10322694668469847B6
:10F9A00005B05DF804FB00BFBC7F00207CC40B00E9
:10F9B000C8BF0B009888002000B585B001204DF02D
:10F9C000A5F8084B186850B1002102916A460AF068
:10F9D000CFFF029B1BB1032269466846984705B0DA
:10F9E0005DF804FB9888002008B5FFF737FE00B1EA
:10F9F00008BD064B1868064A064900F52A6000F063
:10FA0000B5FD0E21044850F0CBFAF1E7BC7F002091
:10FA10008CC40B0038C20B00807D002008B5FFF7B6
:10FA20001DFE00B908BD0D21014850F0B9FAF9E7F3
:10FA3000807D002000B585B0FFF710FEA0B1114B0E
:10FA4000186858B1002302936A4601210AF090FF1A
:10FA5000029B1BB1032269466846984701204DF07E
:10FA600055F805B05DF804FB074B1868074A0849CC
:10FA700000F52A6000F07AFD0E21064850F090FA59
:10FA8000EFE700BF98880020BC7F00208CC40B00EB
:10FA900038C20B00807D002008B5094B1868094A60
:10FAA000094900F52A6000F061FD084BD3F8A80071
:10FAB00022F0E2F8012200214DF0C8FA08BD00BF93
:10FAC000BC7F0020A8C40B00C8BF0B00B0B2002050
:10FAD00008B5094B1868094A094900F52A6000F081
:10FAE00045FD084BD3F8A80022F0C6F800221146C5
:10FAF0004DF0ACFA08BD00BFBC7F0020C0C40B00B5
:10FB0000C8BF0B00B0B2002008B5064B1868064A03
:10FB1000064900F52A6000F029FD6EF0F7FC044B61
:10FB2000186008BDBC7F0020CCC40B00C8BF0B0010
:10FB3000A48800202DE9F04F85B0CD4B1B790393AD
:10FB4000FFF78CFD0246CB4B186800F52A6014467F
:10FB5000002A00F01D820123C74AC84900F006FDB3
:10FB6000002C00F01782C64AC64CC74B01930025F3
:10FB7000009540F6B833C549204650F0A7F9C44B6C
:10FB8000019300950223C34AC349204650F076F9F9
:10FB9000039B022B00F00082BE4ADFF8FC92B94CB6
:10FBA000BE4B01930025009504234946204650F0A2
:10FBB00065F9BB4EBB4B0193009504233246314699
:10FBC000204650F05BF9B84FDFF8E082CDF80480B2
:10FBD000009501233A464946204650F04FF9CDF8AA
:10FBE0000480009501233A463146204650F046F9FC
:10FBF000FFF734FD002800F0D181A14ADFF894928C
:10FC0000A04CAA4F019700250095012349462046A4
:10FC100050F034F9DFF868A20197009501235246AD
:10FC20005146204650F02AF99F4E01970095012336
:10FC300032463146204650F021F9DFF884B2019770
:10FC4000009501235A465946204650F017F9984F1F
:10FC5000DFF87082CDF8048000950A233A468B497C
:10FC6000204650F00BF9CDF8048000950A233A465F
:10FC70008949204650F002F9CDF8048000950A2306
:10FC80003A468749204650F0F9F8CDF804800095AF
:10FC90000A233A464946204650F0F0F8CDF8048051
:10FCA00000950A233A463146204650F0E7F8CDF851
:10FCB000048000950A233A465946204650F0DEF863
:10FCC0007C4FDFF80482CDF80480009510233A467B
:10FCD0006E49204650F0D2F8CDF8048000951023EC
:10FCE0003A466D49204650F0C9F8CDF80480009599
:10FCF00010233A466A49204650F0C0F8CDF80480F7
:10FD0000009510233A464946204650F0B7F8CDF802
:10FD10000480009510233A463146204650F0AEF854
:10FD2000CDF80480009510233A465946204650F0FD
:10FD3000A5F8614F01970095112332465649204698
:10FD400050F09CF801970095112332465449204603
:10FD500050F094F801970095112332464946204609
:10FD600050F08CF801970095112332463146204619
:10FD700050F084F8019700951123524651462046D1
:10FD800050F07CF84D4F01970095072332464946C5
:10FD9000204650F073F8019700950723324631460C
:10FDA000204650F06BF8039B022B40F0F980444E44
:10FDB000DFF8E4B0334CDFF81481CDF8048000257F
:10FDC00000950B2332465946204650F057F8CDF89F
:10FDD000048000950B2332463149204650F04EF8FE
:10FDE000DFF8B090CDF8048000950B2332464946E9
:10FDF000204650F043F8DFF8B0A0CDF8048000951D
:10FE00000B2332465146204650F038F81C4FCDF8AF
:10FE1000048000950B2332463946204650F02EF8D8
:10FE2000DFF8AC80CDF8048000950D233A465946A2
:10FE3000204650F023F8CDF8048000950D233A4673
:10FE40001749204650F01AF8CDF8048000950D238C
:10FE50003A464946204650F011F8CDF80480009506
:10FE60000D233A465146204650F008F832E000BFD4
:10FE7000B0B20020BC7F0020DCC40B0038C20B00F5
:10FE8000D47E0020807D0020F8C40B00747E00200A
:10FE900008C50B00847E0020947E002014C50B0052
:10FEA000B47E00203CC50B00C47E002060C50B0062
:10FEB000A47E0020047F00207CC50B008CC50B00B5
:10FEC000F47E002068C50B0070C50B00C4C50B0094
:10FED000D0C50B004D4B019300950E235246394679
:10FEE00020464FF0CBFF4A4B019300950C2352461E
:10FEF000314620464FF0C2FF464B0193009509233F
:10FF00004A46494620464FF0B9FF434BD3F88C018F
:10FF10001B79022B74D04FF4167121F0A0FE03461A
:10FF20003E4A0192002200923D4A3E493E484FF02F
:10FF3000CDFF394BD3F88C011B79022B62D04FF4E3
:10FF4000167121F08CFE0346344A01920022009281
:10FF5000334A364934484FF0B9FF2F4BD3F88C0160
:10FF60001B79022B50D04FF4167121F078FE034616
:10FF70002B492D4C294A0192002200920A46204624
:10FF80004FF0A4FF204650F062F805B0BDE8F08FB6
:10FF90000023E1E5234AE7E5254AFEE5214A2DE66F
:10FFA000C846DFF88C90234B01932E46009504231E
:10FFB0004246494620464FF061FF1A4D1E4F0197B9
:10FFC000009605232A461D4920464FF057FF01970A
:10FFD000009605232A46494620464FF04FFF0197D9
:10FFE000009605232A46414620464FF047FF0197D9
:10FFF000009605232A46294620464FF03FFFD6E6C5
:020000023000CC
:1000000001218AE701219CE70121AEE7E0C50B0051
:10001000F4C50B0008C60B00B0B200201CC60B00D4
:10002000847E0020C47E0020807D0020D47E0020BD
:10003000B47E0020A0C50B00B4C50B00947E002048
:1000400008B54FF6FF710120FFF748FB08BD00001F
:1000500010B4074CD4F8B800D4F8BC1010401940C4
:1000600050EA010314BF012000205DF8044B7047E3
:10007000B0B2002000B583B00368064A1068009152
:10008000054A064900F52A6000F070FA03B05DF8F1
:1000900004FB00BFBC7F002030C60B0038C20B0041
:1000A000F8B504461546D0E900670A4641EA06005D
:1000B0003946C4E90001BF4208BFB04204D0002362
:1000C0002046FFF7C5FF00B9F8BD29462046FFF7D7
:1000D000D1FFF9E72DE9F84304460B461546D0E970
:1000E0000067CA434FEAE27902EA060009EA07011B
:1000F000C4E90001B94208BFB04205D09AB200235A
:100100002046FFF7A5FF08B9BDE8F8832946204639
:10011000FFF7B0FFF8E7000008B510204CF04CFCEA
:1001200000220023C0E9002300230372014B186062
:1001300008BD00BF147F002008B50A4B93F8F031CA
:100140006BB1084B93F89F22064B93F8A43103B18F
:100150001AB1806803681B689847012008BD014BED
:100160005A79F1E7B0B2002010B5044600F1100151
:1001700001206EF019FCE06010BD00002DE9F04197
:1001800082B0074688460193A021304888F0EEFCF3
:1001900006469F2804D92D4B0A2283F89E209F26CD
:1001A000002403E0294B23221A550134A64209D921
:1001B000264B1D5D284685F04DFE0028F5D10A2D01
:1001C000F0D1F2E7B8F1000F2BD02149404687F07B
:1001D0006BF928B93B685B6805221E493846984789
:1001E0001D49404687F060F928B93B685B680522E5
:1001F0001A49384698471A49404687F055F928B9B0
:100200003B685B68052217493846984716494046BF
:1002100087F04AF928B93B685B68052213493846DC
:1002200098473B685B683246084938469847044619
:10023000B8F1000F05D03B685B6804220C493846D2
:100240009847204602B0BDE8F08100BF187F00202B
:10025000C8BF0B0040C60B0038C20B0048C60B00DD
:1002600050C60B0058C60B00FCBF0B0060C60B004D
:1002700068C60B002DE9F04782B004460D461746CC
:1002800098465749284687F00FF928B923685B68D4
:1002900005225449204698475349284687F004F9D7
:1002A00028B923685B680522504920469847504981
:1002B000284687F0F9F828B923685B6805224D497C
:1002C000204698474C49284687F0EEF828B923681D
:1002D0005B6805224949204698474949284687F0E6
:1002E000E3F828B923685B68052246492046984709
:1002F0000121084609F022F8024600285CD0424B52
:10030000A3FB0201090C414800FB112101F5A831B2
:1003100001F5C07183FB01235E18CB17C3EB2643A5
:1003200000FB13133A4A82FB032909EB03024FEA4D
:10033000E379C9EBE2294FF4616606FB1933354ACC
:1003400082FB032A0AEB03024FEAE37ACAEB621A42
:10035000CAEB0A16A3EB86062A462F4920466CF004
:1003600015FF2E4920466CF011FF6EF0CFF82C4B94
:10037000A3FB003080090190009653464A46294964
:1003800020466CF003FF284B1E6866B127492046C3
:100390006CF0C4FE06F11C0120466CF0B8FE244946
:1003A00020466CF0BBFE43463A4629462046FFF7FE
:1003B000E5FE02B0BDE8F0872A46174920466CF0FA
:1003C000E5FE164920466CF0E1FE6EF09FF8144AF7
:1003D000A2FB00329209174920466CF0D7FED2E703
:1003E000C8BF0B0040C60B0038C20B0048C60B004C
:1003F00050C60B0058C60B00FCBF0B0060C60B00BC
:1004000070C60B0078C60B0007452EC28051010054
:10041000C5B3A2918988888880C60B0068C60B0086
:10042000D34D621084C60B00B0810020ACC60B0017
:10043000B0C60B009CC60B000B78433B142B0CD8AA
:10044000DFE803F01315110B0B0B0D0B0B0B0B0B54
:100450000B0B0B0B0B0B0B0B0F000020704714202A
:1004600070471E20704728207047322070470A20AE
:10047000704700002DE9F047EAB0364C94F8A042EE
:100480006CB10746884616461D46334B1B7833B978
:10049000324B186818B10368DB68984710B96AB026
:1004A000BDE8F087304687F055F8824600F1010933
:1004B00048464CF093FA04462B463246494688F0AB
:1004C00055FB814682450ED214B120464CF09CFA71
:1004D00009F1010948464CF081FA04462B463246A0
:1004E000494688F043FB1E4B1D684FF4D4721D49EA
:1004F000684685F033FD41463846FFF79DFF8DF88D
:10050000A4012146684686F0D9FF1DB1E96961A8BA
:1005100086F0D4FF0121084608F010FF60904FF4E8
:10052000D5704CF05BFA05466B460F4A4FF4D57117
:1005300030F0A4FE02462946084B18684AF09CFD9C
:1005400014B120464CF060FA002DA8D028464CF09B
:100550005BFAA4E7B0B200207988002074880020FC
:10056000B0810020E0C60B0080880C000CB42DE99F
:10057000F04182B006460F46DDF82080404686F006
:10058000E9FF044602304CF029FA0546414686F060
:1005900095FF0A232B55013400232B551A4B93F852
:1005A000F13023B11949384686F07EFF80B1F068FA
:1005B00028B14FF0FF316EF0EFFA01280ED015B1DF
:1005C00028464CF021FA02B0BDE8F04102B0704775
:1005D000002DF8D028464CF017FAF4E709AB019348
:1005E0003268D4682A4639463046A047019B2A46DD
:1005F00039463046FFF73EFF00231A461946F06899
:100600006EF038F9DBE700BFD8BB0020C8BF0B0095
:1006100070B582B005460E4661B1941B01940F2C53
:100620000DD82868012C13D0A4B12246314685F09C
:1006300095FC0FE09142F0D00A487EF0ABF9002221
:1006400001A928467EF00CFB2860019BAB60E8E71F
:1006500033780370019B6B602A680021D15402B08B
:1006600070BD00BFB4C60B000CB42DE9F04182B0E0
:100670000746089E746864000023019303E01B1B77
:1006800032D401331C44A04620464CF0A7F905465D
:100690000198019508B14CF0B7F93168284686F009
:1006A0000DFF09AB009332684146284688F05EFA98
:1006B000031EE4DB9C42E2DD07F108033B60ADB1C1
:1006C000284686F047FF2A184FF00003294638468F
:1006D000FFF79EFF15B128464CF096F9384602B058
:1006E000BDE8F04102B07047DB43CBE76A1EEBE7A1
:1006F00010B5094B1B6843B904204CF05DF9044662
:1007000000F0CCFE044B1C6010BD044B044A0A21CF
:1007100004484CF0A7F900BFB87F0020A0C80B0028
:10072000ACC80B00BCC80B0070B584B005460C46C5
:100730001646104B196803A800F0E5FE0E4B18682A
:10074000009623460D4A0E4900F52A60FFF70EFF7A
:100750000C4E2146304666F07FF901232246314691
:10076000284666F0FBF803A800F0D5FE284604B042
:1007700070BD00BFB87F0020BC7F0020CCC80B003C
:10078000C8BF0B00184C0120F8B504460E461546AC
:1007900000274760084B40F8083B6DF00FFC2A46E5
:1007A000314604F11400FFF7BFFF84F8785084F855
:1007B00079702046F8BD00BFF0C80B0070B500F19D
:1007C0001404204666F0ABFB054608B9284670BD08
:1007D000054E306800F082FE204666F023FB30684C
:1007E00000F086FEF2E700BFB87F002070B5044637
:1007F0000D4600F11406304666F091FB08B9002062
:1008000070BD94F879306B4084F8793029463046D1
:1008100066F052F9F4E72DE9F04105460F46164619
:1008200000F11408404666F07AFB88B10023B34219
:1008300007D2FC5C95F87900444085F87940013393
:10084000F5E732463946404666F043F9BDE8F081A7
:100850000020FBE77047704708B50368DB6A9847DC
:1008600008BDA0F53060FFF7F7BF000008B50349E9
:10087000D0F880062DF037FF08BD00BFA0BB0D00EB
:1008800008B50346084890F8A40118B1064890F846
:100890009F0200B908BD012083F82D0B83F898084A
:1008A00018462AF0A7F8F5E7B0B2002038B505469B
:1008B0000C460A2905D0214605F52A60FFF73CFCC5
:1008C00038BD0D2100F52A60FFF736FCF3E738B597
:1008D0000C46A0F52A650A2905D0214605F52A60AF
:1008E000FFF72AFC38BD0D2105F52A60FFF724FC2F
:1008F000F3E708B5002100F5306000F041FF08BDC6
:1009000070B582B0044616461D4690F82D0B18B1FE
:100910000E4B93F8A0323BB92B46324604F52A60C1
:10092000FFF7A8FC02B070BD04F52A60FFF784FD54
:100930000146074B1B6833B1DA6900953346204600
:100940002DF06CFEEEE7034AF7E700BFB0B20020DF
:10095000B0810020FC230C00A0F52A60FFF7D0BF77
:1009600010B504460A4B03F10802026003F150027D
:10097000C0F8A02A6833C0F8003B00F5306000F0F2
:10098000E9FE044B2360204629F054FE204610BDAA
:1009900050C90B0074700C0010B5A0F530640A4B00
:1009A00003F10802226003F1500240F8602C683322
:1009B000C4F8003B00F0CEFE044B2360204629F033
:1009C00039FE204610BD00BF50C90B0074700C00EA
:1009D00010B504460C4B03F10802026003F150020B
:1009E000C0F8A02A6833C0F8003B00F5306000F082
:1009F000B1FE064B2360204629F01CFE20464BF03A
:100A0000FFFF204610BD00BF50C90B0074700C00E2
:100A100010B5A0F530640B4B03F10802226003F11E
:100A2000500240F8602C6833C4F8003B00F092FE9E
:100A3000054B2360204629F0FDFD20464BF0E0FFEA
:100A4000204610BD50C90B0074700C00F8B5044668
:100A500028F01AFD324B2360324EC4F888664FF4FA
:100A600001773A46002104F28C6085F09FFA002558
:100A7000C4F89058C4F89458012384F898383A463A
:100A8000294604F6990085F091FAC4F8A45A264B39
:100A9000C4F8A03AC4F8A86AC4F8AC5A234B2A4652
:100AA000234904F5306000F089FE224B03F108026F
:100AB000226003F15002C4F8A02A6833C4F8003B56
:100AC00084F82D5B032384F884361B4B1B686BB9B9
:100AD000194B1C60002384F898384FF4E131114819
:100AE000F6F762FD6DF012FD054608E0134B144A5F
:100AF000362114484BF0B6FF64206DF01EFD094806
:100B0000F6F784FD30B941F2883128462DF0EBFD2F
:100B10000028F1D120462DF061FD2046F8BD00BF30
:100B200074700C00186D002090C80B000C80002021
:100B3000FCC80B0050C90B00BC7F00200CC90B0087
:100B400018C90B0038C90B0008B54FF433604BF0DF
:100B500033FFFFF77BFF034B186800F52A60FFF7B0
:100B600003FB08BDBC7F002008B50248F6F7C9FCAE
:100B700008BD00BF186D002010B50446024B03608D
:100B800000F0E8FD204610BD88CA0B0010B50446F1
:100B9000044B036000F0DEFD20464BF031FF2046A1
:100BA00010BD00BF88CA0B00D0F83C0170470000A0
:100BB00008B5FFF7F9FF034BA3FB0030C0F3C220D9
:100BC00008BD00BFC5B3A29170B5044690F8A4510A
:100BD000FFF7EEFF854200D170BD0346214A106841
:100BE000214A224900F52A60FFF7C0FC0623002BAA
:100BF00027DB581C03F1500204EB8202556803F115
:100C0000510204EB8202556003F1580204EB8202A8
:100C1000566803F1590104EB81014E6003F1600154
:100C200004EB81014E6803F1610104EB81014E6028
:100C30000F4941F8205051680E4A42F82010013BFC
:100C4000D5E70023C4F84431C4F86431C4F88431D2
:100C5000074A1360074A13602046FFF7A9FF84F88C
:100C6000A401B9E7BC7F0020D8C90B00C8BF0B00A6
:100C7000E47F0020C47F002008B5FFF795FF074BF5
:100C8000A3FB0023DB080648A0FB0320800800EB41
:100C90004000A3EB4000C0B208BD00BFCDCCCCCC1F
:100CA000ABAAAAAA08B5FFF77FFF064BA3FB001269
:100CB0005209A3FB02304009C0EB0010A2EB8000F8
:100CC000C0B208BD8988888838B50446154669B120
:100CD000012927D0022938D02046FFF7CDFF0C305C
:100CE00054F820202A4444F8202038BD1E4B1868B0
:100CF00013461E4A1E4900F52A60FFF737FCD4F858
:100D000044312B44C4F844311A4A13682B4413600D
:100D10002046FFF7C7FF123054F820302B4444F828
:100D20002030D9E7104B18681346134A104900F5D4
:100D30002A60FFF71BFCD4F864312B44C4F86431FB
:100D40000E4A13682B441360C6E7074B1868134616
:100D50000B4A074900F52A60FFF708FCD4F88431F4
:100D60002B44C4F88431B7E7BC7F002000CA0B00D5
:100D7000C8BF0B00E47F002010CA0B00C47F002016
:100D800020CA0B0070B50446D0F83C310133C0F8DE
:100D90003C31FFF771FF05462046FFF783FF94F8CB
:100DA000383183B3002305E003F11202002144F837
:100DB000221001333B2BF7D9002305E003F10C028D
:100DC000002144F822100133052BF7D9002310E04D
:100DD00003F1500204EB82020021516003F158023A
:100DE00004EB8202516003F1600204EB8202516065
:100DF0000133072BECDD002384F8383184F83951B6
:100E00004FF47A7070BD06462046FFF7DDFE94F879
:100E10003931AB4205D084F839510C35002344F800
:100E2000253094F83A31B342EAD084F83A6106F1B9
:100E30001200002344F82030E2E7000000231A46A5
:100E4000052B06D803F10C0150F821100A44013398
:100E5000F6E707EE902AF8EE677A9FED047A87EEC0
:100E6000870ADFED037A20EE270A704700606A47A1
:100E70000000C84200231A4605E003F1120150F8B1
:100E800021100A4401333B2BF7D907EE902AF8EEE4
:100E9000677A9FED047A87EE870ADFED037A20EE0A
:100EA000270A704700BA5B4A0000C84210B571B10A
:100EB00090F84141FFF7C2FF07EE904AF8EEE77A5B
:100EC000B4EEE70AF1EE10FA04D5012010BD90F857
:100ED0004041EFE7054B18682346054A054900F5F0
:100EE0002A60FFF743FB0020F0E700BFBC7F002033
:100EF0003CCA0B0050C60B0030B52DED028B83B001
:100F00001D4B93F8C4518DBB04461C4B1B6893EDDD
:100F1000038ADFED1B7AB4EEE78AF1EE10FA24D5EE
:100F2000FFF7A8FF94F8423107EE903AF8EEE77A1F
:100F300067EE887ADFED126A87EEA67AB4EEC70A0A
:100F4000F1EE10FA01D5012510E00E4B1C6804F5F6
:100F50002A6417EE100A83F02DFFCDE900010A4A3A
:100F60000A492046FFF702FB00E00125284603B0AE
:100F7000BDEC028B30BD00BFB0B2002028BF002006
:100F80000000C842BC7F002058CA0B0050C60B00AE
:100F90003B23002B1ADB03F1120200EB8202D2ED9D
:100FA000007AF8EE677ADFED0A6A87EEA67A30EE0D
:100FB000470AB4EEE00AF1EE10FA02D4013B5BB24C
:100FC000E7E7D8B2C0F13B00C0B270473C207047A1
:100FD00000A00C4738B50446174B0022174900F013
:100FE000EDFB2346164A43F8302B002525635D6050
:100FF0009D60DD601D615D61F022294604F14800BD
:1010000084F0D4FF012384F8383184F8395184F80E
:101010003A51C4F83C51282384F84031192384F80C
:101020004131322384F842316422294604F5A2700A
:1010300084F0BCFF204638BD0C80002078CA0B002D
:1010400088CA0B0038B503460469826904EB620064
:1010500012F0010F02D15B69984738BD55106259F3
:101060005B69D358F8E7000008B5164B93F85D208C
:10107000531EDBB2012B1CD9042A1AD00B791D2B6D
:1010800010D80A2B15D30A3B132B12D8DFE803F034
:101090000F0F131311111113131313111111161133
:1010A00011160F0FAF2B04D100F08CF901E000F006
:1010B000F9F8002008BD00F061F9FAE700F070F9D6
:1010C000F7E700BFB0B2002070B505460C46061D1C
:1010D0000C204BF071FC846031467DF09AFBEB688C
:1010E0000133EB600C204BF067FC856021467DF0FE
:1010F00090FBA3680133A36070BD000010B584B0FD
:101100000446104B0293002203926B4604A911E996
:10111000030083E80300211DA1606160E2600A4AC8
:101120002260246104F1140293E8030082E80300C2
:10113000064B196811B12046FFF7C6FF204604B0E0
:1011400010BD00BF69100300C4CA0B00BC8600209C
:1011500038B505460068854204D004684BF050FC61
:101160002046F8E738BD2DE9F84307460E460368E8
:101170008046814609E0BB68013BBB6028467DF0A4
:101180004FFB28464BF03CFC23461D4698450AD0B1
:101190001C68996832689142F6D103F108029642C0
:1011A000E9D19946F0E74F4508D0BB68013BBB60E9
:1011B00048467DF035FB48464BF022FCBDE8F883FD
:1011C00030B583B005460D4B036044682B1D9C422F
:1011D00006D0019501A9A068FFF7C5FF2468F5E7CF
:1011E0002C1D2046FFF7B4FFAC606C600023EB6061
:1011F0002046FFF7ADFF284603B030BDB0CA0B0054
:1012000010B50446FFF7DCFF20464BF0F9FB204603
:1012100010BD000010B50446024B0360FFF7D0FF7D
:10122000204610BDC4CA0B0010B50446044B036031
:10123000FFF7C6FF20464BF0E3FB204610BD00BF82
:10124000C4CA0B0000000000F8B5154B93F85D30E0
:10125000013BDBB2012B1ED905460F46104BDB6864
:10126000CBB10024BC4216DA05EBC406726855F80F
:1012700034100B4B187B6CF033FA706883F088FDE8
:1012800005A3D3E9002383F0EDFD84F0C3F86DF0EE
:1012900054F90134E6E7F8BDCDCCCCCCCCCCF43F4E
:1012A000B0B2002000B583B0064A6B4692E8030056
:1012B00083E8030001211846FFF7C6FF03B05DF87D
:1012C00004FB00BFD0CA0B0000B583B06B46064AD2
:1012D00092E8030083E8030001211846FFF7B4FFFA
:1012E00003B05DF804FB00BFD8CA0B0030B587B06F
:1012F0006C46064D0FCD0FC495E8030084E803004B
:1013000003216846FFF7A0FF07B030BDE0CA0B001D
:1013100030B587B06C46064D0FCD0FC495E803007D
:1013200084E8030003216846FFF78EFF07B030BD55
:10133000F8CA0B0030B587B06C46064D0FCD0FC410
:1013400095E8030084E8030003216846FFF77CFF6B
:1013500007B030BD10CB0B0030B587B06C46064DE2
:101360000FCD0FC495E8030084E80300032168460D
:10137000FFF76AFF07B030BD28CB0B0000B583B084
:101380006B46064A92E8030083E8030001211846F1
:10139000FFF75AFF03B05DF804FB00BF40CB0B0022
:1013A00000B583B06B46064A92E8030083E8030069
:1013B00001211846FFF748FF03B05DF804FB00BFAA
:1013C00048CB0B0030B58DB06C46074D0FCD0FC428
:1013D0000FCD0FC495E80F0084E80F000621684682
:1013E000FFF732FF0DB030BD70CB0B0010B50446D7
:1013F0000322002101206DF017FA206008B1204679
:1014000010BD034B034A0C2103484BF02BFB00BFDC
:10141000A0CB0B00ACCB0B00ECCB0B0010B5044603
:1014200000686DF09BFC204610BD10B504464FF4DB
:101430007A7200238802890D84F0BAF90146206887
:101440006DF0AAFB003818BF012010BD08B50023BD
:101450001A46194600686DF00DFA08BD08B5006817
:101460006DF0E4FA08BD10B50446FFF7BFFF204653
:1014700010BD10B50446FFF7D1FF204610BD08B5DA
:10148000FFF7D3FF80F00100C0B208BD08B5FFF739
:10149000DDFF08BD08B5FFF7E1FF08BD10B5044644
:1014A0000322002101206DF0BFF9206038B1002334
:1014B0001A4619466DF0DEF938B1204610BD044BCE
:1014C000044A0B2104484BF0CDFA84F037FB00BFEF
:1014D00018CC0B0020CC0B003CCC0B0008B54FF017
:1014E000FF3100686DF058FB00B108BD84F026FBA9
:1014F00008B500231A46194600686DF0BBF900B123
:1015000008BD84F01BFB10B5044608462160FFF7B8
:10151000E5FF204610BD10B504460068FFF7E8FF60
:10152000204610BD70B504460E4612B91046236B16
:1015300053B90125257523681B680021204698476B
:10154000024B1D702663284670BD00BF96880020A0
:1015500010B5FFF7E7FF044608B9204610BD024862
:10156000FFF794FFF9E700BFB881002038B50C46BB
:1015700011461A46FFF7D6FF054608B9284638BD7A
:1015800021460248FFF786FFF8E700BFB881002038
:1015900070B504460D4611461A46FFF7D9FF0646B8
:1015A00008B9304670BD2946204600F0E9F8F8E752
:1015B00008B5016B0023036311B103681B6A9847E8
:1015C00008BD08B500220275FFF7F2FF4FF0FF30AB
:1015D00008BD08B50022027503681B686FF0004162
:1015E00098476FF0004008BD10B50446034B40F823
:1015F0001C3B6CF09BFC204610BD00BFC4540D008A
:1016000030B583B005464FF056FA0446184B1B78A8
:1016100003B168B9174B1B7813B12B7D03B18CB1A3
:10162000154B1B780BB12B7DC3B1204603B030BDE9
:10163000124B1868EB69124A124900F52A60FEF74E
:1016400095FFE7E70D4B18686B680093EB690E4A4E
:101650000C4900F52A60FEF789FFE1E7074B18689F
:10166000EB690A4A074900F52A60FEF77FFFDCE7CD
:10167000B4810020AC810020AD810020BC7F00201F
:1016800084CC0B00C8BF0B0094CC0B00A8CC0B0083
:1016900038B504460B4B18600368DB69984705466C
:1016A0006CF034FF014620464FF0F4F9002D04DBC6
:1016B00023681B68294620469847024B00221A607F
:1016C00038BD00BFB0810020012800D070474FF620
:1016D000FF739942FAD170B50F4D002128464FF0A3
:1016E000F9FA0E4C0E4E2246314628467DF08CF813
:1016F0000C4D002128464FF0EDFA2246314628468F
:101700007DF082F8084D2846FFF7ADFE22460749D6
:1017100028467DF079F870BD0C8000200060002024
:10172000E9150300DC800020B88100207314030059
:1017300008B5044904486CF0B9FC044904486CF04D
:10174000B5FC08BDBCCC0B0028800020CCCC0B0025
:10175000F880002010B50446074B0360806A10B182
:1017600021464FF0A4FA2046044B40F81C3B6CF095
:10177000DDFB204610BD00BF8CCD0B00C4540D0016
:1017800010B5044641606CF0C1FE63681844E06027
:1017900010BD000008B5054B1B7803B108BD044B14
:1017A000044A8D2104484BF05DF900BF08800020F9
:1017B000DCCC0B00ECCC0B0010CD0B0070B504465C
:1017C0000D461E4600214FF081F90D4B2360A662A5
:1017D000002384F82C30FFF7DDFF294604F11C00BC
:1017E0006CF064FCA06A18B121464FF01DFA08B1F4
:1017F000204670BD034B044A262104484BF032F9C1
:101800008CCD0B0030CD0B0038CD0B0010CD0B0074
:1018100008B54FF6FF710120FFF756FF08BD70476E
:101820007047000082B0084B1B680020DAB262F3F8
:101830000700C3F3072262F30F20C3F3074363F3E8
:10184000174002B0704700BFBC81002000207047E5
:1018500082B0084B1B680020DAB262F30700C3F3C2
:10186000072262F30F20C3F3074363F3174002B06C
:10187000704700BFBC81002000207047024A026010
:1018800000220271704700BFD8CD0B0000B583B0B5
:101890000379B3B1144B1B68ADF804301B0C8DF801
:1018A000063000209DF8043063F307009DF80530F2
:1018B00063F30F209DF8063063F3174003B05DF823
:1018C00004FB0A4B1B68009303685B696A460421AA
:1018D00098478DF80400C0F307238DF80530C0F356
:1018E00007408DF80600DCE7BC810020ACCD0B0082
:1018F00000B583B00D4B5B68ADF800301B0C8DF864
:10190000023003685B696A4603219847034600205A
:10191000DAB262F30700C3F3072262F30F20C3F3C6
:10192000074363F3174003B05DF804FBACCD0B0035
:1019300010B584B003460D4A92E803000190ADF85B
:1019400008101A68546901AA06211846A0470346E0
:101950000020DAB262F30700C3F3072262F30F201C
:10196000C3F3074363F3174004B010BDB4CD0B00BD
:1019700010B584B004466B460C4A07CA03C31A70FC
:1019800023685B696A460921204698470346002080
:10199000DAB262F30700C3F3072262F30F20C3F346
:1019A000074363F3174004B010BD00BFBCCD0B006C
:1019B00000B583B00C4B9B8BADF8003003685B69BE
:1019C0006A460221984703460020DAB262F3070014
:1019D000C3F3072262F30F20C3F3074363F31740F7
:1019E00003B05DF804FB00BFACCD0B00017042708A
:1019F000704710B5044600221146FFF7F7FF204656
:101A000010BD03780BB90A7842B94BB10B784BB1D2
:101A100042784B789A4207D30020704701207047E4
:101A200000207047002070470120704782B0ADF859
:101A300004200170BDF80420A0F8012002B0704716
:101A4000012800D070474FF6FF739942FAD110B5C4
:101A5000044C2046FFF7CDFF226800210248FFF723
:101A6000E5FF10BDC0810020BC81002008B54FF605
:101A7000FF710120FFF7E4FF08BD0000012800D03E
:101A8000704708B54FF6FF73994200D008BD04486F
:101A900000230360034A04497CF0B6FEF6E700BF6A
:101AA000C481002000600020E91A030038B5054613
:101AB000054B1C6834B1606803681B682946984769
:101AC0002468F7E738BD00BFC481002070B50E461A
:101AD00015460868A84204D004684AF091FF2046E1
:101AE000F8E73560284670BD10B50446002201466F
:101AF000FFF7ECFF204610BD38B50C461546082010
:101B00004AF05AFF2A68426022680260206038BDAD
:101B100010B582B00446054B03600190044801AA49
:101B20000146FFF7E9FF204602B010BDF8CD0B00DB
:101B3000C481002008B54FF6FF710120FFF79EFF1A
:101B400008BD10B503685C6800231A46A04710BDA5
:101B5000C069704700238B420CDA10B4C45C944215
:101B600006D001338B42F9DB00205DF8044B70474F
:101B70000120FAE70020704782B0014802B07047A8
:101B80006C3201202DE9F0410C4616461F460878BC
:101B900091F8018040EA0820FFF7EEFF0546414634
:101BA0004BF03BFF2B681B68A178284698474FB144
:101BB0002B681B680021284698472B681B6800216A
:101BC0002846984728464BF09EFF14206CF0B5FC41
:101BD0003246617828464BF01BFF2B68DB682846AD
:101BE000984701280FDD2B681B692846984784B267
:101BF0002402A4B22B681B692846984740EA0407D0
:101C0000BFB200240EE02B68DB682846984728B155
:101C10002B681B692846984787B2F2E70027F0E750
:101C20000134E4B2731E9C420ADA2B68DB68284652
:101C300098470028F4D02B681B6928469847EFE79F
:101C40003846BDE8F081000000B583B00346064A7F
:101C500010680091054A064900F52A60FEF786FCE7
:101C600003B05DF804FB00BFBC7F0020FCCD0B007F
:101C700038C20B002DE9F04385B0ADF80C10039885
:101C8000FFF77AFF05464FF003090026B0460EE045
:101C900044462AE039462648FFF7D6FF4FF00209AE
:101CA0000136F6B2A04535D0032E33D8A0469DF8B4
:101CB0000D70394628464BF0B0FE2B681B6800219A
:101CC0002846984728464BF01EFF012239462846F1
:101CD0004BF09EFE2B68DB68284698470028D7D03B
:101CE0002B681B6928469847C4B204F00F04082CDF
:101CF000D0D0002CCED0E31EDBB2012B03D9062CB2
:101D000001D0072CCCD139460A48FFF79DFF4FF090
:101D10000109C5E7084B186800962346074A084999
:101D200000F52A60FEF722FC484605B0BDE8F083C6
:101D300018CE0B0020CE0B00BC7F002028CE0B005D
:101D4000C8BF0B00104661B130B401E0C96831B1C1
:101D50000D7C1C78A542F9D308468968F7E730BCAA
:101D60007047704770B50E46041D0B4622468168C9
:101D7000FFF7E8FF844203D03278037C9A4200D216
:101D8000204670BD10B582B004468DF807100DF1E5
:101D900007012030FFF7E6FF2434201A18BF012086
:101DA00002B010BD30B585B004468DF8071000F1C3
:101DB000380102A8FFF7A7FB2368DB689DF807102E
:101DC00020469847C0B91B4B1A889B78ADF80C2069
:101DD0008DF80E3002A8FFF79EFB00209DF80C3016
:101DE00063F307009DF80D3063F30F209DF80E306C
:101DF00063F3174005B030BD9DF8075004F1200093
:101E000024340DF1070322468168FFF79BFF8442CB
:101E10000DD09DF80720037C9A4208D3437C827C36
:101E200043EA0222294603A8FFF700FED2E7024850
:101E30007CF0B6FDBC8100204CCE0B00F0B585B027
:101E400005460E46174600F1380101A8FFF75BFB77
:101E50000024B4422DD2395D8DF803102B68DB6865
:101E60002846984708B90134F3E79DF8034005F187
:101E7000200024350DF103032A468168FFF762FF35
:101E8000854213D09DF80320037C9A420ED3437CF5
:101E9000827C43EA0222214603A8FFF7C7FD039B89
:101EA000ADF808301B0C8DF80A3009E00D487CF0C5
:101EB00077FD0D4B1A889B78ADF808208DF80A3015
:101EC00001A8FFF728FB00209DF8083063F3070006
:101ED0009DF8093063F30F209DF80A3063F3174033
:101EE00005B0F0BD4CCE0B00BC81002038B50446D7
:101EF0001D4649B10120231D29467CF0ECFC636995
:101F000001336361284638BD031D9A4205D02B7CFE
:101F1000117C994203D80020EDE70120EBE7012076
:101F2000E9E770B5044616461D4651B10120231D50
:101F3000324629467CF0CFFC636901336361284651
:101F400070BD031D9A4206D002F1100105F1100088
:101F5000FFF757FDEBE70120E9E7104661B130B428
:101F600001E0C96831B10D7C1C78A542F9D308465F
:101F70008968F7E730BC70477047F8B507461646E2
:101F80008C680D1D012202E0E36825461C4644B121
:101F90003378257C9D428CBF01220022F4D9A368AE
:101FA000F3E7284622B1CB68AB4209D07CF091FC24
:101FB000027C33789A4206D23C607D603846F8BD98
:101FC0003C607D60FAE7386000237B60F6E72DE92E
:101FD000F041074688461D460B1D9A4212D0144612
:101FE0002E78137CB3422CD9CB6893421DD0104677
:101FF0007CF06FFC037CB3421DD2C368C3B13C606C
:102000007C600FE04B6943B10B691A7C29789142DF
:1020100003D900220260436004E02A464146384664
:10202000FFF7ABFF3846BDE8F08103604360F9E796
:102030003B607860F6E72A4641463846FFF79DFF49
:10204000F0E7B3421AD20B6993420AD010467CF0F3
:102050002DFC037C9E420BD2E36833B1386078607C
:10206000E0E7002202604360DCE73B607C60D9E788
:102070002A4641463846FFF780FFD3E73A600023FF
:102080004360CFE7F0B583B005460E461F461420E7
:102090004AF092FC04463B681B78074607F8103F5D
:1020A0001130FFF7A6FC3B46324629466846FFF74B
:1020B0008EFF019A32B1234600992846FFF716FF9A
:1020C00003B0F0BD20464AF09BFC0098F8E770B5DD
:1020D0000C4616461D4600E0E4684CB1294604F162
:1020E0001000FFF78EFC0028F6D12646A468F4E71E
:1020F000304670BD2DE9F8430746884615468C6882
:102100000E1D012202E0E36826461C464CB104F194
:1021100010012846FFF775FC02460028F3D0A3689B
:10212000F2E7B1463AB1D8F80C30B3420ED030469F
:102130007CF0CFFB8146294609F11000FFF761FCD6
:1021400038B13C607E603846BDE8F8833C607E6014
:10215000F9E7C7F8009000237B60F4E72DE9F04130
:1021600007460C461E460B1D9A4219D0154602F131
:10217000100841463046FFF744FC98B3E368AB4291
:1021800023D028467CF0A5FB804631461030FFF76F
:1021900038FC08B3D8F80C30D3B13D607D6011E055
:1021A0004B6953B1086931461030FFF72AFC20B162
:1021B00000233B6023697B6004E0324621463846B9
:1021C000FFF798FF3846BDE8F0813B607B60F9E798
:1021D0003B60C7F80480F5E7324621463846FFF7F2
:1021E00089FFEFE731464046FFF70BFC00B3236958
:1021F000AB4210D028467CF059FB804600F110011C
:102200003046FFF7FEFB68B1EB6843B1C7F80080CA
:10221000C7F80480D6E700223A607B60D2E73B60D3
:102220007D60CFE7324621463846FFF763FFC9E7B6
:102230003D6000237B60C5E7F0B583B005460E46E0
:102240001F4614204AF0B8FB04463B681B880382F3
:102250000023837400F11003324629466846FFF7D5
:102260007DFF019A32B1234600992846FFF759FEB7
:1022700003B0F0BD20464AF0C3FB0098F8E7000029
:102280002DE9F047A8B006460C4617461D4600F15A
:10229000380109A8FFF737F9BC4B18682346BC4A38
:1022A000BC4900F52A60FEF761F90022214608A822
:1022B000FFF79CFB08238DF8213000F07CBD0899C6
:1022C0003046FFF7D7FC8DF81F0000F06ABDBDF85F
:1022D0002030ADF81830ADF8283004238DF82A30BE
:1022E000002301220AA93046FFF74CFC022809D03E
:1022F0009DF82110A848FFF7A7FC08238DF81F3090
:1023000000F04FBD9DF82110A448FFF79DFC0B2362
:102310008DF81F3000F045BDBDF82030ADF8183005
:10232000ADF82C3004238DF82E30002301220BA9A8
:102330003046FFF727FC48B19DF821109848FFF779
:1023400083FC46238DF81F3000F02BBD9DF8211033
:102350009448FFF779FC09238DF81F3000F021BD68
:102360009148FFF771FC0A238DF81F3000F019BD6A
:102370008E48FFF769FC04238DF81F3000F011BD73
:10238000BDF82030ADF81830ADF8303090238DF81E
:102390003230002301220CA93046FFF7F3FB48B985
:1023A0009DF821108248FFF74FFC42238DF81F3023
:1023B00000F0F7BC9DF821107E48FFF745FC0C2388
:1023C0008DF81F3000F0EDBCBDF82030ADF81830AE
:1023D000ADF83430D0238DF83630002301220DA91A
:1023E0003046FFF7CFFB602819D00CD808B355282A
:1023F0003BD19DF821107048FFF726FC10238DF883
:102400001F3000F0CEBC61282FD19DF821106B4801
:10241000FFF71AFC0D238DF81F3000F0C2BC9DF8A9
:1024200021106748FFF710FC0E238DF81F3000F0D5
:10243000B8BCBDF82030ADF81830ADF838300D23F9
:102440008DF83A30002301220EA93046FFF79AFB9F
:10245000102840F0A6849DF821105A48FFF7F4FB9D
:102460003F238DF81F3000F09CBCBDF82030ADF844
:102470001830ADF83C3000238DF83E3001220FA912
:102480003046FFF77FFB50280BD0602813D09DF813
:1024900021104D48FFF7D8FB0F238DF81F3000F0B7
:1024A00080BC9DF821104948FFF7CEFB11238DF821
:1024B0001F3000F076BC9DF821104548FFF7C4FBA3
:1024C00011238DF81F3000F06CBC4248FFF7BCFBB5
:1024D00030238DF81F3000F064BCBDF82030ADF81B
:1024E0001830ADF84030FE238DF842300023022230
:1024F00010A93046FFF746FB0446244B18682346D4
:10250000354A244900F52A60FEF730F845F2494380
:102510009C4209D09DF821103048FFF795FB13230A
:102520008DF81F3000F03DBCBDF82030ADF81830FC
:10253000ADF84430FF238DF846300023022211A964
:102540003046FFF71FFB0446104B18682346244A09
:10255000104900F52A60FEF709F842F260239C4218
:1025600009D09DF821101F48FFF76EFB12238DF84C
:102570001F3000F016BC9DF821101B48FFF764FBCC
:102580003C238DF81F3000F00CBC00BFBC7F002046
:1025900054CE0B00C8BF0B0094CE0B0088CE0B00AE
:1025A000A0CE0B00A8CE0B00B0CE0B00B8CE0B0017
:1025B000C0CE0B00C8CE0B00E8CE0B00D8CE0B006F
:1025C000E0CE0B00F8CE0B0010CF0B0000CF0B00BD
:1025D00008CF0B0018CF0B0020CF0B0060CF0B00F3
:1025E00038CF0B0058CF0B0050CF0B00BDF8203078
:1025F000ADF81830ADF84830FE238DF84A3000238E
:10260000022212A93046FFF7BDFA0446CB4B1868E8
:102610002346CB4ACB4900F52A60FDF7A7FF45F2D8
:1026200049439C4226D0BDF82030ADF81830ADF8B3
:102630004C3005238DF84E300123062213A9304675
:10264000FFF7A0FA0446BD4B18682346BE4ABD49B1
:1026500000F52A60FDF78AFF45F205339C4240F001
:10266000A0839DF82110B948FFF7EEFA32238DF8C8
:102670001F3096E39DF82110B548FFF7E5FA1423C3
:102680008DF81F308DE3BDF82030ADF81830ADF86F
:10269000503007238DF852300023022214A930460F
:1026A000FFF770FAB0F5806F1FD0BDF82030ADF89D
:1026B0001830ADF854300F238DF856300023022225
:1026C00015A93046FFF75EFAB0F54C5F04D043F22F
:1026D0003333984240F0658322238DF81F309DF8F4
:1026E00021109C48FFF7B0FA5BE316238DF81F30EA
:1026F0009DF821109848FFF7A7FA52E3BDF8203063
:10270000ADF81830ADF8583089238DF85A300023D1
:10271000022216A93046FFF735FA41F2A213984279
:102720000FD041F2DA1398420BD041F2F3139842E2
:1027300007D040F69C63984203D040F68D43984200
:1027400008D118238DF81F309DF821108348FFF71A
:102750007BFA26E3BDF82030ADF81830ADF85C30D8
:102760007E238DF85E300023022217A93046FFF742
:1027700009FA45F24943984208D017238DF81F30D3
:102780009DF821107648FFF75FFA0AE32D238DF8B4
:102790001F309DF821107348FFF756FA01E3724885
:1027A000FFF752FA19238DF81F30FAE2BDF82030F6
:1027B000ADF81830ADF86030FF238DF8623000239B
:1027C000012218A93046FFF7DDF9152808D0292382
:1027D0008DF81F309DF821106448FFF735FAE0E2CC
:1027E00038238DF81F309DF821106148FFF72CFA2F
:1027F000D7E26048FFF728FA1A238DF81F30D0E29D
:102800005D48FFF721FA1B238DF81F30C9E2BDF8A0
:102810002030ADF81830ADF864300A238DF86630FA
:102820000023012219A93046FFF7ACF9C0282CD0AB
:10283000BDF82030ADF81830ADF8683014238DF8AD
:102840006A30002301221AA93046FFF79BF900F0F5
:102850000303022B22D0BDF82030ADF81830ADF8BC
:102860006C300F238DF86E30002301221BA93046F7
:10287000FFF788F96A281AD01C238DF81F309DF8BD
:1028800021103E48FFF7E0F98BE224238DF81F303A
:102890009DF821103A48FFF7D7F982E245238DF8D9
:1028A0001F309DF821103748FFF7CEF979E2252334
:1028B0008DF81F309DF821103348FFF7C5F970E2FD
:1028C0003248FFF7C1F91D238DF81F3069E2304807
:1028D000FFF7BAF91E238DF81F3062E22D48FFF78B
:1028E000B3F91F238DF81F305BE2BDF82030ADF83F
:1028F0001830ADF870300F238DF8723000230222AB
:102900001CA93046FFF73EF9B0F54C5F03D043F207
:102910003333984208D122238DF81F309DF82110BF
:102920000C48FFF791F93CE223238DF81F309DF806
:1029300021101948FFF788F933E200BFBC7F00205F
:1029400068CF0B00C8BF0B008CCF0B00A8CF0B00CB
:1029500084CF0B00C0CF0B00B8CF0B00C8CF0B004B
:10296000D8CF0B00D0CF0B00E0CF0B00F4CF0B0083
:10297000E8CF0B0000D00B0008D00B0028D00B00D4
:1029800010D00B0018D00B0020D00B0030D00B0063
:102990003CD00B0048D00B0054D00B00BDF82030C9
:1029A000ADF81830ADF8743002238DF8763000237E
:1029B00001221DA93046FFF7E5F89DF821108BB2E2
:1029C000834206D026238DF81F30C648FFF73CF916
:1029D000E7E141238DF81F30C348FFF735F9E0E107
:1029E000C248FFF731F925238DF81F30D9E1C048DF
:1029F000FFF72AF927238DF81F30D2E1BD48FFF7F2
:102A000023F928238DF81F30CBE1BDF82030ADF835
:102A10001830ADF8783012238DF87A300023012277
:102A20001EA93046FFF7AEF8502808D04A238DF88B
:102A30001F309DF82110B048FFF706F9B1E12C23B3
:102A40008DF81F309DF82110AC48FFF7FDF8A8E184
:102A5000AB48FFF7F9F82E238DF81F30A1E1A94804
:102A6000FFF7F2F833238DF81F309AE1A648FFF7FD
:102A7000EBF815238DF81F3093E1A448FFF7E4F835
:102A80003E238DF81F308CE1A148FFF7DDF840238D
:102A90008DF81F3085E19F48FFF7D6F843238DF866
:102AA0001F307EE19C48FFF7CFF844238DF81F309C
:102AB00077E19A48FFF7C8F84E238DF81F3070E190
:102AC000BDF82030ADF81830ADF87C3086238DF895
:102AD0007E30002301221FA93046FFF753F89228C9
:102AE00017D08F4C9DF8211020464AF096FF23689E
:102AF0001B6801212046984720464BF004F888B90E
:102B00004C238DF81F309DF821108648FFF79CF864
:102B100047E147238DF81F309DF821108248FFF7C9
:102B200093F83EE1814B18689DF82130804A814935
:102B300000F52A60FDF71AFD33E17F48FFF784F8BE
:102B400048238DF81F302CE17C48FFF77DF83723B0
:102B50008DF81F3025E17A48FFF776F849238DF884
:102B60001F301EE1BDF82030ADF81830ADF88030D0
:102B70000E238DF882300023012220A93046FFF772
:102B800001F85A2818D0BDF82030ADF81830ADF84B
:102B9000843000238DF88630012221A93046FEF7CB
:102BA000F1FFE02811D03A238DF81F309DF8211055
:102BB0006448FFF749F8F4E02F238DF81F309DF8A3
:102BC00021106148FFF740F8EBE04B238DF81F30F0
:102BD0009DF821105D48FFF737F8E2E0BDF820309E
:102BE000ADF81830ADF8883000238DF88A30012216
:102BF00022A93046FEF7C6FFEA280AD09DF8211028
:102C000069290FD021238DF81F305148FFF71CF898
:102C1000C7E036238DF81F309DF821104D48FFF78F
:102C200013F8BEE031238DF81F304B48FFF70CF846
:102C3000B7E0BDF82030ADF81830ADF88C30002387
:102C40008DF88E30012223A93046FEF79BFF7D28A8
:102C500001D07A2808D13B238DF81F309DF8211030
:102C60003E48FEF7F1FF9CE0304B1C680090662365
:102C70003B4A3C4904F52A60FDF778FC91E0284C7A
:102C800020464AF0CAFE384B93E8030002908DF8C4
:102C90000C10D968986804908DF8141023685B684C
:102CA000052202A92046984720464AF02CFF05221B
:102CB00006A920466AF086FB0246052805D106A92A
:102CC00004A883F03DF9002852D0184B1868274A11
:102CD000184900F52A60FDF749FC34238DF81F30B0
:102CE0005FE000BF68D00B005CD00B0020D00B0071
:102CF00070D00B0078D00B0090D00B0084D00B006C
:102D000098D00B00A4D00B00ACD00B00B8D00B00B7
:102D1000CCD00B00D8D00B00E0D00B00E8D00B00DB
:102D20006C320120FCD00B00F0D00B00BC7F0020E7
:102D300004D10B0038C20B0040D10B004CD10B006A
:102D400054D10B0070D10B005CD10B0068D10B008B
:102D500090D10B007CD10B0088D10B0098D10B00D7
:102D6000B0D10B00C8BF0B0040D20B0004D20B0047
:102D7000BF4B1868BF4AC04900F52A60FDF7F6FB53
:102D80003D238DF81F300CE0B94B18680B46BB4A49
:102D9000B94900F52A60FDF7E9FB02E0042800F0DC
:102DA0000D819DF81F30002B40F013819DF82110FC
:102DB00001318DF821109DF82140772C00F25281CD
:102DC0007DB1224629463846FEF7C4FE0028EDD0E4
:102DD000A74B18682346AA4AAA4900F52A60FDF7BE
:102DE000C5FBA94C9DF8211020464AF016FE20464E
:102DF0004AF089FE00238DF81F300028CED19DF8BF
:102E00002110A1F10D026A2ABED801A353F822F0C5
:102E1000C1280300892D0300892D0300FD2903002B
:102E2000892D0300DD280300572B0300892D0300A3
:102E3000892D0300892D0300892D030087260300B7
:102E4000EB280300A52A0300892D030001280300B5
:102E50007B2A0300CF280300612303009D29030080
:102E60009D2903009D290300C12A0300892D030029
:102E7000892D0300EF290300892D03003B2B03005C
:102E80000B2A03005F2A0300892D0300892D03000C
:102E9000892D0300B32A0300892D0300892D030027
:102EA000892D0300892D0300892D03008123030050
:102EB000892D03006D2A0300972A0300CB24030009
:102EC000892D0300512A0300892D0300BF2203002E
:102ED000892D0300892D030071230300DB240300E7
:102EE000DB240300ED250300DB240300FD260300A3
:102EF000FD260300892D0300892D03007F2C03008C
:102F0000892D0300892D0300892D0300892D0300DD
:102F1000892D0300892D0300892D0300892D0300CD
:102F2000892D0300892D0300892A0300892D0300C0
:102F300019230300892D0300AD270300892D030009
:102F4000892D0300652B0300892D0300F32703005F
:102F5000F3270300892D0300CF220300892D0300EE
:102F6000892D0300492B0300892D0300892D0300BF
:102F7000892D0300332C0300892D0300DD2B030072
:102F8000DD2B0300E12903000F280300892D030036
:102F9000892D0300892D0300892D03009F2703003D
:102FA000892D0300892D0300892D0300892D03003D
:102FB000892D0300C9230300C92303002C4B186883
:102FC0009DF82130314A324900F52A60FDF7CEFAEA
:102FD000E7E606F1200806F124040DF11F0322465E
:102FE000D8F808104046FEF7B8FF03460146844271
:102FF00004D09DF81F40027C94420AD20DF11F03B9
:10300000279326AB009327AB224A4046FFF73AF8B6
:103010000346BDF82020A3F8112006F1080806F1A8
:103020000C0408AB2246D8F808104046FFF74FF8CA
:1030300081468246844205D000F1100108A8FEF7BF
:10304000E0FC50B108AB259324AB009325AB114AAB
:1030500051464046FFF7F0F881469DF81F3089F849
:103060001230A3E609A8FEF756FA28B0BDE8F087AB
:10307000BC7F0020E8D10B0038C20B0004D10B004C
:1030800074CE0B00C8BF0B006C32012020D20B00A5
:10309000FCBF0B0050D20B0030B4022400221346B8
:1030A0008D1EA54206D9055D2B44DBB21A44D2B26F
:1030B0000134F5E743550139425430BC704710B430
:1030C00043790479240404EB036384781C440023CB
:1030D000A1F10A02B3EB920F05D29A000632825890
:1030E00014440133F4E70B1FC454220ACB1EC2540C
:1030F000220C8B1EC254240E013944545DF8044B3B
:103100007047000084B004AB03E90700BDF8040079
:10311000029B064AA2FB03235B09054A02FB00301F
:103120009DF80C3003B1404204B070471F85EB514D
:103130008096980090F8E031013BDBB2042B01D976
:103140000020704701207047D0F8DC01003818BF1C
:103150000120704738B503460469826904EB6200B8
:1031600012F0010F02D15B69984738BD55106259C2
:103170005B69D358F8E738B503460469826904EB04
:10318000620012F0010F02D15B69984738BD5510FB
:1031900062595B69D358F8E710B50446064B1868C6
:1031A000064A074900F52A60FDF7E0F923689B69A4
:1031B00020469847002010BDBC7F002074D20B0031
:1031C00038C20B00000000002DE9F0478EB0044625
:1031D0000D460B6D23F07F42036D23F07F439A422F
:1031E0007DD001262EB1636F1BB16A6F934200F050
:1031F000B280012384F8203095F8507084F8507024
:1032000095F8513084F85130742205F1540104F1DD
:10321000540082F0A3FE002E00F0AF80002F00F0DB
:10322000A3806BF073F9C4F8C800A76DD4F8608070
:10323000D4F88C90D4F8A8A0666F594B1D6805F59A
:103240002A65D4F8B4300C93D4F8A00081F090FD36
:103250004DA3D3E9002381F005FECDE90A015046D4
:1032600081F086FD4AA3D3E9002381F0FBFDCDE97F
:103270000801484681F07CFD43A3D3E9002381F097
:10328000F1FDCDE90601A36E0493404681F080FD77
:1032900041A3D3E9002381F0E5FDCDE902013846E1
:1032A00081F076FD3CA3D3E9002381F0DBFDCDE97D
:1032B000000133463B4A3C492846FDF757F904F1E3
:1032C00028062546A36A1C469E4256D09868036885
:1032D0009B682946984700284FD12368F3E78A6DF9
:1032E000836D9A4201D001267CE70A6E036E9A42F2
:1032F00001D0012676E78A6E836E9A4201D00126BC
:1033000070E7D1F88020D0F880309A4201D00126B1
:1033100068E7D1F88C20D0F88C309A4201D0012691
:1033200060E7D1F8A820D0F8A8309A4201D0012651
:1033300058E7D1F8A020D0F8A0309A4201D0012659
:1033400050E7D1F8B420D0F8B4309A4201D0012629
:1033500048E7002646E7124B1868144A144900F55E
:103360002A60FDF703F944E70D4B1868114A0E492E
:1033700000F52A60FDF7FAF8A1E700200EB0BDE8DD
:10338000F08700BFAFF300807B14AE47E17A843F43
:10339000F168E388B5F8E43E48AFBC9AF2D77A3ECC
:1033A000BC7F0020BCD20B00C8BF0B0084D20B0036
:1033B000FCBF0B000CD30B0008B504280AD8DFE8CB
:1033C00000F00F110305070007480AE0074808E06E
:1033D000074806E0074B084A5721084849F042FBD6
:1033E000074808BD0748FCE71CD30B0028D30B0097
:1033F00018D30B004CC00B003CD30B0070D30B0058
:1034000034D30B00E8F30C002DE9F0479AB00446E2
:1034100015AD00F582760FCE0FC533682B6010AD69
:10342000F0340FCC0FC523682B609DF8543013F097
:10343000010F00F083809DF8403013F0010F01D19F
:1034400000207CE015A84CF0A3FF04469DF8543002
:1034500013F0010F38D19DF8543013F0010F36D11D
:103460004FF0FF30374BA3FB0030800981F080FC28
:103470000022354B81F040FB81F0A4FF0444079407
:1034800015A84CF06FFF089015A84CF05DFF09904F
:1034900010A84CF04BFF0A9010A84CF033FF0138F5
:1034A0000B9010A84CF01AFFA0F26C700C90002347
:1034B0000F930B9B002B3FDB07A9042005F0DCFFDB
:1034C000012809D000203AE06BF020F8C3E76BF048
:1034D0001DF8189BC01AC5E71C4B1C6804F52A642C
:1034E00010A84CF0FBFE054610A84CF00BFF06465A
:1034F0000A9FDDF82480DDF82090DDF81CA09DF8FF
:10350000543013F0010F12D14FF0FF300590CDF879
:1035100010A0CDF80C90CDF80880019700962B46AE
:103520000B4A0C492046FDF721F8012007E06AF01C
:10353000EDFF189BC01AE9E7002000E000201AB058
:10354000BDE8F087D34D62100000E03FBC7F002053
:1035500080D30B00C8BF0B002DE9F04192B00446A8
:1035600090F8CC3180F8E031D0F8D831D0F8E421AF
:103570009A4205D2042B40D8D4F8D831C4F8E431AB
:1035800023685B6A20469847054690B394F8B830A4
:1035900013F0020F05D194F8382112F0020F00F059
:1035A0006C8113F0010F33D1BB4B1D6805F52A6503
:1035B00094F8B83013F0010F40F039814FF0FF3626
:1035C00094F8043113F0010F40F037814FF0FF37CA
:1035D00094F8F03013F0010F40F035814FF0FF30D8
:1035E000019000973346AD4AAD492846FCF7BEFF2F
:1035F0000025284612B0BDE8F081A749086800936D
:103600009B1AA84AA64900F52A60FCF7AFFFB3E76A
:103610006AF07CFFD4F8EC30C01A41F2873398424C
:10362000C2D894F8043113F0010FBDD06AF06EFFD8
:10363000D4F81031C01A41F287339842B4D894F8C4
:10364000F03013F0010FAFD06AF060FFD4F8FC3017
:10365000C01A41F287339842A6D894F8B83003F0E4
:10366000FD0384F8B8300CAE04F1BC070FCF0FC6D1
:1036700097E8030086E803000CAB93E80700FFF728
:1036800041FD894B984200F3FA8012AB13E9070021
:10369000FFF738FD854B984200F3F380022384F84E
:1036A0004C3094F8803103F0FD0384F88031D4F875
:1036B0008461E666304681F05BFB73A3D3E90023A7
:1036C00081F0D0FB81F0A6FEA066002E00F0C18044
:1036D0000CAB93E80700FFF715FD606312AB13E92D
:1036E0000700FFF70FFDE06394F8903103F0FD034E
:1036F00084F89031D4F8940181F04AFB00226C4B9D
:1037000081F0DAFC81F05EFE8046606694F8383124
:1037100003F0FD0384F83831D4F83C0181F038FB24
:103720000022634B81F0C8FC06460F46404681F0FC
:103730002FFB32463B4681F0DFF981F043FEE06526
:103740003046394681F03EFE606494F8E031C4F8BA
:10375000883004F5827630464CF01AFE03903046ED
:103760004CF000FE049030464CF0EEFD059004F164
:10377000F00630464CF0DAFD069030464CF0C2FDC3
:103780000138079030464CF0A9FDA0F26C7008900B
:1037900000230B9303A805F0DFFD206594F8483162
:1037A00013F0020F07D003F0FD0384F84831D4F87A
:1037B0004C31C4F8903094F8283113F0020F17D030
:1037C00013F0010F14D003F0FD0384F82831D4F86E
:1037D0002C3148F69F42934246D8184681F0C8FAE9
:1037E0000022344B81F03EFB81F014FEC4F88400CB
:1037F00094F8183113F0020F3FF4FBAE13F0010FF1
:103800003FF4F7AE03F0FD0384F81831D4F81C013F
:1038100081F0AEFA1EA3D3E9002381F023FB00223E
:10382000234B81F049FC81F0F5FDE067E1E66AF0A9
:103830006DFED4F8EC30C61AC2E66AF067FED4F822
:103840001071C71BC4E66AF061FED4F8FC30C01AE0
:10385000C6E6114B18683346174A114900F52A602D
:10386000FCF784FE0025C4E60B4A1068134A0C4995
:1038700000F52A60FCF77AFEBAE70025B9E60025D4
:10388000B7E60025B5E600BF8FC2F5285C8FF63F8E
:103890006F1283C0CAA1FD3FBC7F0020E8D30B009C
:1038A00050C60B00B8D30B0000E9A43500D2496B19
:1038B0000000594000408F4018D40B0038D40B0052
:1038C00070B51D46049EB52380F82432622380F82B
:1038D000253280F8261280F8272280F8285200220C
:1038E00080F829222B46A91D014481F82422E91DD4
:1038F000014481F82422934206DD911DB45C014409
:1039000081F824420132F6E705F1080100F509705B
:10391000FFF7C2FB05F10800C0B270BD70B51D46CF
:10392000049EBA2380F82432CE2380F8253280F812
:103930002652002480F8274280F8281280F8292295
:103940002B46AA1D024482F82442EA1D024482F852
:10395000244205F10802024482F8244205F10902DA
:10396000024482F824422246934206DD911DB45C53
:10397000014481F824420132F6E705F10A0100F51D
:103980000970FFF79CFB05F10A00C0B270BD000092
:1039900070B5ADF5407D0E461446002500954FF4F8
:1039A0003F72294601A882F001FB6AF0AFFD044492
:1039B0006AF0ACFDA0421FD2114B18680368DB68A7
:1039C00098470028F4D00E4B186803681B69984785
:1039D000C0B20DF80500013540F2FF239D4201D031
:1039E0000D28E5D12A46314668461DF05DFA08B932
:1039F0000025DDE7032000E000200DF5407D70BDCF
:103A0000A46100202DE9F04385B0884691461F4609
:103A10006AF07CFD06460024009401940294ADF8FF
:103A20000C4013E09DF80030BA2B08D09DF801300F
:103A30008DF8003000238DF80130012406E09DF858
:103A40000130CE2BF2D12C460D2C1BD039463046FE
:103A50002AF049FE002837D01D4B18680368DB6840
:103A600098470028F0D01A4B186803681B699847DC
:103A7000651CEDB204AB1C4404F8100C022DD1D02F
:103A80002C46E1E79DF804309DF805209DF80610CE
:103A90009DF80700052B0BD0052B02D10AB9414533
:103AA0000ED00024009401940294ADF80C40CDE7B0
:103AB000012AF1D14145EFD14845EDD1032004E081
:103AC0004845EED1012000E0002005B0BDE8F083BC
:103AD000A46100202DE9F0438FB00F4690461D46AB
:103AE0008DF834108DF83520474B93E803000A9089
:103AF000ADF82C100023CDF82E306AF007FD0446F7
:103B000003AEDFF818C1BCE80F000FC69CE8070041
:103B100003C626F8022B120C32700222052A10DC92
:103B20000EAB134413F8103C9DF830100B44DBB27D
:103B30008DF830309DF831100B448DF83130013262
:103B4000ECE70022012A15DC911D0EAB134413F89B
:103B5000043C0EA8014401F8103C9DF830100B44C1
:103B6000DBB28DF830309DF831100B448DF83130D8
:103B70000132E7E74FF000094E46294620462AF079
:103B8000B2FD00283AD0092E3CD8204B18680368B3
:103B9000DB6898470028F0D01C4B186803681B6945
:103BA0009847C0B20EAB4B4413F82C3C83420BD069
:103BB0004FF000090EAB334413F8103C83420AD097
:103BC000032E0BD00026D8E709F10109B9F11A0F2D
:103BD000F0D1022013E00136F6B2CEE708B100269C
:103BE000CBE70B4B1868CDF800803B46094A0A49E1
:103BF00000F52A60FCF7BAFC012000E000200FB0BD
:103C0000BDE8F0830320FAE70CE30B00A461002079
:103C1000BC7F00205CD40B0050C60B0080D40B008E
:103C20002DE9F84F8A46914698469DF828B00B9D9D
:103C30006AF06CFC044600263746294620462AF0E6
:103C400052FD002843D0234B18680368DB6898476F
:103C50000028F2D01F4B186803681B699847052F8E
:103C6000EBD8DFE807F003080F161D21B528E4D1D3
:103C70000137BFB2E1E7622801D00027DDE7013755
:103C8000BFB2DAE7804501D00027D6E70137BFB2DF
:103C9000D3E7834501D00027CFE70137BFB2CCE798
:103CA00086B20137BFB2C8E746EA002086B24E4569
:103CB00001D30027C1E732465146064B186869F028
:103CC00081FB864201D00027B7E7304600E00020A4
:103CD000BDE8F88FA461002008B5D0F8A4000368FF
:103CE0001B68984708BD10B581F001040121002030
:103CF0006DF0F8FD214600206DF078FE10BD90F8C3
:103D0000003223B9012380F8003280F8FF31704778
:103D100010B5074B18680368DB689847441E30B13C
:103D2000034B186803681B6998472046F6E710BDE7
:103D3000A461002070B584B004460E4615460623E3
:103D4000029305210191042300930323022290F89A
:103D5000B4001DF02CF9002836D04EB1264B18685F
:103D600003681B68FF2198472046FFF7D1FF2BE02F
:103D70002DB194F8B430062B28D000230FE0002298
:103D800001212046FFF7D6FF4FF4FA706AF0D5FB09
:103D9000EFE7DA0025FA02F21849CA540133032B7F
:103DA000F7DD164B009308234122022114480068D6
:103DB000FFF786FD0246104B186803685B681049E0
:103DC000096801F50971984704B070BD002306E049
:103DD000DA0025FA02F2191D0A4842540133032B76
:103DE000F6DD084B009310234122022104480068AD
:103DF000FFF766FD0246DEE7A46100208C6100202B
:103E000020830020946100202DE9F04182B0044617
:103E10000D46174690F8038280F803124046FFF7DC
:103E2000CBFA06462846FFF7C7FA3B4BD3F800C04B
:103E300000903346394A3A490CF52A60FCF796FB64
:103E4000042D33D8DFE805F003031E354A00B8F12E
:103E5000010F2BD92046FFF75BFF324A4FF4006178
:103E6000314B1868FCF71CF901212046FFF734FF9D
:103E700000212046FFF737FF002201212046FFF7EF
:103E800059FF13E0274A4FF40061274B1868FCF7ED
:103E900021F901212046FFF71FFF01212046FFF7EE
:103EA00022FF3A4600212046FFF744FF02B0BDE85A
:103EB000F0811C4A4FF400611B4B1868FCF70AF9AB
:103EC00000212046FFF708FF01212046FFF70BFFE6
:103ED0003A4600212046FFF72DFFE7E7A7B9114A30
:103EE0004FF40061104B1868FCF7F4F800212046ED
:103EF000FFF7F2FE01212046FFF7F5FE00221146F2
:103F00002046FFF717FFD1E7084B094A4FF45871D5
:103F1000084848F0A7FD00BFBC7F00209CD40B00E0
:103F200038C20B00FC230C00147F0020C0D40B000F
:103F3000D0D40B0070D30B0010B50446044802F037
:103F400073FE002211462046FFF75EFF10BD00BF42
:103F50007861002038B504460025057503681B68A4
:103F60006FF0004198472A4604212046FFF74CFF96
:103F70006FF0004038BD00002DE9F04184B00546E7
:103F8000394C204602F0F4FE204602F011FF0746AD
:103F9000204602F055FE0446344BD86E1DF06CFEF0
:103FA0000646334BA3FB0423324A10689B09324A6E
:103FB000324900F52A60FCF7D9FA42F210739E42AA
:103FC00000D93CB9002201212846FFF71DFF04B0AB
:103FD000BDE8F0810623029305210191042300939B
:103FE0000323022295F8B4001CF0E1FFDFF8808083
:103FF000A8FB0730800980F0BBFE9FED171B41EC4A
:10400000100B7BF095FF51EC100B15A3D3E90023A7
:1040100080F028FF81F0FEF90746A8FB0023154A2F
:1040200010689B09164A154900F52A60FCF79EFAAC
:10403000BE4208D3224603212846FFF7E5FE0023AF
:1040400085F8E031C3E7224602212846FFF7DCFE6F
:10405000BDE700BFAFF3008085EB51B81E85F33F8D
:1040600000000000007CA54078610020B0B2002074
:10407000D34D6210BC7F002004D50B00C8BF0B00DD
:104080001CD50B00F8B5054690F80332EBB9284B68
:1040900018680368DB68984740F2FE33984211DDE8
:1040A000244B1C6804F52A64214B18680368DB68FC
:1040B00098470346204A21492046FCF757FA2846EC
:1040C000FFF726FE00273E4614E0FFF721FE0027FB
:1040D0003846F8BD00260DE03246194905F509704D
:1040E0001CF0E2FE0028F5D0D5F820330133C5F8E6
:1040F000203300260E4B18680368DB6898470028B9
:10410000E6DD0B4B186803681B6998470446C1B28B
:10411000AB1983F8241205F1B8004CF02BFC38439E
:10412000C7B2F02ED8D80D2CD6D00136E2E700BFAA
:10413000A4610020BC7F002054D50B0050C60B00AA
:1041400098D50B002DE9F84F0D4691461B02464AC3
:1041500082FB0312DF17C7EBA227B3F5961F05DB1F
:10416000B7F5006F03DD4FF4006700E080273846A5
:1041700048F034FC06467B1E0246002B04DB00217F
:1041800002F8011B013BF8E76AF0C0F904464FF062
:1041900000086AF0BBF9001BA8425CD2334B1868D8
:1041A0000368DB6898470028F3D0304B1868036831
:1041B0001B699847C0B27B1E984507DA08F10103D6
:1041C0009BB206F808000022F25498462C2822D010
:1041D000B8F1010F05D906EB080313F8023C0D2BCB
:1041E00013D0B8F1010FD4D906EB080313F8023C41
:1041F0000D2BCED106EB080313F8013C0A2BC8D1D6
:104200004FF0000886F80080C3E706EB080313F8B8
:10421000013C0A2BE5D1D9F80030D9F804B09A4610
:104220005B45DED0D968304683F005FA10B90AF153
:104230001C03F4E70E4B1868DAF800300D4A0E49FB
:1042400000F52A60FCF792F916B1304648F0DCFB25
:104250009AF8180004E02EB1304648F0D5FB08204B
:10426000BDE8F88F0820FBE7B5814E1BA461002054
:10427000BC7F0020C8D50B0038C20B002DE9F043ED
:10428000ADF5797D05460F46002138914FF43F7218
:1042900039A881F08BFE95F8E861062E00F22185A1
:1042A000DFE816F007005300DD008A0123027B02DD
:1042B0008703A84C206803685B6A984720680368F6
:1042C000DB69394698474FF4AB720021A24881F070
:1042D0006DFE64206AF031F9206803685B6826226D
:1042E0009E49984714206AF028F9206803685B68A3
:1042F0001D229B499847206803685B681D229949E5
:104300009847206803685B681D22974998471420E6
:104310006AF013F9206803685B6814229349984790
:10432000206803685B6814229149984720680368F5
:104330005B6814228F4998471423C5F8EC31012398
:1043400085F8E831082600F0DDBC8B4C214607A833
:1043500069F034FE21460AA869F030FE07248DF882
:104360003440864E31460EA869F028FE314611A829
:1043700069F024FE8DF85040814C214615A869F063
:104380001DFE214618A869F019FE0F238DF86C3028
:104390000023049305930693542048F00DFB064632
:1043A000049000F15403069307AC1CAB9C420ED062
:1043B0002146304669F068FE04F10C0106F10C005C
:1043C00069F062FE237E33761C341C36EDE70596D9
:1043D0001CAC07AB9C4208D01C3C04F10C0069F0FB
:1043E000A5FD204669F0A2FDF3E7664B1868664B11
:1043F0000093664B664A674900F52A60FCF7B6F8F9
:104400002846FFF785FC534B186803685B680A224F
:10441000614998473B4604AA4FF4FA712846FFF7D2
:1044200091FE0646082805D11423C5F8EC31022375
:1044300085F8E831049C059DA54208D004F10C00E4
:1044400069F074FD204669F071FD1C34F4E70498AE
:10445000002800F0578448F0D3FA00F053BC4F49CD
:1044600007A869F0ABFD4E490AA869F0A7FD002432
:104470008DF834404B490EA869F0A0FD4A4911A8B7
:1044800069F09CFD8DF85040049405940694382002
:1044900048F092FA0646049000F13803069307AC00
:1044A00015AB9C420ED02146304669F0EDFD04F17B
:1044B0000C0106F10C0069F0E7FD237E33761C3415
:1044C0001C36EDE7059615AC07AB9C4208D01C3CAA
:1044D00004F10C0069F02AFD204669F027FDF3E79E
:1044E000284B1868314B0093314B294A294900F574
:1044F0002A60FCF73BF82846FFF70AFC154B1868C2
:1045000003685B680E222B4998473B4604AA4FF488
:10451000FA712846FFF716FE0646082805D114232F
:10452000C5F8EC31032385F8E831049C059DA542CC
:1045300008D004F10C0069F0F9FC204669F0F6FCA3
:104540001C34F4E70498002800F0DC8348F058FAA3
:10455000D8E300BFA4610020C8810020D4D50B009F
:10456000FCD50B001CD60B003CD60B005CD60B0018
:1045700074D60B008CD60B00A4D60B00ACD60B0067
:10458000B4D60B00BC7F0020DCD60B00BCD60B00E1
:10459000C8D60B00C8BF0B00ECD60B00F8D60B003A
:1045A00004D70B0020D70B002CD70B0058D70B00DB
:1045B00048D70B0068D70B00B14C206803685B68D4
:1045C0001122B0499847206803685B681122AE4900
:1045D0009847206803685B680D22AC499847AC494E
:1045E00007A869F0EBFCAB490AA869F0E7FC0C23CB
:1045F0008DF83430A8490EA869F0E0FCA74911A84D
:1046000069F0DCFC0D248DF85040A54915A869F02F
:10461000D5FCA44918A869F0D1FC8DF86C400023A2
:10462000049305930693542048F0C6F90646049077
:1046300000F15403069307AC1CAB9C420ED02146FC
:10464000304669F021FD04F10C0106F10C0069F01F
:104650001BFD237E33761C341C36EDE705961CAC1F
:1046600007AB9C4208D01C3C04F10C0069F05EFCD6
:10467000204669F05BFCF3E78B4B18688B4B00938B
:104680008B4B8C4A8C4900F52A60FBF76FFF28465C
:10469000FFF73EFB7A4B186803685B680D22874979
:1046A00098473B4604AA4FF47A712846FFF74AFD23
:1046B0000646082805D11423C5F8EC31042385F8F3
:1046C000E831049C059DA54208D004F10C0069F076
:1046D0002DFC204669F02AFC1C34F4E704980028DD
:1046E00000F0108348F08CF90CE36F4B1868744BA2
:1046F0000093744B6F4A704900F52A60FBF736FF50
:104700002846FFF705FB5E4B186803685B680F22BD
:104710006D4998474FF4FA726C492846FFF738F90B
:10472000032824D0604B1868694B0093694B614A99
:10473000614900F52A60FBF719FF2846FFF7E8FA00
:104740004F4B186803685B680E22634998474FF423
:10475000FA7262492846FFF71BF9032812D0142386
:10476000C5F8EC31052385F8E8310826CAE24E4B3E
:104770001868534B5A4A5B4900F52A60FBF7F6FE6E
:104780000D26BFE2484B1868514B554A554900F574
:104790002A60FBF7EBFE0126B4E2394B1868036888
:1047A0005B68332250499847142069F0C6FE4F4990
:1047B00007A869F003FC4E490AA869F0FFFB092429
:1047C0008DF834404B490EA869F0F8FB4A4911A80E
:1047D00069F0F4FB0A238DF85030484915A869F0B8
:1047E000EDFB474918A869F0E9FB0B238DF86C3005
:1047F00044491CA869F0E2FB43491FA869F0DEFBAD
:104800008DF88840414923A869F0D8FB404926A883
:1048100069F0D4FB8DF8A4403E492AA869F0CEFB8C
:104820003D492DA869F0CAFB8DF8C0403B4931A82D
:1048300069F0C4FB3A4934A869F0C0FB8DF8DC404C
:104840000023049305930693C42048F0B5F8064668
:10485000049000F1C403069307AC38AB9C4261D0CE
:104860002146304669F010FC04F10C0106F10C0001
:1048700069F00AFC237E33761C341C36EDE700BF5A
:10488000A461002078D70B008CD70B00A0D70B00B9
:10489000B0D70B00B8D70B00C8D70B00D0D70B0090
:1048A000E0D70B00E8D70B00BC7F002010D80B002E
:1048B00004D80B00C8D60B00C8BF0B0020D80B00D3
:1048C00040D80B0030D80B0048D80B0058D80B004C
:1048D00078D80B0068D80B0080D80B0090D80B005C
:1048E000C8D50B0038C20B00A4D80B00E0D80B00D1
:1048F000D8D80B00E8D80B00F0D80B00F8D80B0084
:1049000000D90B0008D90B0010D90B0020D90B00DF
:1049100018D90B0024D90B002CD90B0034D90B006B
:1049200038D90B00059638AC07AB9C4208D01C3C2C
:1049300004F10C0069F0FAFA204669F0F7FAF3E79F
:10494000B74B1868B74B0093B74BB84AB84900F556
:104950002A60FBF70BFE2846FFF7DAF9B54B18681B
:1049600003685B680D22B44998473B4604AA4FF49C
:10497000FA712846FFF7E6FB0646082805D11423FE
:10498000C5F8EC31062385F8E831049C059DA54265
:1049900008D004F10C0069F0C9FA204669F0C6FAA3
:1049A0001C34F4E70498002800F0AC8148F028F8A3
:1049B000A8E104ACA14B93E8030084E803000821BC
:1049C0002046FEF769FB2846FFF7A2F9994B1868C5
:1049D00003685B6808222146984740F2EE230822CC
:1049E00006212846FFF776F800283CD002284CD054
:1049F0004FF440742246002138A881F0D7FA904B3A
:104A000093E8030007908DF820100023ADF82130C3
:104A10008DF82330082107A8FEF73EFB2846FFF754
:104A200077F9844B186803685B68082207A99847E0
:104A30004FF496630193042300930A23224638A976
:104A40002846FFF7EDF883B2002B00F04A810023DF
:104A50001A461D2B23DC38A98C5C7A49CC540132D0
:104A600092B20133F5E76E4B18683B46764A7749B8
:104A700000F52A60FBF77AFD4FF4FA63C5F8EC31D4
:104A8000002385F8E83108263CE1654B18683B4671
:104A90006F4A704900F52A60FBF768FDA8E700231C
:104AA000092B24DC38A98C5C664919448C770132C7
:104AB00092B20133F4E7634B93F828400DF1E00C18
:104AC0001CF802C0C4EB041403EB44030B4483F84A
:104AD00029C0013292B201311D29ECDD594991F80A
:104AE00028300133DBB281F82830092B06D802F1D7
:104AF0001D0381B28B4201DA0021EDE74C4CDFF857
:104B00002081D8F80000544A214600F52A60FBF7BE
:104B10002DFDDFF83091D8F800004B464F4A214672
:104B200000F52A60FBF722FDD8F8000009F11E030A
:104B30004B4A214600F52A60FBF718FDD8F8000023
:104B400099F82830474A214600F52A60FBF70EFD08
:104B500000243C4B93F82830A34210DDC4EB04132F
:104B60005B002833374A13442D4A106801333E4A0C
:104B70002F4900F52A60FBF7F9FC0134E9E74FF40F
:104B80004072002138A881F011FA4FF000080DE0C2
:104B9000C8EB08135B002C332A4A13444FF44072CD
:104BA000591C38A882F003FD08F10108254B93F841
:104BB0002830434572DDC8EB0814640004F1280373
:104BC000204C1C44013404222849204682F0DDFC9C
:104BD0000028DDD007222649204682F0D6FC002896
:104BE000E2D100230393C8EB08135B003033154A6E
:104BF00013444FF44072591C38A882F0D8FC084B7B
:104C0000186838AB1B4A0A4900F52A60FBF7AEFC6E
:104C10009DF8E03083BB0B4B002283F85521C3E79E
:104C2000BC7F00204CD90B0040D90B00C8D60B002C
:104C3000C8BF0B00A461002058D90B0018E30B007B
:104C400020E30B00C881002068D90B0050C60B0080
:104C500088D90B0038C20B00ACD90B00BCD90B00B3
:104C6000D0D90B00E4D90B00F4D90B00FCD90B0010
:104C700004DA0B000CDA0B000A2203A938A883F02F
:104C8000E9FCC3B2424A82F85531424A1068424AAE
:104C9000424900F52A60FBF769FC85E70822404994
:104CA000404882F072FC002831D008223E493D483D
:104CB00082F06BFC002837D008223C49394882F04A
:104CC00064FC00283DD008223949364882F05DFC5A
:104CD000002843D008223749324882F056FC002889
:104CE00049D02C4B18683B46334A344900F52A60BA
:104CF000FBF73CFC4FF4FA63C5F8EC31002385F870
:104D0000E831082630460DF5797DBDE8F083214B6A
:104D100018682B4B00932B4B2B4A2C4900F52A602B
:104D2000FBF724FC0226EDE71A4B1868284B00938A
:104D3000284B254A254900F52A60FBF717FC032676
:104D4000E0E7144B1868244B0093244B1E4A1F497C
:104D500000F52A60FBF70AFC0426D3E70D4B186820
:104D60001F4B00931F4B184A184900F52A60FBF7A8
:104D7000FDFB0526C6E7074B18681B4B00931B4B32
:104D8000114A124900F52A60FBF7F0FBBAE700BFB1
:104D9000C8810020BC7F002020DA0B00C8BF0B00B8
:104DA0002CDA0B00E681002048DA0B0064DA0B00F5
:104DB0007CDA0B0098DA0B0068D90B0050C60B00A8
:104DC00044DA0B0038DA0B00C8D50B0038C20B00F0
:104DD00060DA0B0054DA0B0054FA0B0070DA0B00A7
:104DE00094DA0B0088DA0B00D0C20B00A4DA0B00B7
:104DF000F0B585B0504B93F98870504B1C68002C6F
:104E000000F087804FF44A7047F0D6FD04464C4BC3
:104E100000224C49FCF7D2FC20464B4B40F8303B7B
:104E20007422002181F0C2F80025C4F8A45004F1D6
:104E3000A803C4F8AC30C4F8A830C4F8B0500823B4
:104E400084F8B43004F1B8004BF015F984F8E0515F
:104E5000C4F8E45184F8E8514FF4FA63C4F8EC3133
:104E6000C4F8F051C4F8F451C4F8F85184F8FC5176
:104E700084F8FD5184F8FE5184F8FF5184F8005203
:104E800084F8015284F80252042384F8033284F82F
:104E900004522E4B029303956B4604AA12E90300B9
:104EA00083E8030004F50372C4F81022C4F80C224E
:104EB000C4F81452264AC4F80822C4F8184204F56B
:104EC000077282E80300FA22294604F5097081F08E
:104ED0006DF8C4F8205384F824530123C4F8F43146
:104EE000C4F8F8310C2047F067FD06468560194B81
:104EF000036002230371C4F8A4006FB92046FFF7D2
:104F00001BF80E4B186820B10368DB694FF416518B
:104F10009847204605B0F0BD082047F04DFD0546F6
:104F20000D4B036047600C2047F046FD2A46314692
:104F3000F9F7F4FBE2E700BFB0B20020A461002063
:104F40000C800020A81F0C00D4E50B009931030051
:104F500000E30B00B0C10B00E0C10B0038B5044604
:104F6000094D284601F066FE0123237523681B685E
:104F7000322120469847284601F056FE002211466D
:104F80002046FEF741FF38BD7861002010B5044689
:104F9000154B93F88C30012B01D09BB110BD124BF7
:104FA000002283F88C20114B1868114A114900F532
:104FB0002A60FBF7DBFAFCF7ABF923689B69204614
:104FC0009847EBE7084B012283F88C20074B1868C1
:104FD000094A084900F52A60FBF7C8FAFCF786F988
:104FE0002046FFF7BBFFD9E7B0B20020BC7F00200E
:104FF000B0DA0B0038C20B00D4DA0B000320704784
:1050000070B505460C46061D0C2047F0D5FC8460A3
:10501000314679F0FEFBEB680133EB600C2047F082
:10502000CBFC8560214679F0F4FBA3680133A360D3
:1050300070BD00002DE9F04385B00446AE4B1D78ED
:10504000002D40F0E280D0F8F8311BB190F8B43078
:10505000082B67D094F8B430082B00F0DC80204691
:10506000FEF74DFE94F8B400012800F0AF80092847
:1050700000F0D5800A2800F002810B2800F01D8185
:10508000002800F07181072800F0EA810D230C222E
:1050900002211BF08CFF002800F03682974B93F81A
:1050A000B8310A2B02D0192B40F00A82944B1868B1
:1050B00003685B68192293499847914D28680368F3
:1050C0005B68112290499847286803685B68112241
:1050D0008E499847286803685B6811228C49984775
:1050E000286803685B6811228A4998472868036822
:1050F0005B68112288499847286803685B68112219
:1051000086499847286803685B6811228449984754
:10511000FA2069F012FA286803685B680D22814959
:1051200098476FE090F8FD31012B2CD994F8FD31B0
:10513000022B8FD194F8FC217B4B53F82210204690
:10514000FFF79CF884F8B400082883D194F8E8317C
:10515000002B7FF47FAF94F8FC610136F6B284F83F
:10516000FC617148FFF74AFF86427FF473AF6F4BD3
:1051700018684FF416536E4A6E4900F52A60FBF723
:10518000F5F9012547E090F8FC216B4B53F822100C
:10519000FFF774F884F8B4000828C7D194F8E83110
:1051A000002BC3D194F8FC610136F6B284F8FC619F
:1051B0006148FFF723FF8642B8D1002384F8FC3111
:1051C00094F8FD31013384F8FD31AFE74C4D286888
:1051D00003685B680E2259499847FA2069F0ADF9D7
:1051E000286803685B68262255499847FA2069F0C9
:1051F000A4F9286803685B680E2252499847FA2090
:1052000069F09BF93C4B01221A704F4904F502707A
:10521000FFF7F6FE0125284605B0BDE8F083384DBE
:10522000286803685B681722484998474FF47A70EA
:1052300069F083F9286803685B683322444998471A
:10524000FA2069F07AF9286803685B680F224149FF
:105250009847FA2069F071F9286803685B6813229F
:105260003D499847FA2069F068F9286803685B6847
:105270000F223A499847FA2069F05FF9C2E7204DBA
:10528000286803685B681722354998474FF47A709D
:1052900069F053F9286803685B6833222C49984702
:1052A000FA2069F04AF9286803685B680F222949E7
:1052B0009847FA2069F041F9A4E7114D286803687E
:1052C0005B681722274998474FF47A7069F035F9DF
:1052D000286803685B6833221D499847FA2069F003
:1052E0002CF9286803685B680F221A499847FA204E
:1052F00069F023F986E700BF1E830020B0B20020CA
:10530000A4610020DCDC0B0014DD0B0028DD0B00A9
:1053100078D70B008CD70B003CDD0B0050DD0B0069
:1053200064DD0B00A0D70B007CE40B00BC7F0020E9
:10533000F8DA0B0050C60B0070E30B001CDB0B000F
:105340002CDB0B0054DB0B00C430012064DB0B00B2
:105350007CDB0B00B0DB0B00C0DB0B00D4DB0B00F5
:10536000E4DB0B00FCDB0B00594B00932C230722E2
:1053700006212046FEF7D2FA0246564B186801680D
:105380004D6804F509773946A847FA230722062114
:105390002046FEF737FB03281BD14F4B0093042315
:1053A0001A4606212046FEF7B9FA0246494B18680C
:1053B00001684D683946A847FA2304220621204691
:1053C000FEF720FB03280DD10423ADF8083000259B
:1053D0001BE0424B1868424A424900F52A60FBF73D
:1053E000C5F8DAE73D4B18683F4A3E4900F52A60A8
:1053F000FBF7BCF8E8E7394B186843463B4A3949A4
:1054000000F52A60FBF7B2F80135012D3FF6FAAE40
:1054100000238DF80F304E238DF80C3001268DF8C7
:105420000E6004AB2B4413F8088C8DF80D8003AB91
:1054300000930423324606212046FEF76FFA024607
:10544000244B18680168D1F804903946C847FA23FC
:10545000324606212046FEF7D5FA0328D4D0CAE703
:105460001C4D286803685B6810222149984740F268
:10547000EE2069F062F8286803685B680F221D4916
:105480009847FA2069F059F8286803685B680F228A
:1054900019499847FA2069F050F8286803685B6852
:1054A0000F2216499847FA2069F047F828680368E0
:1054B0005B680F2212499847FA2069F03EF8A1E68E
:1054C000044B186803685B6819220E499847F4E595
:1054D00010E50B00A461002000E50B00BC7F00205C
:1054E00014DC0B0050C60B0034DC0B0060DC0B003E
:1054F00088DC0B009CDC0B00ACDC0B00BCDC0B0084
:10550000CCDC0B00F8DC0B0094F8B400022800F0AF
:10551000CC81052300930423032211461BF047FD91
:10552000002800F0848594F8B430032B00F0E48365
:10553000C84B00932C233E2206212046FEF7C0F9DB
:105540000246C54B186801684D6804F50971A84703
:105550004FF448733E2206212046FEF7BBFA01288D
:1055600000F0E38394F8B430032B00F0E783BB4BE7
:105570001868BB4ABB4900F52A60FAF7F7FF4FF4F9
:105580007A7068F0DAFF2046FEF7C2FBB64B009354
:105590000A23022206212046FEF792F90246AE4B6C
:1055A000186801684E6804F509752946B0474FF43C
:1055B000FA73022206212046FEF78CFA032840F0F7
:1055C000C68394F8B430042B00F0CB83A74B009330
:1055D0000823392206212046FEF772F902469E4B27
:1055E000186801684E682946B0474FF4FA733922AB
:1055F00006212046FEF76EFA032840F0FD839C4BFF
:1056000000932823232206212046FEF759F902465B
:10561000914B186801684E682946B0474FF4FA73F9
:10562000232206212046FEF755FA032840F0EF8397
:10563000904B00930623082219462046FEF740F9B6
:105640000246854B186801684E682946B0474FF4FA
:10565000FA73082206212046FEF73CFA032840F0A0
:10566000E083854B00930823012206212046FEF7A4
:1056700027F90246784B186801684E682946B047FA
:105680004FF4FA73012206212046FEF723FA03287D
:1056900040F0D183794B0093082301220621204654
:1056A000FEF70EF902466C4B186801684E682946F1
:1056B000B0474FF4FA73012206212046FEF70AFA9A
:1056C000032840F0C2836E4B009308230122062179
:1056D0002046FEF7F5F802465F4B186801684E68F1
:1056E0002946B0474FF4FA73012206212046FEF7FF
:1056F000F1F9032840F0B383624B009308230122A1
:1057000006212046FEF7DCF80246534B1868016874
:105710004E682946B0474FF4FA730122062120460D
:10572000FEF7D8F9032840F0A483574B00930823D1
:10573000012206212046FEF7C3F80246464B1868B0
:1057400001684E682946B0474FF4FA7301220621DA
:105750002046FEF7BFF9032840F095834B4B00939A
:105760000823012206212046FEF7AAF802463A4BFA
:10577000186801684E682946B0474FF4FA73012251
:1057800006212046FEF7A6F9032840F0BD83404BD2
:1057900093F85531112B40F2FB832046FEF7B8FAFF
:1057A0003C4B00930823862206212046FEF788F80A
:1057B0000246294B186801684E682946B0474FF4E5
:1057C000FA73862206212046FEF784F9032840F06A
:1057D000A583314B00932C233B2206212046FEF764
:1057E0006FF802461C4B186801684E682946B0479E
:1057F0004FF4FA733B2206212046FEF76BF903288B
:1058000040F0968394F8B430042B00F09B83234B34
:1058100000930D23092206212046FEF751F8024687
:105820000D4B186801684E682946B0474FF4FA637B
:10583000092206212046FEF74DF9032800F0ED83EA
:10584000064B1868164A174900F52A60FAF78EFECB
:105850002AE000BFE4E30B00A4610020BC7F00202D
:1058600080DF0B0038C20B0004E50B003CE40B00AA
:10587000A8E30B0028E30B0040E30B0048E30B0018
:1058800050E30B0068E30B0060E30B0038E30B0010
:10589000C881002058E30B0010E40B0090E30B00DC
:1058A000D8DE0B0050C60B00ACE42046FEF730FA01
:1058B000C04B00930A23022206212046FEF700F87F
:1058C0000246BD4B186801684E6804F50975294603
:1058D000B0474FF4FA73022206212046FEF7FAF889
:1058E000032840F05281B54B00930823392206214A
:1058F0002046FDF7E5FF0246AF4B186801684E6889
:105900002946B0474FF4FA73392206212046FEF7A4
:10591000E1F8032840F04381A94B00932823232278
:1059200006212046FDF7CCFF0246A34B186801680C
:105930004E682946B0474FF4FA73232206212046C9
:10594000FEF7C8F8032840F05F819E4B00930623C2
:10595000082219462046FDF7B3FF0246964B186809
:1059600001684E682946B0474FF4FA7308220621B1
:105970002046FEF7AFF8032840F05081924B009389
:105980000823012206212046FDF79AFF02468A4B92
:10599000186801684E682946B0474FF4FA7301222F
:1059A00006212046FEF796F8032840F04181874BF8
:1059B00000930823012206212046FDF781FF0246BD
:1059C0007D4B186801684E682946B0474FF4FA735A
:1059D000012206212046FEF77DF8032840F032819F
:1059E0007B4B00930823012206212046FDF768FF28
:1059F0000246714B186801684E682946B0474FF45B
:105A0000FA73012206212046FEF764F8032840F0CD
:105A10002381704B00930823012206212046FDF7C5
:105A20004FFF0246644B186801684E682946B0472C
:105A30004FF4FA73012206212046FEF74BF80328A3
:105A400040F01481644B0093082301220621204674
:105A5000FDF736FF0246584B186801684E68294624
:105A6000B0474FF4FA73012206212046FEF732F8C0
:105A7000032840F00581594B009308230122062199
:105A80002046FDF71DFF02464B4B186801684E6823
:105A90002946B0474FF4FA73012206212046FEF74B
:105AA00019F8032840F0F6802046FEF731F94C4BF8
:105AB00000930223112206212046FDF701FF024632
:105AC0003D4B186801684E682946B0474FF4FA7399
:105AD000112206212046FDF7FDFF032840F0E48057
:105AE000404B00932C233B2206212046FDF7E8FE85
:105AF0000246314B186801684E682946B0474FF49A
:105B0000FA733B2206212046FDF7E4FF032840F00C
:105B1000D580354B00930823012206212046FDF74E
:105B2000CFFE0246244B186801684E682946B047EC
:105B30004FF4FA73012206212046FDF7CBFF03281C
:105B400040F0C680294B00930D23092206212046F0
:105B5000FDF7B6FE0246184B186801684E682946E4
:105B6000B0474FF4FA63092206212046FDF7B2FF41
:105B7000032800F0B7801E4B18681E4A1E4900F526
:105B80002A60FAF7F3FCFFF73DBB194B18681B4B73
:105B90001B4A194900F52A60FAF7E8FCA3E6144B02
:105BA0001868184B164A144900F52A60FAF7DEFC0B
:105BB000B2E600BF04E50B00A46100203CE40B004A
:105BC000A8E30B0028E30B0040E30B0048E30B00C5
:105BD00050E30B0068E30B0060E30B0038E30B00BD
:105BE00088E40B0010E40B0030E30B0090E30B00A3
:105BF000BC7F0020D8DE0B0050C60B0078DD0B0008
:105C000098DD0B00A8DD0B00A44B1868A44BA54A37
:105C1000A54900F52A60FAF7A9FC96E69F4B18689B
:105C2000A24BA04AA04900F52A60FAF79FFCA5E61E
:105C30009A4B18689E4B9B4A9B4900F52A60FAF7DD
:105C400095FCB4E6954B18689A4B964A964900F530
:105C50002A60FAF78BFCC3E6904B1868964B914A82
:105C6000914900F52A60FAF781FCD2E68B4B18685F
:105C7000924B8C4A8C4900F52A60FAF777FCE1E6F2
:105C8000864B18688E4B874A874900F52A60FAF7D9
:105C90006DFCF0E6814B18688A4B824A824900F518
:105CA0002A60FAF763FCFFE67C4B1868864B7D4A56
:105CB0007D4900F52A60FAF759FC11E7774B18681F
:105CC000824B784A784900F52A60FAF74FFC20E7C2
:105CD000724B18687E4B734A734900F52A60FAF7D5
:105CE00045FC2FE76D4B18687A4A7B4900F52A601E
:105CF000FAF73CFCFFF786BA684B1868774A784990
:105D000000F52A60FAF732FC764B009314233E220A
:105D100006212046FDF7D4FD0246734B1868016842
:105D20004D6804F50971A84712E45C4B18686F4A86
:105D30006B4900F52A60FAF719FC24E4574B186800
:105D40006B4A654900F52A60FAF710FC17E4534BDB
:105D50001868684B534A544900F52A60FAF706FC64
:105D60002FE42046FDF7D4FF634B0093082339222C
:105D700006212046FDF7A4FD02465B4B186801682A
:105D80004E682946B0474FF4FA733922062120465F
:105D9000FDF7A0FE032825D12046FDF7B9FF574B9C
:105DA00000932823232206212046FDF789FD024681
:105DB0004D4B186801684E682946B0474FF4FA7396
:105DC000232206212046FDF785FE03283FF430AC50
:105DD000324B18684A4B334A334900F52A60FAF7C8
:105DE000C5FB25E42D4B1868464B2E4A2E4900F57D
:105DF0002A60FAF7BBFBCFE7284B1868414B294ACA
:105E0000294900F52A60FAF7B1FBFFF7F8BB234BED
:105E10001868234B234A244900F52A60FAF7A6FBA9
:105E200006E41E4B1868214B1E4A1F4900F52A60E4
:105E3000FAF79CFB15E4194B18681D4B194A1A49CF
:105E400000F52A60FAF792FB24E4144B1868194B0A
:105E5000144A154900F52A60FAF788FB33E40F4B22
:105E60001868154B0F4A104900F52A60FAF77EFBB7
:105E700042E40A4B1868114B0A4A0B4900F52A60A4
:105E8000FAF774FB51E4054B18680D4B054A0649B7
:105E900000F52A60FAF76AFB60E400BFBC7F0020CF
:105EA000CCDD0B0098DD0B0050C60B00E8DD0B00CD
:105EB00000DE0B0014DE0B0028DE0B003CDE0B00C6
:105EC00050DE0B0064DE0B0078DE0B00A0DE0B0062
:105ED000C4DE0B00FCDE0B0038C20B0018DF0B0029
:105EE000C8BF0B00D0E30B00A461002028DF0B002B
:105EF0006CDF0B0078DD0B00A0E30B0044E40B002B
:105F0000A4DF0B00A8DD0B00574B1868574B584A0D
:105F1000584900F52A60FAF729FB38E4524B186813
:105F2000554B534A534900F52A60FAF71FFB50E4DA
:105F30004D4B1868514B4E4A4E4900F52A60FAF70E
:105F400015FB5FE42046FDF7E3FE4D4B0093142361
:105F5000172206212046FDF7B3FC0246494B18687C
:105F600001684E682946B0474FF4FA73172206219C
:105F70002046FDF7AFFD03283FF449AC3A4B1868C3
:105F8000414B3B4A3B4900F52A60FAF7EFFA3EE401
:105F90003E4B00930223112206212046FDF790FC80
:105FA0000246384B186801684E682946B0474FF4DE
:105FB000FA73112206212046FDF78CFD032822D119
:105FC000334B00932C233B2206212046FDF778FC1F
:105FD00002462C4B186801684E682946B0474FF4BA
:105FE000FA733B2206212046FDF774FD03283FF497
:105FF0000EAC1D4B1868214B1D4A1E4900F52A6046
:10600000FAF7B4FA03E4184B1868224B184A1949F6
:1060100000F52A60FAF7AAFAD2E7134B18681E4A6D
:106020001E4900F52A60FAF7A1FAFFF7EBB894F8D9
:10603000B430062B38D00F2B7FF4E4A8114D28681C
:1060400003685B68142216499847FA2068F075FACD
:10605000286803685B68142212499847FA2068F0A0
:106060006CFAFFF7CFB800BFBC7F002064DE0B00E6
:1060700098DD0B0050C60B00C4DF0B00A0DE0B0048
:106080007CE30B00A4610020E0DF0B008CE40B003C
:1060900010E40B00F4DF0B0014E00B0038C20B001F
:1060A000E0E10B00F8E10B004FF47A7068F045FA7C
:1060B0002046FDF72DFECA4B009322238A2206219B
:1060C0002046FDF7FDFB0246C64B186801684E6886
:1060D00004F509752946B0474FF496738A220621C4
:1060E0002046FDF7F7FC032840F06F8140F2EE20D8
:1060F00068F023FA2046FDF70BFEBB4B00931323F9
:106100008A2206212046FDF7DBFB0246B54B1868C4
:1061100001684E682946B0474FF496738A220621DB
:106120002046FDF7D7FC032840F0808140F2EE20A6
:1061300068F003FA2046FDF7EBFDAC4B0093092312
:106140008A2206212046FDF7BBFB0246A54B1868B4
:1061500001684E682946B0474FF496738A2206219B
:106160002046FDF7B7FC032840F06A8140F2EE209C
:1061700068F0E3F92046FDF7CBFD9D4B0093092322
:106180008A2206212046FDF79BFB0246954B1868A4
:1061900001684E682946B0474FF496738A2206215B
:1061A0002046FDF797FC032840F0548140F2EE2092
:1061B00068F0C3F98F4B009326238A2206212046DC
:1061C000FDF77EFB0246874B186801684E6829463A
:1061D000B0474FF496738A2206212046FDF77AFCD9
:1061E000032840F0418140F2EE2068F0A6F9824B8E
:1061F000009326238A2206212046FDF761FB0246F2
:10620000784B186801684E682946B0474FF496737A
:106210008A2206212046FDF75DFC032840F02E81EE
:1062200040F2EE2068F089F9744B00930E238A2225
:1062300006212046FDF744FB02466A4B18680168B8
:106240004E682946B0474FF496738A2206212046AD
:10625000FDF740FC032840F01B8140F2EE2068F07F
:106260006CF9674B00930E238A2206212046FDF726
:1062700027FB02465B4B186801684E682946B04709
:106280004FF496738A2206212046FDF723FC03284B
:1062900040F0088140F2EE2068F04FF9594B00932E
:1062A0000E238A2206212046FDF70AFB02464D4BAB
:1062B000186801684E682946B0474FF496738A22E1
:1062C00006212046FDF706FC032840F0F58040F249
:1062D000EE2068F032F94C4B00930E238A220621FF
:1062E0002046FDF7EDFA02463E4B186801684E68FD
:1062F0002946B0474FF496738A2206212046FDF7BF
:10630000E9FB032840F0E28040F2EE2068F015F946
:106310003E4B00930E238A2206212046FDF7D0FA39
:106320000246304B186801684E682946B0474FF462
:1063300096738A2206212046FDF7CCFB032840F005
:10634000CF8040F2EE2068F0F8F8314B00930E2336
:106350008A2206212046FDF7B3FA0246214B18682F
:1063600001684E682946B0474FF4FA738A22062125
:106370002046FDF7AFFB032840F0BC8040F2EE2042
:1063800068F0DBF8234B00930D23092206212046F9
:10639000FDF796FA0246134B186801684E682946C5
:1063A000B0474FF4FA63092206212046FDF792FB1D
:1063B000032800F0A980184B1868184A184900F5FE
:1063C0002A60FAF7D3F8FEF71DBF134B1868154B78
:1063D000154A134900F52A60FAF7C8F886E600BFA7
:1063E00070E50B00A46100205CE50B00C0E50B002C
:1063F000B4E50B00B8E40B0090E40B00F0E40B00F4
:10640000E0E40B00A4E50B0094E50B003CE50B0079
:106410004CE50B006CE40B00BC7F0020D8DE0B00C9
:1064200050C60B0038E00B0098DD0B003B4B1868A2
:106430003B4B3C4A3C4900F52A60FAF797F875E671
:10644000364B1868394B374A374900F52A60FAF756
:106450008DF88BE6314B1868354B324A324900F5DE
:106460002A60FAF783F8A1E62C4B1868314B2D4AC5
:106470002D4900F52A60FAF779F8B4E6274B186839
:106480002D4B284A284900F52A60FAF76FF8C7E62D
:10649000224B1868294B234A234900F52A60FAF752
:1064A00065F8DAE61D4B1868254B1E4A1E4900F5B3
:1064B0002A60FAF75BF8EDE6184B1868214B194A89
:1064C000194900F52A60FAF751F800E7134B1868EC
:1064D0001D4B144A144900F52A60FAF747F813E7F0
:1064E0000E4B1868194B0F4A0F4900F52A60FAF74E
:1064F0003DF826E7094B1868154B0A4A0A4900F58A
:106500002A60FAF733F839E7044B1868114A124940
:1065100000F52A60FAF72AF8FEF774BEBC7F002067
:106520005CE00B0098DD0B0050C60B0080E00B0018
:10653000A8E00B00D0E00B00F4E00B0018E10B002A
:106540003CE10B0060E10B007CE10B0098E10B00EB
:10655000BCE10B0014E00B0038C20B0038B5054657
:106560000068854204D0046846F04AFA2046F8E7FD
:1065700038BD38B505460068854204D0046846F049
:106580003FFA2046F8E738BD38B505460068854231
:1065900004D0046846F034FA2046F8E738BD2DE907
:1065A000F84307460E4603688046814609E0BB680B
:1065B000013BBB60284678F033F9284646F020FAC4
:1065C00023461D4698450AD01C6899683268914256
:1065D000F6D103F108029642E9D19946F0E74F451A
:1065E00008D0BB68013BBB60484678F019F94846C3
:1065F00046F006FABDE8F8832DE9F84307460E4653
:1066000003688046814609E0BB68013BBB602846C1
:1066100078F006F9284646F0F3F923461D469845DA
:106620000AD01C68996832689142F6D103F10802D9
:106630009642E9D19946F0E74F4508D0BB68013B47
:10664000BB60484678F0ECF8484646F0D9F9BDE81A
:10665000F883000030B583B005460D4B03604468F5
:106660002B1D9C4206D0019501A9A068FFF7C4FF2D
:106670002468F5E72C1D2046FFF770FFAC606C60C6
:106680000023EB602046FFF769FF284603B030BDCA
:10669000B4E20B0010B50446FFF7DCFF204646F0DD
:1066A000AFF9204610BD000010B50446024B036050
:1066B000FFF7D0FF204610BDC8E20B0010B504461E
:1066C0000A4B03600A4B40F8343FFFF7C3FF2046F4
:1066D000084B40F8283BF8F7A7FC2046064B40F84B
:1066E000043FF8F711FD204610BD00BFDCE20B00AF
:1066F000C8E20B0038C30B0024C30B0010B50446DE
:10670000044B0360FFF7A6FF204646F079F92046C8
:1067100010BD00BFC8E20B0010B504460B4B036070
:106720000B4B40F8343FFFF795FF2046094B40F8EC
:10673000283BF8F779FC2046074B40F8043FF8F770
:10674000E3FC204646F05CF9204610BDDCE20B007D
:10675000C8E20B0038C30B0024C30B0090F8FF31D4
:10676000002B00F09B802DE9F047BEB004460025C9
:1067700080F8FF514A4B1E6806F52A66076D90F8AF
:10678000FE81D0F8909003685B6A98470290CDF83C
:106790000490CDF800803B46424A43493046F9F721
:1067A000E5FE94F8FEA194F80092404B93F88C60BB
:1067B000013E18BF012604F130083D4B3A933B954A
:1067C00005AB29463A4883E8030007AA09A90A91BC
:1067D00009910B95374908910C920DAF93E803008E
:1067E00087E803008DF83C50109511A91291119182
:1067F00013953149079131493C913D953EA911E9E5
:10680000030083E8030015A91691159117952C49EB
:106810001491189219AA93E8030082E803007427E0
:106820003A4629461CA87FF0C1FB39958DF86CA02B
:106830008DF86D908DF86E603A4641461CA87FF049
:106840008DFB04F1A805D4F8A8301C469D4207D062
:10685000986803689B6807A9984708B92368F4E714
:10686000124B93F88C30012B13D0134B0793144B1E
:10687000149314A8FFF7EEFE124B079311A8F8F734
:10688000D3FB0C4B089308A8F8F73EFC3EB0BDE8DC
:10689000F0870D4B186836F00FF8E6E7704700BF39
:1068A000BC7F002010E20B00C8BF0B00B0B200207C
:1068B00057E8020024C30B00DCE20B00C9310300DF
:1068C000C8E20B0038C30B00282201202DE9F0415B
:1068D000044690F8013263BB774B1B6893B1774B4A
:1068E00093F88C30022B0DD003681B6A9847B8B11F
:1068F000724B93F88C30012B15D023689B6920468E
:1069000098470BE06E4B18686E4A6F4900F52A6095
:10691000F9F72CFE23689B6920469847BDE8F08173
:10692000D4F8EC01FAE7012384F801322046FFF79E
:1069300015FF2368DB6A20469847D8B95F4B93F868
:10694000693013B994F80332C3B994F8E06194F84C
:106950000332E3B1594B93F86930002B00F0A48067
:1069600094F8FE31002B00F09F8023689B6920463D
:106970009847D3E72046FDF7C2F9DFE7534800F018
:1069800088F90028E1D02046FDF7D6FADDE74B4B29
:10699000D86E1BF071F9054602F052FB03288CBF3C
:1069A0000127002705D823681B6B2046984700B1B4
:1069B000074623685B6B20469847804640B142F209
:1069C00010739D4229D8012384F8FE3184F8FF31E9
:1069D0003E4800F065F9054610B1B8F1000F39D016
:1069E000D4F8F031002B4ED1002694F8FF3113B9C2
:1069F0000DB9002EAED02FB194F8FE3113B10123A2
:106A000084F8FF3194F8FF31002B46D10DB9002EE8
:106A1000A0D02046FDF7B0FA9CE794F8FE3103B110
:106A200086B9012384F8FE31A5F51C55103D44F6C6
:106A300020639D4200D91D4667F068FD0544C4F8F7
:106A4000F051C5E7D4F8F061323667F05FFD864259
:106A5000BED2E6E71A4B18681D4A1E4900F52A60A7
:106A6000F9F784FD94F8FE31002BB9D0742200218F
:106A700004F130007FF09AFA002384F8FE310123FC
:106A800084F8FF31ACE767F041FDD4F8F03198426B
:106A900001D90126A9E70026A7E70023C4F8F031B1
:106AA0002046FFF75BFEB1E794F803320BB93220C2
:106AB00034E741F2883031E7A4610020B0B2002011
:106AC000BC7F002044E20B0038C20B00786100203C
:106AD00068E20B0050C60B002DE9F84307460E464E
:106AE00003688046814609E0BB68013BBB602846DD
:106AF00077F096FE284645F083FF23461D469845CD
:106B00000AD01C68996832689142F6D103F10802F4
:106B10009642E9D19946F0E74F4508D0BB68013B62
:106B2000BB60484677F07CFE484645F069FFBDE80B
:106B3000F88310B584B0044601910846039403A974
:106B4000FFF7CAFF01A9201DFFF729FD04B010BD02
:106B500030B583B005460D4B036044682B1D9C4245
:106B600006D0019501A9A068FFF7B6FF2468F5E7F4
:106B70002C1D2046FFF7FDFCAC606C600023EB6031
:106B80002046FFF7F6FC284603B030BDECE20B00D0
:106B900010B50446FFF7DCFF204645F031FF2046E4
:106BA00010BD000010B50446024B0360FFF7D0FF94
:106BB000204610BD00E30B0038B504460B4B0360C4
:106BC00000F502750A492846FFF7B3FF094BC4F8E0
:106BD00008322846FFF7BCFF04F1A800FFF7D4FCF9
:106BE0002046FAF7B7FD204638BD00BFD4E50B00BC
:106BF000C430012000E30B0010B50446FFF7DCFFB2
:106C0000204645F0FDFE204610BD000010B50446AC
:106C1000044B0360FFF79CFF204645F0F1FE204641
:106C200010BD00BF00E30B0010B5044667F06EFC1A
:106C3000206010BD0023036043608360C360704721
:106C400038B5054667F062FC0446094BD86E1B79DF
:106C5000022B09D078211BF002F86A680244EB6825
:106C6000D31A181B02D438BD0249F4E70020FAE712
:106C7000B0B2002080510100026843689A4201D8F6
:106C80000020704710B5044667F040FC2368C01A26
:106C900010BD08B5FFF7D4FFB0FA80F0400908BD79
:106CA00038B50546124B586E1B79022B16D04FF49F
:106CB00061711BF081F80E4B1B79022B11D04FF440
:106CC00061711AF0CCFF0446B0F1FF3F0CD02846AA
:106CD000FFF7D2FFA04209D9012006E04AF6C00121
:106CE000E7E74AF6C001ECE7002038BD0020FCE7EA
:106CF000B0B2002008B5436802689B1A2CD48268A1
:106D0000012A2BD0012A17D9D0ED046A07EE903A58
:106D1000F8EEE77A67EEA67AB7EE007A77EE666A63
:106D200090ED037AB8EE477A27EE267A77EE877AE7
:106D3000FCEEE77AC0ED037A01328260C368084A4C
:106D4000A2FB0323074A10689B09074A074900F57D
:106D50002A60F9F70BFC08BD0023D0E7C360EBE71E
:106D6000D34D6210BC7F00200CE60B00C8BF0B00A7
:106D700010B5044667F0CAFB60602368C31A084870
:106D8000A0FB0323074A10689B09074A074900F53F
:106D90002A60F9F7EBFB2046FFF7ACFF10BD00BF00
:106DA000D34D6210BC7F00202CE60B00C8BF0B0047
:106DB000C06870470023036043608360C360036161
:106DC00043618361C361036243628362C36203639D
:106DD00043638363C363036443648364C3640123C1
:106DE00080F85030704700002DE9D04359EC108BEB
:106DF00057EC116B04460022002310EE100A49469E
:106E00007EF0A2FA00287FD14E23237200220023B5
:106E1000404649467EF098FA002878D149EC108B1C
:106E200078F09AFC51EC100B7EF0F4FAC0B22070AE
:106E30007DF0AEFF02460B46404649467DF05AFEC5
:106E40000022384B7EF00EF88046894649EC108BC4
:106E500078F082FC51EC100B7EF0DCFAC0B260706E
:106E60007DF096FF02460B46404649467DF042FEC5
:106E700000222C4B7DF0F6FF7EF0CCFA6060002201
:106E80000023304639467EF05FFA002843D145237F
:106E9000237400220023304639467EF055FA00283C
:106EA0003CD147EC106B78F057FC51EC100B7EF0A6
:106EB000B1FAC0B260727DF06BFF02460B463046FD
:106EC00039467DF017FE0022164B7DF0CBFF0646BB
:106ED0000F4647EC106B78F03FFC51EC100B7EF046
:106EE00099FAC0B2A0727DF053FF02460B463046BD
:106EF00039467DF0FFFD00220A4B7DF0B3FF7EF0A6
:106F000089FAE060BDE8D083532323727EE709F15C
:106F10000043994682E757232374BAE707F10043F9
:106F20001F46BEE700004E402DE9F84F2DED088BBF
:106F300057EC106B59EC118B55EC124B5BEC13AB0F
:106F400012EE102A2B4610EE100A39467EF0F2F9A6
:106F500040B152465B46404649467EF0EBF9002878
:106F600040F0B5805DA3D3E90023304639467EF07A
:106F7000A3F841EC190B59A3D3E900234046494635
:106F80007EF09AF841EC1B0B54A3D3E90023204672
:106F900029467EF091F841EC180B50A3D3E9002369
:106FA000504659467EF088F841EC1A0BB0EE480A7C
:106FB000F0EE680A78F070F955EC104BB0EE490A23
:106FC000F0EE690A78F068F957EC106BB0EE4B0AF6
:106FD000F0EE6B0A78F060F951EC100B32463B464C
:106FE0007DF040FF22462B467DF03CFF80468946DF
:106FF000B0EE4A0AF0EE6A0A78F04EF953EC102B24
:10700000404649467DF02EFF80468946B0EE4B0A49
:10701000F0EE6B0A78F0C8FC51EC100B32463B46A0
:107020007DF020FF22462B467DF01CFF04460D46D6
:10703000B0EE4A0AF0EE6A0A78F0B6FC53EC102B78
:10704000204629467DF00EFF06460F46B0EE490A5F
:10705000F0EE690A78F0A8FC55EC104BB0EE480A47
:10706000F0EE680A78F0A0FC53EC102B204629467D
:107070007DF0F8FE04460D4632463B464046494602
:107080007DF03AFD22462B467DF036FD41EC100B9B
:1070900078F058FD55EC104B10EE102A2B4610EEF0
:1070A000100A29467EF078F970B90EA3D3E90023BF
:1070B000204629467DF0D6FE7EF0CCF900EE100A7F
:1070C000BDEC088BBDE8F88F00240025EDE79FEDAF
:1070D000020AF5E7AFF3008000000000F8C1631A70
:1070E000DCA54C4000000000CC48584110B50446D7
:1070F0003E4980F0D9F9002856D03D49204680F01D
:10710000D3F9002852D03B49204680F0CDF9002821
:107110004ED03949204680F0C7F900284AD0374977
:10712000204680F0C1F9002846D03549204680F03D
:10713000BBF9002842D03349204680F0B5F9002839
:107140003ED03149204680F0AFF900283AD02F498F
:10715000204680F0A9F9B8B32D49204680F0A4F963
:10716000A0B32C49204680F09FF988B32A492046D5
:1071700080F09AF970B32949204680F095F958B308
:107180002749204680F090F948B32649204680F0F0
:107190008BF938B32449204680F086F908B10020E5
:1071A00003E040F2511000E0002010BD1620FCE783
:1071B0002D20FAE74320F8E75A20F6E77020F4E79D
:1071C0008720F2E79D20F0E7B420EEE7CA20ECE745
:1071D000E120EAE7F720E8E74FF48770E5E74FF4AE
:1071E0009270E2E740F23B10DFE700BF88070C0037
:1071F00044E60B0048E60B004CE60B0060070C0071
:1072000050E60B00309E0C0054E60B0004D90B0036
:1072100058E60B005CE60B0060E60B0064E60B0032
:1072200068E60B006CE60B0070E60B000000000047
:1072300038B52DED028BB0EE408AF0EE608A55EC49
:10724000114B0022002311EE100A29467EF072F83D
:1072500028BB00220023204629467EF093F850B137
:1072600045EC114BB0EE480AF0EE680A78F060FE8B
:10727000BDEC028B38BD224605F1004343EC112BD7
:10728000B0EE480AF0EE680A78F052FE53EC102B8C
:10729000002007497DF010FF41EC100BE8E79FED5F
:1072A000020BE5E7AFF30080000000000000F03FB4
:1072B0000000F03F000000002DE9F04F93B08DED8D
:1072C000020B55EC114B01909D4B0AAE0FCB07C63C
:1072D000338004AE9B4F0FCF0FC697E8030046F8EC
:1072E000040B31700022984BCDE90E230022974BFE
:1072F000CDE9102351EC100B7EF044F808BB10AE22
:107300000022914BD6E900017EF01EF800B90EAEC6
:10731000D6E9006700228C4B304639467EF014F8DF
:1073200088B100228A4B204629467EF00DF818B31A
:107330000022884B204629467DF0DEFB04460D46A0
:10734000EFE702AEDCE79FED721B9FED730BFFF7DB
:107350006FFF51EC100B00227F4B7DF0ADFE002241
:107360007E4B7DF07FFD02460B46304639467DF070
:10737000C1FB06460F46D4E70022794B204629463A
:107380007DF0F6FF40B10022724B204629467DF089
:10739000B1FB04460D46EFE761A3D3E90023304675
:1073A00039467DF05FFD60A3D3E900237DF0A4FBA7
:1073B0007EF02AFA06460F465DA3D3E90023204655
:1073C00029467DF04FFD5CA3D3E900237DF094FBBB
:1073D0007EF01AFA04460D464FF000084FF00B09F4
:1073E0000EE01AF1FF3A6AF0030313F1010A19E003
:1073F000940844EA83749D1008F10108DDF80090B8
:10740000B8F1040F2CD805220023304639467EF00F
:107410007FF904F0030A05F0004BBAF1000F7BF18D
:107420000003DEDB0AEB820209F1FF33009312ABAB
:107430001A4412F8382C4B4403F8202C0522002360
:10744000304639467EF064F906460F4622462B4602
:10745000002C75F10001CBDAE21C45F10003C7E70F
:107460004FF0000A4FF00A0902E00AF1010AD9467A
:10747000BAF1040F3BD814220023304639467EF07F
:1074800047F9904614220023204629467EF040F911
:1074900009F1FF3312A90A4412F8381C12AA4A440F
:1074A00002F8201CA9F1020B12AA904418F8382CFB
:1074B00012A90B4403F8202C14220023304639462D
:1074C0007EF026F906460F46142200232046294660
:1074D0007EF01EF904460D46BAF1000FC5D112AB7D
:1074E0009B442B230BF8203CA9F1030BBDE70023A1
:1074F000019905E012AA1A4412F8202CCA5401334B
:107500000A2BF7D90023019AD37213B0BDE8F08F8C
:1075100000000000000008C000000000000034402F
:107520000000000084D77741000000D088C3E0410C
:107530000000000000405F410000000000F9D5415C
:1075400074E60B0084E60B0000805640008056C0B5
:10755000008066C000807640000014400000E03FDC
:10756000008066400000000008B551EC100B07A336
:10757000D3E900237DF076FC0022034B7DF09CFDD7
:1075800041EC100B08BD00BF00806640182D44542C
:10759000FB210940F8B52DED088B57EC116BB0EECF
:1075A000429AF0EE629A55EC134BFFF7DDFFB0EE16
:1075B000408AF0EE608AB0EE490AF0EE690AFFF701
:1075C000D3FFB0EE409AF0EE609A32463B4620463A
:1075D00029467DF08FFA41EC100BFFF7C5FFB0EEA6
:1075E00040BAF0EE60BA78F0DFF957EC106BB0EE0D
:1075F000490AF0EE690A77F04FFE55EC104B10EE99
:10760000102A2B46304639467DF02CFC41EC1A0BF3
:10761000B0EE480AF0EE680A77F03EFE57EC106BC9
:10762000B0EE490AF0EE690A78F0BEF953EC102B7F
:10763000304639467DF016FC06460F46B0EE480A45
:10764000F0EE680A78F0B0F953EC102B204629468A
:107650007DF008FC04460D46B0EE4B0AF0EE6B0AD6
:1076600077F01AFE53EC102B204629467DF0FAFBEA
:1076700002460B46304639467DF03CFA41EC110B90
:10768000B0EE4A0AF0EE6A0A78F096FA51EC100B66
:107690007DF0E0FE00EE100ABDEC088BF8BD0000A6
:1076A0002DE9F04F2DED048B8BB0B0EE418AF0EE5A
:1076B000618A08900991FFF757FFB0EE409AF0EE0B
:1076C000609AB0EE480AF0EE680AFFF74DFFB0EEA0
:1076D000408AF0EE608AB0EE490AF0EE690A78F06E
:1076E00063F957EC106B9FEDD61B78F021FC51EC41
:1076F000100BF0A3D3E900237DF0B4FB02460B4648
:107700000020EB497DF0F6F941EC100B78F0E2FC3B
:1077100053EC102BCCA1D1E900017DF0CDFC8046CB
:107720008946002200237DF0E7F904460D46B0EEBD
:10773000490AF0EE690A77F0AFFD53EC102B2046B2
:1077400029467DF08FFB04460D46B0EE480AF0EE68
:10775000680A77F0A1FD53EC102B204629467DF0F6
:1077600081FB82468B46B0EE480AF0EE680A78F05C
:107770001BF953EC102B204629467DF073FBCDE915
:107780000001B3A3D3E90023404649467DF06AFBDC
:10779000002200237DF0B0F902460B463046394600
:1077A0007DF060FB804689469FEDAB0BFFF7DCFE6A
:1077B0008DED040B9FEDAA0BFFF7D6FE8DED060BAA
:1077C0009FEDA90BFFF7D0FE55EC104BA8A3D3E912
:1077D0000023504659467DF045FBA7A3D3E900237B
:1077E0007DF088F906460F4622462B46DDE900016A
:1077F0007DF038FB02460B46304639467DF07AF97B
:1078000006460F46DDE90623404649467DF02AFB41
:1078100002460B46304639467DF06EF9CDE902014D
:1078200022462B46504659467DF01CFB94A3D3E9D3
:1078300000237DF061F904460D468DA3D3E90023B2
:10784000DDE900017DF00EFB02460B46204629468D
:107850007DF052F904460D46DDE9042340464946D1
:107860007DF000FB02460B46204629467DF042F99A
:1078700006460F46DDE90623504659467DF0F2FAEA
:1078800002460B4680A1D1E900017DF033F90446A0
:107890000D46DDE90423DDE900017DF0E3FA02464F
:1078A0000B46204629467DF027F904460D4670A375
:1078B000D3E90023404649467DF0D4FA02460B4600
:1078C000204629467DF018F982468B46DDE90245BF
:1078D00022462B46204629467DF0C4FA04460D4632
:1078E00032463B46CDE90067304639467DF0BAFA6C
:1078F00002460B46204629467DF0FEF841EC100B6F
:1079000078F0E8FB55EC104B10EE102A2B4610EEE9
:10791000100A29467DF0A6FA06460F4652465B46F7
:10792000504659467DF09EFA02460B46304639468F
:107930007DF0E2F841EC100B78F0CCFB59EC108BA9
:1079400053A3D3E90023504659467DF08BFA0646EF
:107950000F4651A3D3E90023204629467DF082FA41
:1079600002460B46304639467DF0A6FB06460F46DA
:1079700042464B464AA1D1E900017DF09DFB002221
:107980004B4B7DF0B9F802460B46304639467DF048
:1079900069FA06460F4602460B467DF063FA00225E
:1079A000434B7DF0A9F841EC100B78F093FB53ECBE
:1079B000102B304639467DF07FFB804689463246A3
:1079C0003B467DF079FB06460F4635A3D3E90023FD
:1079D000404649467DF046FA42464B467DF042FA23
:1079E00042464B467DF03EFA804689462EA3D3E9B7
:1079F0000023304639467DF035FA32463B467DF06D
:107A000031FA32463B467DF02DFA02460B462046BF
:107A100029467DF06FF841EC180B52465B46404614
:107A200049467DF069F8B0EE481AF0EE681A41EC6C
:107A3000100B78F0C1F8089B40E000BFAFF3008066
:107A4000000000000000004000000040A654584123
:107A5000D6021CDE28C9EF3FD688C2A3DCDF05BFF3
:107A6000725ED8E969FC11BFF377DCDDF0A82EBFA8
:107A7000BDD8147C1500F03FBA490C022BE77B40BF
:107A8000355EBA490C4A5F4014AE47E17AF080C0D7
:107A9000560E2D3A483F5841621058D91654584155
:107AA000A457FB9A8CD7E440BD9AE555B9C5E4408C
:107AB0000000F03FF094FEF1906B7B3F83ED000BF4
:107AC0009DED021B9DED000B78F076F8099B83ED90
:107AD000000B0BB0BDEC048BBDE8F08F0000000084
:107AE0002DE9F04F2DED068BA7B0B0EE408AF0EEF9
:107AF000608AB0EE419AF0EE619A0D901FACDC4DB9
:107B00000FCD0FC495E8070003C422809FEDC00B82
:107B1000FFF72AFD55EC104B9FEDBF0BFFF724FD3F
:107B20008DED0A0B1AA91CA8B0EE491AF0EE691ADD
:107B3000B0EE480AF0EE680AFFF7B2FD9DED1C8B2F
:107B40009DED1AABB0EE480AF0EE680A77F02CFF14
:107B500057EC106BB2A3D3E9002310EE100A39469C
:107B60007DF080F902460B46CDE900673046394684
:107B70007DF078F902460B460020BE497CF0BAFF42
:107B800041EC190B41EC100B78F0A4FA53EC102BDC
:107B9000A5A1D1E900017DF08FFA804689469FEDCD
:107BA000A41BB0EE490AF0EE690A78F0C1F953EC73
:107BB000102BA1A1D1E900017DF07EFA02460B460F
:107BC000404649467DF078FA02460B46CDE90E2341
:107BD0000022A84B7CF08EFFCDE9020122462B4605
:107BE00051EC180B7CF086FF06460F4694A3D3E9B0
:107BF00000237DF037F9CDE9040147EC106B77F0F5
:107C0000D3FE51EC100B90A3D3E900237DF02AF9A9
:107C100082468B4653EC182B204629467CF06CFF9D
:107C200004460D4645EC104B77F036FB53EC102B19
:107C3000504659467DF016F982468B4632463B4601
:107C4000304639467CF058FF41EC100B77F0ACFE23
:107C500051EC100B7EA3D3E900237DF003F9CDE9AD
:107C6000060122462B46204629467CF045FF41EC82
:107C7000100B77F011FB53EC102BDDE906017DF0C2
:107C8000F1F8CDE9060100227B4B304639467DF004
:107C9000E9F841EC100B77F087FE51EC100B6EA366
:107CA000D3E900237DF0DEF806460F460022724B32
:107CB000204629467DF0D6F841EC100B77F0ECFA1F
:107CC00053EC102B304639467DF0CCF804460D4677
:107CD00052465B46DDE904017CF00CFFDDE906233A
:107CE0007CF00AFF22462B467CF004FF5CA3D3E91C
:107CF00000237DF0B7F806460F46B0EE480AF0EED6
:107D0000680A77F0C9FA55EC104B10EE102A2B4692
:107D100010EE100A29467DF0A5F802460B462046D3
:107D200029467DF09FF80A460146CDE90412134624
:107D30000246204629467DF095F802460B4620462D
:107D400029467DF08FF8CDE90601B0EE480AF0EE45
:107D5000680A77F081FE51EC100B10EE102A0B46EA
:107D60007DF080F882468B4602460B467DF07AF81D
:107D7000CDE908013CA3D3E90023304639467CF025
:107D8000B9FECDE9100100223C4B404649467DF04A
:107D900069F802460B46DDE90067304639467DF05A
:107DA00061F802460B46204629467DF05BF8CDE996
:107DB00012010022324B404649467DF07DF90246D1
:107DC0000B46CDE90067304639467DF04BF8DDE9DA
:107DD00004237DF047F806460F4652465B460020D6
:107DE00028497CF087FECDE914010022264BDDE90D
:107DF00002017DF037F802460B46DDE914017CF004
:107E00007BFE02460B46304639467DF02BF83DE0BE
:107E1000000000000080484000000000000000C09A
:107E2000002A717791527B3FF785C81E9B515841BC
:107E3000000000000000F83F187DB0E91328584109
:107E400096FC7270DD06F03FC1E30B175098743F4B
:107E500009CFE71D4C86C73EBDE60CDA9D1E343EB9
:107E6000C8C6539FCE3C584100000000006AF8404D
:107E70009CE60B000000F03F000008400000E03FDF
:107E8000000038400000144000002240CDE91401F9
:107E900000229F4B404649467DF00EF902460B46B4
:107EA000DDE900017CF0DEFFDDE906237CF0DAFF8E
:107EB00006460F460022974B504659467CF0D2FFAB
:107EC0000A460146CDE900121346024600209249B7
:107ED0007CF010FEDDE908237CF00EFE02460B4626
:107EE000304639467CF0BEFFCDE9160142464B468E
:107EF000204629467CF0B6FFCDE918010022874BC9
:107F0000404649467DF0D8F8DDE904237CF0AAFF1D
:107F100004460D4652465B46DDE90E017CF0EAFD63
:107F200002460B46204629467CF09CFFCDE9040121
:107F300000227B4B404649467DF0BEF8DDE9062332
:107F40007CF090FF04460D460022764B5046594681
:107F50007CF088FF02460B46002073497CF0CAFD86
:107F6000DDE908237CF0C8FD06460F4600226F4B72
:107F7000DDE90289404649467CF074FF02460B4623
:107F8000304639467CF0B8FD06460F4642464B4621
:107F9000DDE900017CF066FF02460B4630463946BB
:107FA0007CF0A8FD02460B46204629467CF05AFF8D
:107FB00082468B46DDE90A2351EC1A0B7CF09AFDD0
:107FC00006460F4602460B467CF04CFF04460D4623
:107FD00002460B46DDE912017CF044FFDDE9102387
:107FE0007CF08AFD8046894622462B46DDE9140155
:107FF0007CF038FF22462B467CF034FF02460B46CD
:10800000404649467CF078FD8046894622462B460C
:10801000DDE916017CF026FF22462B467CF022FF8C
:1080200022462B467CF01EFF02460B464046494640
:108030007CF062FDCDE9000132463B46DDE91801E6
:108040007CF010FF2CA3D3E900237CF055FD804683
:10805000894622462B46DDE904017CF003FF3246C7
:108060003B467CF0FFFE02460B46404649467CF00C
:1080700043FD8046894622462B46504659467CF0B1
:10808000F1FE22462B467CF0EDFE32463B467CF06C
:10809000E9FE02460B46404649467CF02DFD04466B
:1080A0000D46002200237DF04FF9C0B914A3D3E997
:1080B0000023204629467DF065F980B9002200237F
:1080C000DDE90067304639467DF03EF938B90EA348
:1080D000D3E90023304639467DF054F950B3144BB0
:1080E00093E807000D9B83E8070027B0BDEC068BE3
:1080F000BDE8F08FAFF3008000000000006A184177
:1081000000000000C05C25410000000020D6334183
:108110000080864000004D4000804E400000184026
:1081200000005E40000032400000144000002C407F
:1081300024E70B0043A3D3E90023204629467CF023
:10814000BBFF41EC100B77F007FB51EC100B7DF0FF
:1081500061F982463BA3D3E90023DDE900017CF00D
:10816000ABFF41EC100B77F0F7FA51EC100B7DF000
:1081700051F90646C0F11307DFF8D0B0ABFB073268
:1081800022F0030303EB9203FF1A0744C7F113071E
:108190000AF10A00ABFB003080087CF0E9FD804664
:1081A000894638467CF0E4FD42464B467CF0A4FC10
:1081B0007DF008F9C6EB8673C6EB83065F361E4B6F
:1081C000A3FB0623DB0803EB830303EB8303F31A10
:1081D000ABFB0A2B2BF0030202EB9B0BAAEB0B0A67
:1081E000534426AA42FA80F010F81C2C0D9E3270DF
:1081F00026AA42FA83F313F81C3C737020462946E2
:108200007DF0E0F80D4D85FB0032C317C3EB623300
:108210000B4C04FB13037360DDE900017DF0D2F821
:1082200085FB0035C317C3EB653304FB1303B36051
:108230005BE700BFAFF300801F85EB5189B5F814F1
:10824000A086010000000000006AF840CDCCCCCC34
:1082500008B551EC100B0022074B7CF003FE04A381
:10826000D3E900237CF028FF41EC100B08BD00BFD0
:10827000182D4454FB210940008066400000000096
:108280002DE9F04F2DED028B97B059EC108B8DED51
:10829000020B57EC116B044612AB1093D84A4FF007
:1082A0000003A2F1150110A8F8F7B2F90022D54B8E
:1082B000304639467CF020FC06460F460022D24B61
:1082C0007CF0FAFE0022D14B7CF016FC7DF07AF8AF
:1082D000207000224FF07F53404649467CF0C2FD9B
:1082E0000022CB4B7CF008FC7DF06CF8109B1B5CF3
:1082F00063700022C74B304639467CF0DDFE7DF0CE
:1083000061F84FF4B47303FB00F07CF041FD0246CA
:108310000B46304639467CF0EDFB0022B94B7CF031
:10832000E9FB06460F4649EC108BFFF71DF9B0EE4E
:10833000408AF0EE608A47EC106BFFF715F98DED7F
:10834000080B0022B44B404649467DF011F8B0B10D
:108350000022B24B404649467CF0F6FF78B100223D
:10836000AF4B304639467DF003F840B10022AD4BAB
:10837000304639467CF0E8FF08B120232370002204
:10838000A94BDDE90289404649467CF0F1FFD0B1B6
:108390000022A64B404649467CF0D6FF98B1002209
:1083A0000023304639467CF0E3FF002800F0648269
:1083B00000229F4B304639467CF0C6FF002800F073
:1083C0005B821F2323702078013800EB40004000BF
:1083D000B1387CF0DDFC41EC100BFFF7C5F859EC2F
:1083E000108BB0EE480AF0EE680A77F0DDFA57EC31
:1083F000106B71A3D3E9002310EE100A39467CF00C
:1084000031FD02460B46304639467CF02BFD0246D4
:108410000B4600207D497CF06DFB41EC100B77F0A2
:1084200059FE53EC102B66A1D1E900017CF044FE0B
:10843000CDE90401B0EE480AF0EE680A77F00CFBD3
:1084400056EC105B10EE102A33468DED060B10EE45
:10845000100A31467CF006FDCDE90001B0EE480A75
:10846000F0EE680A76F018FF57EC106B56A3D3E9CC
:10847000002310EE100A39467CF0F4FC02460B464D
:10848000304639467CF0EEFC82468B4642464B46EF
:10849000DDE908017CF02EFB02460B4630463946EA
:1084A0007CF0E0FC06460F4649A3D3E9002351ECDB
:1084B000180B7CF0D7FC8046894653EC182B51EC06
:1084C000180B7CF019FB41EC100B77F06DFA51ECB6
:1084D000100B41A3D3E900237CF0C4FC02460B46F9
:1084E000404649467CF006FB804689460022514BB7
:1084F00051EC180B7CF0B6FC41EC100B77F054FA01
:1085000051EC100B36A3D3E900237CF0ABFC024600
:108510000B46404649467CF0EFFA804689460022E9
:10852000394B51EC180B7CF09DFC41EC100B77F0B3
:108530003BFA51EC100B2CA3D3E900237CF092FC06
:1085400002460B46404649467CF0D4FA1CA3D3E9C8
:1085500000237CF087FCCDE9080125A3D3E90023A3
:10856000DDE904017CF07EFCCDE90A01DDE90023B0
:10857000002026497CF0BEFA52465B467CF0BCFAED
:10858000804689469FED1C1B47EC106B77F0D0FCB2
:1085900053EC102B404649467CF064FC00221A4BF9
:1085A0007CF08AFD32463B467CF0A6FACDE90C0110
:1085B0000022214B42E000BF8004ACF2906B7B3F75
:1085C00000000040A6545841DDA447E2DF9A7B3FFB
:1085D00061AE94CC45F2EF3F2C024D638399643F2A
:1085E0004ABA6F364F23C63EFC48CCE45C5C2D3E55
:1085F000789CA223B9FCEF3F000000000000084077
:10860000CDE60B0000806640000018400000F03FFF
:10861000000024400080764000004C4000005040A4
:108620000000084000002840000052400000554073
:10863000000022400000104000003240DDE900014F
:108640007CF010FC02460B460020B7497CF052FA41
:1086500080468946DDE9000102460B467CF002FCBB
:108660000A460146CDE90E121346024640464946E7
:108670007CF042FA804689460022AC4B504659466F
:108680007CF0F0FB02460B46404649467CF034FA4B
:108690009BA3D3E900237CF02DFA32463B467CF0C5
:1086A000E1FB32463B467CF0DDFB32463B467CF04C
:1086B000D9FB32463B467CF0D5FB32463B467CF04C
:1086C000D1FB00229A4B7CF0F7FC02460B46DDE919
:1086D0000C017CF011FA02460B46DDE90A017CF040
:1086E000C1FB89A3D3E900237CF006FA7CF092FE5B
:1086F0006060DDE90423DDE906017CF0B3FBCDE930
:10870000040132463B46304639467CF0ABFB002242
:10871000884B7CF0A7FBCDE90601DDE900230020B2
:1087200081497CF0E7F9804689460022824B504619
:1087300059467CF097FB02460B46404649467CF082
:10874000DBF98046894600227C4B504659467CF036
:1087500089FB52465B467CF085FB02460B46404651
:1087600049467CF0C9F932463B467CF07BFB3246F9
:108770003B467CF077FB32463B467CF073FB32464F
:108780003B467CF06FFB00226D4B7CF095FC024673
:108790000B46DDE906017CF0AFF9CDE906010022C8
:1087A000684BDDE900017CF05DFB02460B460020D2
:1087B00065497CF09FF902460B46DDE90E017CF02D
:1087C0009BF9804689460022604B504659467CF012
:1087D00049FB02460B46404649467CF08DF94CA3C6
:1087E000D3E900237CF086F932463B467CF03AFB25
:1087F00032463B467CF036FB32463B467CF032FB51
:1088000032463B467CF02EFB32463B467CF02AFB50
:1088100032463B467CF026FB00224D4B7CF04CFC64
:1088200002460B46DDE906017CF066F902460B467E
:10883000DDE904017CF016FBDDE908237CF05CF93E
:1088400035A3D3E900237CF00DFB7CF0E3FD054666
:10885000A06000220023DDE902017CF075FD002804
:1088600041D1109812AB984201D044F0C9F817B02A
:10887000BDEC028BBDE8F08F00222F4B304639460D
:108880007CF076FD48B10022324B304639467CF010
:108890005BFD10B12123237095E500222D4B30465E
:1088A00039467CF065FD48B100222B4B30463946F5
:1088B0007CF04AFD10B12323237084E50022264B6F
:1088C000304639467CF054FD00283FF47CAD002250
:1088D000224B304639467CF037FD00283FF473AD1B
:1088E000252323706FE528467CF042FA0CA3D3E9D8
:1088F00000237CF001F97CF08DFDA060B1E700BFA2
:1089000068ED10E55A04D93F0000000080841E4144
:10891000422DD84CD2CA0140789CA223B9FCEF3F2B
:1089200000000000D01263410000144000005240DB
:1089300000005E400000E03F0000224000001040C8
:108940000000384000004D4000804E4000C0824092
:1089500000808640000035400080404000004540D7
:10896000F0B52DED048BA3B0B0EE408AF0EE608A36
:10897000B0EE419AF0EE619A064612AB1093604A4F
:108980004FF00003A2F1080110A8F7F741FE18AB61
:1089900016935C4A4FF00003A2F1080116A8F7F7FE
:1089A00037FE1EAB1C93584A4FF00003A2F108019A
:1089B0001CA8F7F72DFE06AB0493544A4FF00003B2
:1089C000A2F1140104A8F7F723FE0CAB0A93504A56
:1089D0004FF00003A2F114010AA8F7F719FE01A84D
:1089E000B0EE491AF0EE691AB0EE480AF0EE680AE5
:1089F000FFF746FC9DF8044034709DF80530737015
:108A0000029F7809434BA3FB0030C0097CF0B0F90A
:108A1000013C414D85FB0435A5EBE47505EB4505AF
:108A2000651B00223D4B7CF065F87CF0F3FC05EB08
:108A3000450522AB03EBC50555F8483C1B5CB370FC
:108A4000039D28467CF094F92BA3D3E900237CF006
:108A500033FB41EC100B76F07FFE51EC100B7CF0F9
:108A6000B1FC2F4A82FB0032C317C3EBE20303EBD6
:108A70008303A0EB8303002C04F00104B8BF64421D
:108A800004EB440422AA02EBC40454F8782CD35C0F
:108A9000F370244B83FB0721FA17C2EB61322249A2
:108AA00001FB1272726083FB0532EB17C3EB62337A
:108AB00001FB1353B36010AC04AB9C4208D0183CCC
:108AC000234653F8080B8342F6D043F099FFF3E7AF
:108AD00022AC10AB9C4208D0183C234653F8080B3C
:108AE0008342F6D043F08CFFF3E723B0BDEC048B58
:108AF000F0BD00BFAFF3008000000000006AF84046
:108B0000D8E60B00E4E60B00F0E60B0008E70B00EC
:108B100020E70B00C55A7C0A565555550000F03F1A
:108B20006766666689B5F814A0860100000000003B
:108B300010B52DED048B044600687CF029F92AA3BA
:108B4000D3E900237CF08EF941EC180B60687CF0CF
:108B50001FF925A3D3E900237CF084F941EC190B1C
:108B600004F10C00B0EE491AF0EE691AB0EE480AB2
:108B7000F0EE680AFEF738F904F12000B0EE491A69
:108B8000F0EE691AB0EE480AF0EE680AFFF778FBDB
:108B900004F12C00B0EE491AF0EE691AB0EE480A62
:108BA000F0EE680AFFF7DCFE04F13800B0EE491A77
:108BB000F0EE691AB0EE480AF0EE680AFEF790FF90
:108BC00004F14400B0EE491AF0EE691AB0EE480A1A
:108BD000F0EE680AFEF770FB002384F85030BDEC1D
:108BE000048B10BDAFF3008048AFBC9AF2D77A3E39
:108BF00010B504460160426083600023C3600361D6
